:100000000C94F4500C9425510C9425510C942551CA
:100010000C9425510C9425510C9425510C94255188
:100020000C9425510C9425510C9425510C94255178
:100030000C94D7840C9425510D94AF100D94F30DAE
:100040000C9425510D941D190C9425510C94255197
:100050000C9425510C9425510C9425510C94B37695
:100060000C9425510C9432630C9425510C94255119
:100070000C9425510C9442BA0C9425510C942551A2
:100080000D94F9120C9425510C9425510C94255182
:100090000C94EE620C9425510C9425510C9425512E
:1000A0000C9425510C9425510D94180B0C9425514A
:1000B0000C9425510D940D0B0C9425510C94255145
:1000C0000C9425510C9425510C9425510D94CD0A76
:1000D0000C9425510C9425510C9425510C942551C8
:1000E0000C942551000000000000000000000000FA
:1000F0000000000000000000000000000000000000
:100100005F5345435F4C414E470000000000000034
:1001100000000000000000000000000000000000DF
:1001200000000000000000000000000000000000CF
:1001300000000000000000000000000000000000BF
:1001400000000000000000000000000000000000AF
:103600000000536F6D652070726F626C656D206590
:103610006E636F756E74657265642C205A2D6C65CF
:1036200076656C696E6720656E666F72636564208F
:103630002E2E2E0001004D65736820626564206C9B
:103640006576656C696E67206661696C65642E20BD
:103650005072696E742063616E63656C65642E00E0
:10366000020048656174696E672064697361626C09
:103670006564206279207361666574792074696D70
:1036800065722E000300472D636F646520736C69BB
:1036900063656420666F7220612064696666657286
:1036A000656E74206C6576656C2E000400472D6392
:1036B0006F646520736C6963656420666F72206156
:1036C00020646966666572656E74206C6576656CEB
:1036D0002E20506C656173652072652D736C696373
:1036E0006520746865206D6F64656C206167616931
:1036F0006E2E000500472D636F646520736C69634F
:10370000656420666F722061206E65776572206641
:1037100069726D776172652E000600472D636F64D4
:103720006520736C6963656420666F722061206E2A
:1037300065776572206669726D776172652E2050BB
:103740006C6561736520757064617465207468656B
:10375000206669726D776172652E000700472D63E0
:103760006F646520736C6963656420666F722061A5
:1037700020646966666572656E74207072696E7425
:10378000657220747970652E000800472D636F64A0
:103790006520736C6963656420666F7220612064C4
:1037A0006966666572656E74207072696E746572A2
:1037B00020747970652E20506C6561736520726588
:1037C0002D736C69636520746865206D6F64656C2A
:1037D00020616761696E2E00090050726573732065
:1037E000746865206B6E6F6220746F2070726568FC
:1037F000656174206E6F7A7A6C6520616E642063F7
:103800006F6E74696E75652E000A00506C65617389
:103810006520707265737320746865206B6E6F62CB
:1038200020746F20756E6C6F61642066696C616DC9
:10383000656E74000B00616E642070726573732096
:10384000746865206B6E6F62000C00496E73657260
:10385000742066696C616D656E74000D00436F6C59
:103860006F72206E6F7420636F7272656374000EE6
:103870000046696C616D656E74206E6F74206C6FAC
:1038800061646564000F004368616E67656420636E
:103890006F72726563746C790010004C6F616469BB
:1038A0006E6720636F6C6F720011004368616E6712
:1038B00065207375636365737321001200506C6536
:1038C000617365206F70656E2069646C657220613C
:1038D0006E642072656D6F76652066696C616D65DA
:1038E0006E74206D616E75616C6C792E00130057DB
:1038F00061732066696C616D656E7420756E6C6FA6
:103900006164207375636365737366756C3F00143F
:1039100000506C6561736520757067726164652E17
:103920000015004E6577206669726D7761726520BB
:1039300076657273696F6E20617661696C61626C25
:10394000653A00160057616974696E6720666F7288
:103950002050494E44412070726F626520636F6F42
:103960006C696E67001700506C6561736520776144
:1039700069740018004E6F206D6F76652E00190077
:103980005761697420666F7220757365722E2E2ED2
:10399000001A00537461626C6520616D6269656E26
:1039A000742074656D706572617475726520323152
:1039B0002D323643206973206E656564656420612D
:1039C000207269676964207374616E642069732072
:1039D00072657175697265642E001B00506C6561BB
:1039E00073652072756E2058595A2063616C696244
:1039F000726174696F6E2066697273742E001C00A8
:103A00005072656865617420746865206E6F7A7A9B
:103A10006C6521001D004552524F523A001E00595C
:103A20002064697374616E63652066726F6D206DCA
:103A3000696E001F004C656674002000526967685B
:103A4000740021004D6561737572656420736B6548
:103A500077002200536C6967687420736B65770088
:103A6000230053657665726520736B6577002400CB
:103A70005B303B305D20706F696E74206F666673DB
:103A8000657400250041646A757374696E67205A15
:103A9000002600526561722073696465205BE46DE5
:103AA0005D00270046726F6E7420736964655BE485
:103AB0006D5D002800526967687420736964655BF6
:103AC000E46D5D0029004C656674207369646520AF
:103AD0005BE46D5D002A005365742074656D70654C
:103AE0007261747572653A002B00417265206C65D5
:103AF000667420616E64207269676874205A2D6351
:103B0000617272696167657320616C6C2075703FCA
:103B1000002C0043616C6962726174696E672058A1
:103B2000595A2E20526F7461746520746865206B39
:103B30006E6F6220746F206D6F76652074686520EB
:103B40005A20636172726961676520757020746FB5
:103B50002074686520656E642073746F7070657280
:103B6000732E20436C69636B207768656E20646FE9
:103B70006E652E002D0043616C6962726174696E1E
:103B800067205A2E20526F74617465207468652016
:103B90006B6E6F6220746F206D6F76652074686540
:103BA000205A2063617272696167652075702074A4
:103BB0006F2074686520656E642073746F70706523
:103BC00072732E20436C69636B207768656E206486
:103BD0006F6E652E002E0050494E44412063616C8B
:103BE0006962726174696F6E206661696C656400F8
:103BF0002F0050494E44412063616C6962726174C8
:103C0000696F6E2069732066696E697368656420E8
:103C1000616E64206163746976652E204974206347
:103C2000616E2062652064697361626C65642069FD
:103C30006E206D656E752053657474696E67732DA3
:103C40003E50494E44412063616C2E00300045785F
:103C50007472756465720031004D6F7665205A008C
:103C600032004D6F766520590033004D6F76652028
:103C700058003400536865657420252E37730A5A3E
:103C8000206F66667365743A20252B312E33666D7E
:103C90006D0A2563436F6E74696E75650A256352FC
:103CA00065736574003500506C65617365206C6FD9
:103CB00061642066696C616D656E742066697273FB
:103CC000742E00360053656C6563742066696C6100
:103CD0006D656E743A00370043616E63656C003841
:103CE0000052756E6E696E672057697A6172642042
:103CF00077696C6C2064656C65746520637572729D
:103D0000656E742063616C6962726174696F6E20A4
:103D1000726573756C747320616E64207374617264
:103D2000742066726F6D2074686520626567696EC5
:103D30006E696E672E00390050726568656174693E
:103D40006E67206E6F7A7A6C652E20506C65617399
:103D50006520776169742E003A00506C6561736567
:103D600020696E736572742066696C616D656E742E
:103D700020696E746F20746865206578747275644C
:103D800065722C207468656E207072657373207480
:103D90006865206B6E6F6220746F206C6F616420A9
:103DA00069742E003B00506C6561736520696E7309
:103DB0006572742066696C616D656E7420696E74DD
:103DC0006F2074686520666972737420747562650B
:103DD000206F6620746865204D4D552C20746865F1
:103DE0006E20707265737320746865206B6E6F62ED
:103DF00020746F206C6F61642069742E003C005445
:103E00006865207072696E7465722077696C6C20C9
:103E10007374617274207072696E74696E67206168
:103E2000207A69672D7A6167206C696E652E205251
:103E30006F7461746520746865206B6E6F622075A5
:103E40006E74696C20796F75207265616368207487
:103E50006865206F7074696D616C2068656967685A
:103E6000742E20436865636B2074686520706963F5
:103E7000747572657320696E207468652068616E60
:103E800064626F6F6B202843616C69627261746950
:103E90006F6E2063686170746572292E003D005357
:103EA000656C6563742074656D706572617475729C
:103EB00065207768696368206D6174636865732045
:103EC000796F7572206D6174657269616C2E003E48
:103ED0000053656C65637420612066696C616D6573
:103EE0006E7420666F722074686520466972737400
:103EF000204C617965722043616C696272617469FA
:103F00006F6E20616E642073656C656374206974E4
:103F100020696E20746865206F6E2D73637265650D
:103F20006E206D656E752E003F004E6F7720492024
:103F300077696C6C2063616C69627261746520647E
:103F4000697374616E6365206265747765656E2060
:103F5000746970206F6620746865206E6F7A7A6C61
:103F60006520616E642068656174626564207375A4
:103F700072666163652E0040005A2063616C69625D
:103F8000726174696F6E207265636F6D6D656E64CA
:103F900065642E2052756E206974206E6F773F0025
:103FA0004100506C656173652072656D6F766520A8
:103FB000737465656C2073686565742066726F6DD7
:103FC00020686561746265642E0042004973207345
:103FD0007465656C207368656574206F6E20686514
:103FE00061746265643F004300506C6561736520D5
:103FF000636865636B206F75722068616E64626FC1
:104000006F6B20616E64206669782074686520702B
:10401000726F626C656D2E205468656E20726573D8
:10402000756D65207468652057697A6172642062D5
:1040300079207265626F6F74696E6720746865209D
:104040007072696E7465722E004400416C6C206958
:104050007320646F6E652E204861707079207072D5
:10406000696E74696E6721004500596F7520636140
:104070006E20616C7761797320726573756D652050
:104080007468652057697A6172642066726F6D206A
:1040900043616C6962726174696F6E202D3E2057B6
:1040A000697A6172642E004600496620796F752036
:1040B00068617665206164646974696F6E616C2003
:1040C000737465656C207368656574732C20636117
:1040D0006C696272617465207468656972207072BF
:1040E000657365747320696E2053657474696E67B7
:1040F00073202D204857205365747570202D205350
:104100007465656C207368656574732E0047005094
:104110006C6561736520636C65616E2068656174B0
:1041200062656420616E64207468656E20707265DB
:10413000737320746865206B6E6F622E00480044B4
:104140006F20796F752077616E7420746F207265AF
:1041500070656174206C6173742073746570207471
:104160006F20726561646A75737420646973746129
:104170006E6365206265747765656E206E6F7A7A0E
:104180006C6520616E6420686561746265643F00DF
:10419000490053656C656374206E6F7A7A6C652094
:1041A000707265686561742074656D7065726174A4
:1041B000757265207768696368206D6174636865EE
:1041C0007320796F7572206D6174657269616C2EF0
:1041D000004A0049732066696C616D656E74206CDD
:1041E0006F616465643F004B004E6F772049207714
:1041F000696C6C2070726568656174206E6F7A7A84
:104200006C6520666F7220504C412E004C00492096
:1042100077696C6C2072756E207A2063616C6962BC
:10422000726174696F6E206E6F772E004D004E6F55
:10423000772072656D6F766520746865207465738C
:1042400074207072696E742066726F6D207374656D
:10425000656C2073686565742E004E00506C656156
:1042600073652072656D6F7665207368697070691B
:104270006E672068656C706572732066697273740E
:104280002E004F00492077696C6C2072756E207883
:10429000797A2063616C6962726174696F6E206EF5
:1042A0006F772E2049742077696C6C2074616B6580
:1042B00020757020746F203234206D696E732E006B
:1042C000500046697273742C20492077696C6C2009
:1042D00072756E207468652073656C66746573749E
:1042E00020746F20636865636B206D6F7374206347
:1042F0006F6D6D6F6E20617373656D626C79207088
:10430000726F626C656D732E00510048692C2049F4
:1043100020616D20796F7572204F726967696E61D7
:104320006C205072757361206933207072696E74ED
:1043300065722E20576F756C6420796F75206C69DB
:104340006B65206D6520746F2067756964652079E1
:104350006F75207468726F75676820746865207364
:10436000657475702070726F636573733F005200DF
:1043700048692C204920616D20796F7572204F7239
:104380006967696E616C20507275736120693320B2
:104390007072696E7465722E20492077696C6C208A
:1043A000677569646520796F75207468726F7567C9
:1043B0006820612073686F72742073657475702053
:1043C00070726F636573732C20696E207768696300
:1043D0006820746865205A2D617869732077696C4C
:1043E0006C2062652063616C696272617465642E21
:1043F000205468656E2C20796F752077696C6C206D
:10440000626520726561647920746F207072696ED4
:10441000742E00530050617573650054004653209C
:10442000416374696F6E005500436F6E742E0056C1
:1044300000462E206A616D206465746563740057C0
:1044400000462E206175746F6C6F616400580046E1
:104450002E2072756E6F7574005900437574746503
:1044600072005A0046616E207370656564005B00DF
:10447000426564005C0046616E7320636865636B2F
:10448000005D004D6F64656C005E004E6F7A7A6C63
:1044900065005F00506C6561736520756E6C6F61BF
:1044A00064207468652066696C616D656E74206651
:1044B000697273742C207468656E20726570656112
:1044C00074207468697320616374696F6E2E006074
:1044D00000436865636B730061004E6F7A7A6C65A8
:1044E00020642E006200416C706861626574006334
:1044F00000536F727400640054696D650065004E6E
:104500006F726D616C0066005344206361726400D9
:10451000670053656C656374206C616E67756167D5
:10452000650068004E6F7A7A6C65206368616E671B
:10453000650069004857205365747570006A004C27
:104540006F6164696E672054657374006B00446921
:104550007361626C65207374657070657273006C52
:10456000004D6F76652061786973006D0054656D4C
:104570007065726174757265006E0050494E4441F9
:104580002063616C2E006F0052657365742058596A
:104590005A2063616C6962722E00700053686F77F5
:1045A00020656E642073746F70730071005049440D
:1045B0002063616C6962726174696F6E007200429F
:1045C0006564206C6576656C20636F7272656374D8
:1045D0000073004D65736820426564204C65766504
:1045E0006C696E6700740043616C69627261746526
:1045F000205A00750043616C6962726174652058CD
:10460000595A00760053656C6674657374007700C0
:1046100057697A61726400780054657374696E67D3
:104620002066696C616D656E740079004C6F616421
:1046300020416C6C007A00506C6561736520707568
:104640006C6C206F75742066696C616D656E74208A
:10465000696D6D6564696174656C79007B00526594
:10466000736574007C0052656E616D65007D004667
:1046700069727374206C617965722063616C2E00BD
:104680007E0053656C656374007F00537465656CD0
:1046900020736865657473008000537570706F7265
:1046A000740081004661696C207374617473204DDD
:1046B0004D550082004661696C207374617473000B
:1046C0008300537461746973746963730084004375
:1046D000616C6962726174696F6E00850041757406
:1046E0006F4C6F61642066696C616D656E740086E5
:1046F000004C6F61642066696C616D656E74008743
:1047000000556E6C6F61642066696C616D656E74D6
:104710000088004C6F616420746F206E6F7A7A6C31
:10472000650089005072656C6F616420746F204D64
:104730004D55008A004E6F2053442063617264001F
:104740008B005072696E742066726F6D2053440046
:104750008C00526573756D65207072696E74008D82
:10476000005061757365207072696E74008E00531D
:104770006574205265616479008F00536574206E02
:104780006F742052656164790090005072656865AD
:10479000617400910054756E650092004C697665F5
:1047A0002061646A757374205A00930052657072B8
:1047B000696E74009400496E666F2073637265655C
:1047C0006E0095004173736973740096004F6E63B9
:1047D00065009700536F756E640098004C6F7564A8
:1047E00000990046696C2E2073656E736F72009A93
:1047F000004368616E67652066696C616D656E7403
:10480000009B00466C6F77009C00537065656400E8
:104810009D004D61676E65747320636F6D702E002F
:104820009E004E2F41009F005A2D70726F626520CE
:104830006E722E00A0004D65736800A10053657470
:1048400074696E677300A20059657300A3004E6F10
:1048500000A40053746F70207072696E7400A5001C
:10486000436865636B696E672066696C6500A600C6
:1048700046696C6520696E636F6D706C6574652E3A
:1048800000A700845265667265736800A8004D61D8
:10489000696E00A90057616974696E6720666F725E
:1048A000206E6F7A7A6C6520616E64206265642088
:1048B000636F6F6C696E6700AA0053656C66746500
:1048C0007374204F4B00AB0053656C667465737452
:1048D00020737461727400AC00537761707065640A
:1048E00000AD0046726F6E742F6C65667420666151
:1048F0006E7300AE004178697300AF004178697350
:10490000206C656E67746800B0004C6F6F73652033
:1049100070756C6C657900B100456E6473746F706E
:10492000206E6F742068697400B200456E64737401
:104930006F7000B3004D6F746F7200B400456E6409
:1049400073746F707300B500576972696E67206584
:1049500072726F7200B6004265642F4865617465BB
:104960007200B7004E6F7420636F6E6E656374657E
:104970006400B8004865617465722F546865726D93
:104980006973746F7200B900506C65617365206360
:104990006865636B3A00BA0053656C66746573743E
:1049A000206572726F722100BB0046696C616D6593
:1049B0006E742073656E736F7200BC005072696E06
:1049C000742066616E3A00BD00486F74656E6420A5
:1049D00066616E3A00BE0043616C6962726174691F
:1049E0006E6720686F6D6500BF0053656C66746507
:1049F0007374206661696C656400C000416C6C2052
:104A0000636F727265637400C100436865636B69AC
:104A10006E672073656E736F727300C200436865C2
:104A2000636B696E6720686F74656E6400C30043D2
:104A30006865636B696E672062656400C4004368E3
:104A400065636B696E67205A206178697300C500E1
:104A5000436865636B696E672059206178697300EC
:104A6000C600436865636B696E672058206178698A
:104A70007300C700436865636B696E6720656E6489
:104A800073746F707300C800436172642072656D47
:104A90006F76656400C9004261636B00CA004175AE
:104AA000746F20706F77657200CB0053696C656E10
:104AB0007400CC004D6F646500CD004869676820C4
:104AC000706F77657200CE0053747269637400CFA3
:104AD000005761726E00D0004E6F6E6500D10048C5
:104AE0006F74656E64206174203238304321204E2B
:104AF0006F7A7A6C65206368616E67656420616EA9
:104B000064207469676874656E656420746F2073CF
:104B1000706563733F00D200466F722061204E6F54
:104B20007A7A6C65206368616E676520706C656178
:104B3000736520726561640A70727573612E696FA6
:104B40002F6E6F7A7A6C652D6D6B337300D30050C6
:104B500049442063616C2E2066696E6973686564E0
:104B600000D4005049442063616C2E00D50050727F
:104B7000696E742070617573656400D60050726947
:104B80006E742061626F7274656400D700436F7049
:104B9000792073656C6563746564206C616E6775FC
:104BA0006167653F00D8004E6F7A7A6C6520646952
:104BB000616D6574657220646966666572732066EE
:104BC000726F6D2074686520472D636F64652E00D9
:104BD000D9004E6F7A7A6C65206469616D65746581
:104BE0007220646966666572732066726F6D2074E8
:104BF000686520472D636F64652E20506C65617376
:104C00006520636865636B207468652076616C75E8
:104C10006520696E2073657474696E67732E00DA9F
:104C2000005468657265206973206E6F2066696C38
:104C3000616D656E74206C6F616465642E00DB00CD
:104C40005468657265206973207374696C6C2061A7
:104C5000206E65656420746F206D616B65205A203D
:104C600063616C6962726174696F6E2E20506C654D
:104C700061736520666F6C6C6F7720746865206D5A
:104C8000616E75616C2C206368617074657220467A
:104C9000697273742073746570732C207365637408
:104CA000696F6E2043616C6962726174696F6E2016
:104CB000666C6F772E00DC005072696E746572202E
:104CC000686173206E6F74206265656E2063616C2D
:104CD00069627261746564207965742E20506C6518
:104CE00061736520666F6C6C6F7720746865206DEA
:104CF000616E75616C2C206368617074657220460A
:104D0000697273742073746570732C207365637497
:104D1000696F6E2043616C6962726174696F6E20A5
:104D2000666C6F772E00DD0053656C667465737476
:104D30002077696C6C2062652072756E20746F201C
:104D400063616C696272617465206163637572612D
:104D500074652073656E736F726C65737320726512
:104D6000686F6D696E672E00DE004F6C642073659E
:104D70007474696E677320666F756E642E20446567
:104D80006661756C74205049442C204573746570BD
:104D900073206574632E2077696C6C2062652073C4
:104DA00065742E00DF005761726E696E673A20628B
:104DB0006F7468207072696E7465722074797065A2
:104DC00020616E64206D6F74686572626F617264D9
:104DD0002074797065206368616E6765642E00E0F9
:104DE000005761726E696E673A207072696E746501
:104DF000722074797065206368616E6765642E0047
:104E0000E1005761726E696E673A206D6F74686574
:104E100072626F6172642074797065206368616E7C
:104E20006765642E00E200536865657400E3005511
:104E30006E6578706563746564206572726F722048
:104E40006F636375727265642E00E4004D36303016
:104E50002046696C616D656E74204368616E67659C
:104E60002E204C6F61642061206E65772066696C2E
:104E7000616D656E74206F7220656A65637420745D
:104E80006865206F6C64206F6E652E00E5005265CA
:104E90006D6F76652074686520656A656374656406
:104EA0002066696C616D656E742066726F6D20742A
:104EB00068652066726F6E74206F66207468652066
:104EC0004D4D552E00E60046696C616D656E74208F
:104ED000646574656374656420756E657870656378
:104EE0007465646C792E20456E73757265206E6FE3
:104EF0002066696C616D656E74206973206C6F61EA
:104F00006465642E20436865636B20746865207354
:104F1000656E736F727320616E6420776972696E5B
:104F2000672E00E700496E7465726E616C207275C1
:104F30006E74696D65206572726F722E205472797D
:104F400020726573657474696E6720746865204D9E
:104F50004D55206F72207570646174696E6720749E
:104F60006865206669726D776172652E00E8004D94
:104F70004D552046572076657273696F6E206973B0
:104F800020696E636F6D70617469626C652077690A
:104F90007468207072696E7465722046572E557061
:104FA0006461746520746F2076657273696F6E201A
:104FB000332E302E332E00E9004D4D5520466972B8
:104FC0006D7761726520696E7465726E616C2065C3
:104FD00072726F722C20706C6561736520726573DC
:104FE000657420746865204D4D552E00EA005265A9
:104FF000717565737465642066696C616D656E7446
:1050000020746F6F6C206973206E6F7420617661FD
:10501000696C61626C65206F6E20746869732068CA
:10502000617264776172652E20436865636B2074DA
:10503000686520472D636F646520666F7220746F0A
:105040006F6C20696E646578206F7574206F6620C0
:1050500072616E6765202854302D5434292E00EB80
:105060000043616E6E6F7420706572666F726D20A2
:1050700074686520616374696F6E2C2066696C6169
:105080006D656E7420697320616C7265616479204E
:105090006C6F616465642E20556E6C6F616420696D
:1050A000742066697273742E00EC004D4D55206EAD
:1050B0006F7420726573706F6E64696E6720636FC2
:1050C00072726563746C792E20436865636B20741B
:1050D000686520776972696E6720616E6420636F0E
:1050E0006E6E6563746F72732E00ED004D4D55202A
:1050F0006E6F7420726573706F6E64696E672E20B8
:10510000436865636B2074686520776972696E67B0
:1051100020616E6420636F6E6E6563746F72732EB0
:1051200000EE004D6F72652064657461696C7320D8
:105130006F6E6C696E652E00EF00546865204964DF
:105140006C65722063616E6E6F7420686F6D652090
:1051500070726F7065726C792E20436865636B2086
:10516000666F7220616E797468696E6720626C6F19
:10517000636B696E6720697473206D6F76656D650A
:105180006E742E00F00043616E2774206D6F76659B
:105190002053656C6563746F72206F722049646C74
:1051A00065722E00F1005468652053656C65637468
:1051B0006F722063616E6E6F7420686F6D65207012
:1051C000726F7065726C792E20436865636B206620
:1051D0006F7220616E797468696E6720626C6F63AC
:1051E0006B696E6720697473206D6F76656D656E8F
:1051F000742E00F2004C6F6164696E6720746F203A
:105200006578747275646572206661696C65642E78
:1052100020496E7370656374207468652066696CDC
:10522000616D656E74207469702073686170652E9D
:1052300020526566696E65207468652073656E73BB
:105240006F722063616C6962726174696F6E2C2089
:105250006966206E65656465642E00F30053656CB5
:105260006563746F722063616E2774206D6F76655D
:105270002064756520746F2046494E444120646562
:1052800074656374696E6720612066696C616D6521
:105290006E742E204D616B652073757265206E6F84
:1052A0002066696C616D656E7420697320696E207B
:1052B00053656C6563746F7220616E642046494E5D
:1052C000444120776F726B732070726F7065726CDF
:1052D000792E00F40046696C616D656E742073650B
:1052E0006E736F722074726967676572656420748B
:1052F0006F6F206561726C79207768696C65206CCE
:105300006F6164696E6720746F206578747275646C
:1053100065722E20436865636B2074686572652032
:1053200069736E277420616E797468696E67207383
:105330007475636B20696E20505446452074756205
:10534000652E20436865636B207468617420736503
:105350006E736F722072656164732070726F706516
:10536000726C792E00F50050756C6C6579206D6F4C
:10537000746F72207374616C6C65642E20456E735B
:10538000757265207468652070756C6C6579206332
:10539000616E206D6F766520616E64206368656361
:1053A0006B2074686520776972696E672E00F6005D
:1053B00046696C616D656E742073656E736F7220E3
:1053C0006469646E277420737769746368206F66FC
:1053D00066207768696C6520756E6C6F6164696EB4
:1053E000672066696C616D656E742E20456E7375FD
:1053F00072652066696C616D656E742063616E20F4
:105400006D6F766520616E64207468652073656ECB
:10541000736F7220776F726B732E00F70046696CA2
:10542000616D656E742073656E736F72206469645C
:105430006E27742074726967676572207768696C7B
:1054400065206C6F6164696E6720746865206669A9
:105450006C616D656E742E20456E73757265207477
:1054600068652073656E736F722069732063616C69
:105470006962726174656420616E6420746865207D
:1054800066696C616D656E742072656163686564E0
:105490002069742E00F80046494E44412064696436
:1054A0006E277420737769746368206F666620774F
:1054B00068696C6520756E6C6F6164696E672066E3
:1054C000696C616D656E742E2054727920756E6CF6
:1054D0006F6164696E67206D616E75616C6C792EA9
:1054E00020456E737572652066696C616D656E74BA
:1054F0002063616E206D6F766520616E6420464981
:105500004E444120776F726B732E00F90046494E6E
:105510004441206469646E2774207472696767650A
:1055200072207768696C65206C6F6164696E6720B2
:105530007468652066696C616D656E742E20456EB9
:1055400073757265207468652066696C616D656E3F
:10555000742063616E206D6F766520616E642046F5
:10556000494E444120776F726B732E00FA004469F4
:105570007361626C6500FB0053746F7000FC004C3B
:105580006F616400FD00556E6C6F616400FE005237
:10559000657365744D4D5500FF0052657472790056
:1055A0000001426564206C6576656C696E672066F3
:1055B00061696C65642E2053656E736F7220646937
:1055C000646E277420747269676765722E20446563
:1055D00062726973206F6E206E6F7A7A6C653F20FD
:1055E00057616974696E6720666F722072657365B2
:1055F000742E00010153656E73697469766974795C
:10560000000201446F6E65000301526573756D6998
:105610006E67207072696E7400040150494E4441F7
:105620002048656174696E6700050143616C6962B9
:10563000726174696F6E20646F6E6500060143616C
:105640006C6962726174696E67205A000701426575
:105650006420646F6E6500080142656420486561DE
:1056600074696E6700090148656174696E6720643A
:105670006F6E652E000A0148656174696E67000BE4
:1056800001546F74616C000C014C61737420707272
:10569000696E74000D014D4D55206661696C730093
:1056A0000E014D4D55206C6F6164206661696C730D
:1056B000000F014D4D5520706F776572206661694E
:1056C0006C730010014D6174657269616C206368D0
:1056D000616E6765730011014C61737420707269AB
:1056E0006E74206661696C75726573001201546F87
:1056F00074616C206661696C757265730013014694
:10570000696C2E2072756E6F757473001401546588
:105710006D70657261747572657300150153656E05
:10572000736F7220696E666F00160145787472752A
:1057300064657220696E666F00170158595A2063BC
:10574000616C2E2064657461696C7300180150727D
:10575000696E74657220495020416464723A001980
:1057600001756E6B6E6F776E001A014D4D5520639B
:105770006F6E6E6563746564001B01446174653A05
:10578000001C01746F20756E6C6F61642066696C1B
:10579000616D656E74001D01746F206C6F61642013
:1057A00066696C616D656E74001E0150726573737D
:1057B00020746865206B6E6F62001F01507265680F
:1057C000656174696E6720746F20637574002001D1
:1057D00050726568656174696E6720746F20656AD0
:1057E00065637400210150726568656174696E6754
:1057F00020746F20756E6C6F6164002201507265B9
:1058000068656174696E6720746F206C6F616400F5
:105810002301436F6F6C646F776E00240146696CDF
:10582000616D656E7420657874727564696E672049
:1058300026207769746820636F72726563742063D1
:105840006F6C6F723F002501456A65637400260125
:105850004175746F6C6F6164696E672066696C6115
:105860006D656E74206973206163746976652C20A0
:105870006A75737420707265737320746865206B29
:105880006E6F6220616E6420696E7365727420664B
:10589000696C616D656E742E2E2E002701546F7435
:1058A000616C2066696C616D656E74002801546FCF
:1058B00074616C207072696E742074696D65002962
:1058C0000146696C616D656E742075736564002AAC
:1058D000015072696E742074696D65002B01466514
:1058E0006564696E6720746F204653656E736F72CE
:1058F000002C014D6F76696E672073656C6563746B
:105900006F72002D01486F6D696E67002E01526540
:1059100074726163742066726F6D2046494E444113
:10592000002F01456A656374696E672066696C6162
:105930006D656E740030015061726B696E67207323
:10594000656C6563746F7200310152657475726EB7
:10595000696E672073656C6563746F720032015005
:105960006572666F726D696E6720637574003301CE
:1059700050757368696E672066696C616D656E74D9
:10598000003401507265706172696E6720626C61EB
:10599000646500350153656C656374696E672066E4
:1059A000696C2E20736C6F74003601556E6C6F61DC
:1059B00064696E672066696C616D656E740037019D
:1059C00045525220544D43206661696C656400382D
:1059D000014552522048656C702066696C616D65A6
:1059E0006E7400390145525220496E7465726E61C1
:1059F0006C003A01455252205761697420666F72FB
:105A00002055736572003B0146696E697368696E63
:105A100067206D6F76656D656E7473003C0141762D
:105A20006F6964696E67206772696E64003D014644
:105A3000656564696E6720746F206E6F7A7A6C6535
:105A4000003E0146656564696E6720746F20657865
:105A5000747275646572003F0146656564696E67BE
:105A600020746F2046494E4441004001556E6C6FD2
:105A70006164696E6720746F2070756C6C65790065
:105A80004101556E6C6F6164696E6720746F2046CA
:105A9000494E4441004201446973656E676167691C
:105AA0006E672069646C6572004301456E676167CB
:105AB000696E672069646C65720044014F4B004554
:105AC00001554E4B4E4F574E204552524F520046B5
:105AD0000146494C414D454E54204348414E4745AF
:105AE00000470146494C414D454E5420454A4543E7
:105AF000544544004801554E4C4F4144204D414EC1
:105B000055414C4C5900490146572052554E544975
:105B10004D45204552524F52004A014D4D552046A9
:105B20005720555044415445204E45454445440076
:105B30004B0151554555452046554C4C004C0149AB
:105B40004E56414C494420544F4F4C004D0146495C
:105B50004C2E20414C5245414459204C4F41444524
:105B600044004E01434F4D4D554E49434154494F1A
:105B70004E204552524F52004F014D4D55204E4F31
:105B80005420524553504F4E44494E470050014D0A
:105B90004D55204D4355204552524F520051014D15
:105BA0004D552053454C4654455354204641494C8D
:105BB0004544005201544D43204452495645522019
:105BC00053484F52544544005301544D4320554EC1
:105BD000444552564F4C544147452045525200547B
:105BE00001544D4320445249564552205245534595
:105BF00054005501544D43204452495645522045C6
:105C000052524F52005601544D43204F5645524870
:105C1000454154204552524F520057015741524E70
:105C2000494E4720544D4320544F4F20484F540075
:105C3000580149444C45522043414E4E4F54204D4B
:105C40004F564500590149444C45522043414E4E60
:105C50004F5420484F4D45005A0153454C4543543D
:105C60004F522043414E4E4F54204D4F5645005BFE
:105C70000153454C4543544F522043414E4E4F54DF
:105C800020484F4D45005C014C4F414420544F206B
:105C9000455854522E204641494C4544005D014927
:105CA0004E53504543542046494E4441005E014600
:105CB00053454E534F5220544F4F204541524C595B
:105CC000005F0150554C4C45592043414E4E4F54B6
:105CD000204D4F56450060014653454E534F5220CC
:105CE00046494C2E20535455434B006101465345C1
:105CF0004E534F52204449444E5420545249474732
:105D00002E00620146494E44412046494C414D2EE9
:105D100020535455434B00630146494E44412044AF
:105D200049444E5420545249474745520064014E5D
:105D30006F74207370696E6E696E670065015370D1
:105D4000696E6E696E670066014C65667420686FE7
:105D500074656E642066616E3F00670146726F6E07
:105D600074207072696E742066616E3F006801462F
:105D7000616E207465737400690158595A2063611B
:105D80006C6962726174696F6E20616C6C207269FB
:105D90006768742E20536B65772077696C6C20627E
:105DA0006520636F72726563746564206175746FDA
:105DB0006D61746963616C6C792E006A0158595A7F
:105DC0002063616C6962726174696F6E20616C6CD2
:105DD0002072696768742E20582F59206178657386
:105DE0002061726520736C696768746C7920736BCD
:105DF000657765642E20476F6F64206A6F622100AB
:105E00006B0158595A2063616C6962726174696FE1
:105E10006E206F6B2E20582F59206178657320619A
:105E200072652070657270656E646963756C61720D
:105E30002E20436F6E67726174756C6174696F6E4A
:105E40007321006C0158595A2063616C6962726158
:105E500074696F6E20636F6D70726F6D69736564C6
:105E60002E2052696768742066726F6E74206361B9
:105E70006C6962726174696F6E20706F696E7420F4
:105E80006E6F7420726561636861626C652E006D6F
:105E90000158595A2063616C6962726174696F6E4E
:105EA00020636F6D70726F6D697365642E2046722A
:105EB0006F6E742063616C6962726174696F6E20C9
:105EC000706F696E7473206E6F74207265616368A1
:105ED00061626C652E006E0158595A2063616C69CD
:105EE00062726174696F6E206661696C65642E20F0
:105EF00052696768742066726F6E742063616C69A2
:105F000062726174696F6E20706F696E74206E6F5B
:105F10007420726561636861626C652E006F015860
:105F2000595A2063616C6962726174696F6E206690
:105F300061696C65642E2046726F6E742063616CBB
:105F40006962726174696F6E20706F696E7473201C
:105F50006E6F7420726561636861626C652E00709B
:105F60000158595A2063616C6962726174696F6E7D
:105F7000206661696C65642E20506C6561736520D4
:105F8000636F6E73756C7420746865206D616E75D7
:105F9000616C2E00710158595A2063616C696272FC
:105FA0006174696F6E206661696C65642E2042655C
:105FB000642063616C6962726174696F6E20706FD6
:105FC000696E7420776173206E6F7420666F756ED2
:105FD000642E007201506C6561736520706C6163A2
:105FE0006520737465656C207368656574206F6ED9
:105FF00020686561746265642E007301446973747E
:10600000616E6365206265747765656E2074697082
:10601000206F6620746865206E6F7A7A6C652061E7
:106020006E642074686520626564207375726661B1
:10603000636520686173206E6F74206265656E20F1
:10604000736574207965742E20506C6561736520CA
:10605000666F6C6C6F7720746865206D616E75611A
:106060006C2C206368617074657220466972737469
:106070002073746570732C2073656374696F6E2070
:106080004669727374206C617965722063616C6912
:1060900062726174696F6E2E007401506C61636589
:1060A0002061207368656574206F6620706170657B
:1060B0007220756E64657220746865206E6F7A7ADE
:1060C0006C6520647572696E672074686520636111
:1060D0006C6962726174696F6E206F6620666972A6
:1060E0007374203420706F696E74732E204966209B
:1060F000746865206E6F7A7A6C652063617463687A
:106100006573207468652070617065722C20706FF3
:10611000776572206F666620746865207072696E9C
:1061200074657220696D6D6564696174656C792E42
:10613000007501536561726368696E67206265640A
:106140002063616C6962726174696F6E20706F693F
:106150006E740076014D6561737572696E672072A9
:1061600065666572656E6365206865696768742039
:106170006F662063616C6962726174696F6E207012
:106180006F696E74007701506C6561736520636C94
:1061900065616E20746865206E6F7A7A6C65206622
:1061A0006F722063616C6962726174696F6E2E2018
:1061B000436C69636B207768656E20646F6E652E33
:1061C0000078014175746F20686F6D650079014337
:1061D00075742066696C616D656E74007A01456A3C
:1061E0006563742066726F6D204D4D55007B014CC8
:1061F0006F6164696E672066696C616D656E7400BD
:106200007C014D4D552052657472793A2052657368
:10621000746F72696E672074656D706572617475F4
:1062200072652E2E2E007D01536F7274696E672089
:1062300066696C6573007E01536F6D652066696CDD
:1062400065732077696C6C206E6F742062652073B3
:106250006F727465642E204D61782E204E6F2E2053
:106260006F662066696C657320696E203120666FE9
:106270006C64657220666F7220736F7274696E67EA
:10628000206973203130302E007F0153544F50501D
:1062900045442E0080014F66660081014F6E006507
:1062A0006E717565696E67202200446F6E6520709F
:1062B00072696E74696E672066696C65004E6F2046
:1062C0004C696E65204E756D6265722077697468E1
:1062D00020636865636B73756D2C204C617374204B
:1062E0004C696E653A20004E6F20436865636B739E
:1062F000756D2077697468206C696E65206E756DA8
:106300006265722C204C617374204C696E653A2072
:1063100000636865636B73756D206D69736D61747F
:1063200063682C204C617374204C696E653A2000C0
:106330004C696E65204E756D626572206973206EC2
:106340006F74204C617374204C696E65204E756DBE
:106350006265722B312C204C617374204C696E6520
:106360003A2000257520627974657320777269740C
:1063700074656E20746F20255320617420616464FD
:1063800072657373203078253038780A00442564AC
:10639000202D20526561642F577269746520255342
:1063A0000A003F3F00526F6D616E61004872766176
:1063B00074736B69004D616779617200536C6F761D
:1063C000656E63696E61004E6F72736B0053766524
:1063D0006E736B61004E656465726C616E64730010
:1063E000506F6C736B69004974616C69616E6F000A
:1063F0004672616E6361697300457370616E6F6CA4
:1064000000446575747363680043657374696E61F5
:1064100000456E676C6973680020436F756E742069
:10642000583A200045303A25642052504D205052B1
:106430004E313A25642052504D204530403A257562
:106440002050524E31403A25750A00526573656EF0
:10645000640025533A20256C640A25530A002F2F27
:10646000616374696F6E3A6E6F74696669636174B3
:10647000696F6E2025530A0046696C616D656E7404
:106480002072756E6F7574206465746563746564DD
:10649000210064697361626C656400656E61626CA1
:1064A000656400454550524F4D005352414D0044E4
:1064B0002D31202D20456E646C657373206C6F6FD9
:1064C000700A00416374697665204578747275645A
:1064D00065723A203000496E76616C696420657897
:1064E000747275646572004D323230205325640039
:1064F0005344207072696E74696E672062797465A6
:106500002000257500556E6B6E6F776E20636F6D82
:106510006D616E643A2022004D32303020496E7633
:10652000616C696420657874727564657220007AA4
:106530005F6D61783A20007A5F6D696E3A2000796C
:106540005F6D696E3A2000545249474745524544B1
:10655000006F70656E00785F6D696E3A200052655D
:10656000706F7274696E6720656E6473746F7020EB
:10657000737461747573004D3131322063616C6CDA
:1065800065642E20456D657267656E63792053746E
:106590006F702E002F2F616374696F6E3A75766C81
:1065A0006F5F7265636F766572795F72656164793A
:1065B0000025533A256C7520636D0A25533A256CE6
:1065C00075206D696E0A0053494C454E54004E4F7C
:1065D000524D414C002553204D4F44453A205065C3
:1065E0007263656E7420646F6E653A202568686416
:1065F0003B207072696E742074696D652072656DE0
:1066000061696E696E6720696E206D696E733A20EC
:1066100025643B204368616E676520696E206D6963
:106620006E733A2025640A005072696E7465725365
:10663000746174653A2025640A00456E64206669B9
:106640006C65206C69737400426567696E206669C9
:106650006C65206C69737400556E6B6E6F776E207D
:10666000256320636F64653A2025730A000A504948
:106670004E44412074656D70657261747572653A3F
:1066800020252E3166205A20736869667420286D93
:106690006D293A20252E3366000A537465703A201E
:1066A00025642F360A000A537465703A2025642F3A
:1066B000362028736B6970706564290A50494E440E
:1066C000412074656D70657261747572653A20253C
:1066D00064205A20736869667420286D6D293A30E9
:1066E0000A000A5A45524F3A20252E33660A007393
:1066F000746172742074656D706572617475726511
:106700003A20252E31660A0025642020252E326687
:1067100000255320583A20252E356620593A202549
:106720002E3566205A3A20252E35660A00536C65B0
:1067300065702E2E2E0045303A25642052504D0AA9
:1067400050524E303A25642052504D0A004739309D
:10675000004D3130370025362E32666D6D002553E1
:106760000A25530A25533A0A25533A0025332E3277
:10677000668100252D31342E3134533A0A25530ACF
:10678000252D31342E3134533A25332E3266810A89
:10679000252D31342E3134533A25332E3266810083
:1067A0002020300020203100423A20253364202070
:1067B00020202058643A2536640A533A2025336451
:1067C000202020202059643A2536640046494E4452
:1067D000410050494E44410057697A617264206516
:1067E0006E642073746174653A2025640A005370E6
:1067F0006F6F6C4A6F696E004669726D7761726582
:1068000000537570657250494E44410048426564BA
:10681000206F6E206C6F616400466C617368416923
:1068200072004572723A484F54454E442046414EDC
:10683000204552524F52002F2F616374696F6E3A98
:10684000726573756D6564002F2F616374696F6E77
:106850003A726573756D65002F2F616374696F6E91
:106860003A7265616479002F2F616374696F6E3AC3
:106870006E6F745F7265616479002F2F6163746954
:106880006F6E3A63616E63656C004D3834004F4B38
:10689000004C434420737461747573206368616EA7
:1068A00067656400534420636172642072656C659F
:1068B00061736564002F2F616374696F6E3A73743E
:1068C00061727400473931004D3730320047323839
:1068D0002057004D3530300042616420696E746588
:1068E0007272757074005761746368646F672074A6
:1068F000696D656F757400537461746963206D65AB
:106900006D6F7279206861730A6265656E206F76BB
:1069100065727772697474656E004649524D5741CD
:106920005245204352415348210A43726173682003
:10693000726561736F6E3A0A002020506C616E6E52
:10694000657242756666657242797465733A2000B5
:106950002046726565204D656D6F72793A20002082
:106960007C20417574686F723A2000204C6173740A
:1069700020557064617465643A200020536F66741A
:106980007761726520526573657400205761746386
:1069900068646F67205265736574002042726F7778
:1069A0006E206F757420526573657400204578748D
:1069B00065726E616C20526573657400506F776507
:1069C000725570006572726F722077726974696EA9
:1069D0006720746F2066696C6500446F6E65207374
:1069E0006176696E672066696C652E006F6B004684
:1069F000696C616D656E7400312F390088002074F8
:106A00006F6F206C6F6E6720657874727573696F35
:106A10006E2070726576656E7465640020636F6CBD
:106A20006420657874727573696F6E207072657614
:106A3000656E746564004D6F76652061626F727477
:106A40006564004572723A5052494E542046414E98
:106A5000204552524F520025632533642F2564810F
:106A6000005A25362E32662563005A2020202D2D0F
:106A70002D2000862533642525002D2D2D2525006C
:106A80002533642525002053440020202000204881
:106A90004F002046524D2000872D2D3A2D2D2020CD
:106AA00000872533756820256325630087253032EC
:106AB000753A2530327525632563002F2F61637485
:106AC000696F6E3A706175736564002F2F6163742E
:106AD000696F6E3A70617573650044756D702074EE
:106AE0006F2073657269616C0068656C702E7072DE
:106AF00075736133642E636F6D00666F72756D2EF2
:106B0000707275736133642E636F6D00707275738C
:106B10006133642E636F6D004D3730310025533A79
:106B20000A2531382E32666D200A25533A0A25315E
:106B3000306C646420253032646820253032646D06
:106B40000025533A0A2531382E32666D200A255326
:106B50003A0A2531306C646820253032646D202576
:106B600030326473004D6561737572656420736BB8
:106B70006577733A2025662025660A004669747495
:106B8000696E67206661696C6564203D3E206361C3
:106B90006C6962726174696F6E206661696C6564AC
:106BA0002E0A0043616C6962726174696F6E2073B2
:106BB0007563636573732E0A00416C6C2034206327
:106BC000616C6962726174696F6E20706F696E7456
:106BD0007320666F756E642E0A00312F3400312FDA
:106BE0003400312F39005072757361206933204DA4
:106BF0004B322E35204F4B2E00534420636172647C
:106C0000206F6B006F70656E526F6F7420666169E4
:106C10006C656400766F6C756D652E696E697420A5
:106C20006661696C656400534420696E697420660E
:106C300061696C006F70656E206661696C65642CBB
:106C40002046696C653A200043616E6E6F74206562
:106C50006E746572207375626469723A20004D36F5
:106C60003030004D3234004D3233202573005072E5
:106C7000696E7465722073746F70706564206475DA
:106C80006520746F206572726F72732E2053757059
:106C90006572766973696F6E207265717569726568
:106CA000642E0047312045252D2E3366204632378D
:106CB0003030004D383300084AD73B3BCE016E845C
:106CC000BCBFFDC12F3D6C74319ABD56833DDA3D8A
:106CD00000C77F11BED9E4BB4C3E916BAAAABE008F
:106CE0000000803F05A84CCDB2D44EB93836A90279
:106CF0000C50B9918688083CA6AAAA2ABE000000BA
:106D0000803F07634236B79BD8A71A39685618AE3A
:106D1000BAAB558C1D3CB7CC5763BD6DEDFD753ED0
:106D2000F6177231BF000000803F08000000BE92DD
:106D30002449123EABAAAA2ABECDCCCC4C3E0000C0
:106D40000080BEABAAAAAA3E00000000BF0000005F
:106D5000803F0000000000084178D3BB4387D11377
:106D60003D190E3CC3BD4282AD2B3E68EC8276BE1F
:106D7000D98FE1A93E4C80EFFFBE01C4FF7F3F00E9
:106D8000000000000C94CBEA0C945FC90C94C4D8AA
:106D90000C942BD90C9475F90D9453240C9453C076
:106DA0000C94B1EA0C9410BB0C943AC20C94AEBC97
:106DB0000C9474F80C9405BB0D9446240C9451F774
:106DC0000D941C0D0D94CD010D944F0D0C941DBD13
:106DD0000D94DE9C0C946CCE0C940FF50C9483CD2A
:106DE0000C9446BD0D94BB240C9431D20C94ACD8B9
:106DF0000C941CD90D943D250C94E6D10C9411BD36
:106E00000D94BE020D94D30C0C94B9CC0C94F7766F
:106E10000C943FBE0C9471E70C94BDCD0C948F7A0A
:106E20000C9412F80C9416C00C947A780C94AED191
:106E30000C9487E70C94C0CD0C9458CE0C946BC284
:106E40000D947A0A0C94F4E70C94C6CD0D940525A4
:106E50000C94D2D10D94520E0C9448CE0C9472C264
:106E60000C943CBD0C94DACE0C9450CE0C9444BBE4
:106E70000D94E3960C94EBC60C9432BB0D94E59CF8
:106E80000D9454150D947C0D0C949CBD0C949F6333
:106E90000C9423BE0C94AADC0D944A050C94C0F605
:106EA0000C94FDEA0C94CAD10C9471C10C9420BBD3
:106EB0000C94F8BF0D94DB020C94FBBA0C9476C1D1
:106EC0000C94F8D40C9488CE0D94EC240C944AC6FF
:106ED0000C9486CE0C9459D50C9460CE0C947ABD4B
:106EE0000C9464C20C94A4D10C94D6CA0C9415F5DD
:106EF0000C9436BB0D94B2020C943CBB0C9401BBB9
:106F00000C9432CC0C94BFBC0C946DEA0C9480C1F0
:106F10000C948AD60D94600D0C941FD90C9470BDFE
:106F20000D9409240C949FFC0D9468960C943DE9F3
:106F30000D94C29C0D940D250C94DCD10C9477CE4D
:106F40000C9485C10C9447D70C944FF60C949FD1A8
:106F50000C945CBE0C9405770D94F2240C9433DDF4
:106F60000C94C9CD0C94E6EA0C947BC10D94870176
:106F70000C9447770C945EDD0C9428C60D9425255F
:106F80000C9418CA0C9485BD0C94E2EA0C94D2CDF2
:106F90000C94C2D10C94BCF60C9467C10D943525A9
:106FA0000C94F6BC0D94E0960C94DFCE0D94003159
:106FB0000D9415250C94B8D10C9453C60D94492406
:106FC0000C9452730C9448BB0C943BBB0C94EFFC98
:106FD0000D94EE9C0D948F040D94E7960D94B824B7
:106FE0000D9424020D9401640C9477EA0D947C9C1A
:106FF0000C9461EA0C9480C20C9478BE0D942D25FB
:107000000C945CBD0C9416D90C941DD20C944DBB01
:107010000D94F5240C9428BB0C9413D20D94220AE1
:107020000C9497D10C9455BE0D948C240C9411EBB8
:107030000C9496DC0C94EC760C945CC60C943FC9D2
:107040000C948EC10D94C00C0D94CF020D946D055F
:107050000D9481960D9450240C940AD90C94DCEA7A
:107060000C9483C40C9420FC0C9424770C9402BDE3
:107070000C944CBF0C94A8F70C94C3CD0C9424CF63
:107080000C9441C60C948AFC0C94FDC30C9419D941
:107090000C9407FD0C942EBB0C947CDC0D94620BBD
:1070A0000C94F0D10C946CC10C9427D20C9491E305
:1070B0000C9458CD0D9469050D94DE020C94B4BC6B
:1070C0000C946DE10C943B730C94C5C50C9424BBDB
:1070D0000C9441EA0C94AFBD0D9421240C9409BB8F
:1070E0000C94FFD10C94CCC10D94E3040D94EF24C7
:1070F0000C9440BB0C9416BB0C948BCE0C9450BDDE
:107100000C9416F80D94BE240C948AC10D94C408F6
:107110000D94FD240D94F39C0D941D250C9432BD0B
:107120000C94D2760C9437D90C94BACD0C9407E712
:107130000C9479C20C941ABB0C941B770C9459775D
:107140000D9445250C944ECD0D9465090C940DBB02
:107150000C94A0D80D944D250D9473020D94E19CD0
:107160000D940D020C94F4EA0D94C3960C9409D27C
:107170000C9428BD0C9466BD6E616E00696E66004D
:1071800000407A10F35A00A0724E18090010A5D4DE
:10719000E80000E87648170000E40B54020000CA3B
:1071A0009A3B000000E1F505000080969800000081
:1071B00040420F000000A0860100000010270000E0
:1071C0000000E803000000006400000000000A0066
:1071D000000000000100000000002C76D888DC6769
:1071E0004F0823DFC1DFAE59E1B1B796E5E3E453C1
:1071F000C63AE651997696E8E6C28426EB898C9BDE
:1072000062ED407C6FFCEFBC9C9F40F2BAA56FA57D
:10721000F490055A2AF75C936B6CF9676DC11BFCFF
:10722000E0E40D47FEF520E6B500D0ED902E03001A
:10723000943577050080841E080000204E0A000067
:1072400000C80C333333330F986E12831141EF8D26
:107250002114893BE65516CFFEE6DB18D1844B3866
:107260001BF77C1D901DA4BBE424203284725E2297
:107270008100C9F124ECA1E53D27220000204553FF
:107280005000204E535000204F464600204F4E00E5
:107290005056303100205B4D505D2000256920683C
:1072A0006F757273202569206D696E757465730042
:1072B00052582074696D656F7574004D333130001C
:1072C0004D313132004D3131300046756C6C2052F9
:1072D00058204275666665720053657474696E67FE
:1072E000732053746F7265640053746F7265642009
:1072F00073657474696E67732072657472696576FC
:1073000065640048617264636F6465642044656607
:1073100061756C742053657474696E6773204C6F6B
:107320006164656400563200000000C8420000C875
:10733000420000C8430000054300004843000048E5
:1073400043000040410000F042E8030000E8030071
:1073500000C80000008813000000409C4400409CCE
:10736000440000000000000000204E00000000204B
:107370004100002041CDCCCC3E00009040000000F8
:10738000000000000000000000CDCCCC3E3D0A8192
:1073900041FF08433EB099AB438F42FC42E65A346A
:1073A0003F4C62B045000000000040400000344205
:1073B000000000000000000000000041000000E0AC
:1073C0003F00002C4300002C43000040410000F02F
:1073D00042C0030000C0030000C800000088130082
:1073E000001010101000409C440000803F0000007E
:1073F0003F191400000020307800203078006572BA
:10740000726F723A2000443233202D20656D657210
:1074100067656E63792073657269616C2064756D50
:107420007000437573746F6D004E796C6F6E5041D0
:1074300000536174696E2020005465787475720081
:10744000536D6F6F746800312E3000312E3500554A
:107450004E4B4E4F574E004C413130433A204C6911
:107460006E65617220416476616E6365206D6F6444
:10747000653A20004C413130433A2041646A7573CB
:1074800074656420452D4A65726B3A2000C35AE743
:10749000103E0FA8AF00480069960000DF60255538
:1074A0005887680427F2E0005E3403CC1960F33C8F
:1074B0000EF88F00DB08029492003E1C079A8700AA
:1074C000E524008528527E06001BE4007E781270B9
:1074D000787061F812788F8841784270787061789E
:1074E0002570787061F850788F88D1F0252707874C
:1074F00061F025278F88412C0D27AA50D1BC0707A2
:10750000871161BE788F881141785270787061F868
:1075100052788F8841201278887063205278887062
:10752000634852788887430311179970641812785A
:10753000F870654412F8F8F045184278F87065184C
:107540002578F87065185278F87065185078F870DA
:10755000650C078F872365A20F8F8F1145001206D8
:10756000227069001207222749002506227069004F
:10757000250722274900120622276C026236A270D4
:107580006C40456C44704C03622222706C438888C6
:1075900088F04C7812BC88806E7852BC88806E3837
:1075A000127888706F78127888874F3842788870A0
:1075B0006F38257888706F3A0079AC786F3D079AFC
:1075C000AC786F7850788887EF39497888706F0881
:1075D00052BC8880729852F88F985220127870F0BE
:1075E0007348127863875320527870F0734852784A
:1075F0006387531007870F247312786387245360BF
:10760000699A988BE22304E4443074104E44432476
:10761000747C12888960753C50888870557825285C
:107620008960757949088960753C12887070790C99
:1076300012885222594412F124F07A4452F124F073
:107640007A8C52F0368F5A4420F124F07A0040149C
:1076500054CDCCCC3D0AD7233C17B7D13877CC2BAF
:10766000329595E6241FB14F0A000020410000C862
:107670004200401C4620BCBE4CCA1B0E5AAEC59DE3
:10768000744E414E494E4600007A4300005243007A
:1076900000524300000000000080C09A99193E008B
:1076A000000000000080C09A99193E20503A002046
:1076B00042403A0020403A00202F002054303A0047
:1076C000202F0020423A00202F00543A0025534535
:1076D000786365737369766520626564206C65768E
:1076E000656C696E6720636F7272656374696F6E33
:1076F0003A202569206D6963726F6E730A004265D6
:1077000064206C6576656C696E67206661696C657E
:10771000642E20546F6F206D7563682076617269E6
:107720006174696F6E2066726F6D20656570726F2F
:107730006D206D65736800426564206C6576656CCC
:10774000696E67206661696C65642E2053656E738F
:107750006F722074726967676572656420746F6FF9
:1077600020736F6F6E002020004D65617375726528
:107770006420706F696E74733A005A207365617289
:107780006368206865696768743A20352E30660042
:107790004E756D20582C593A20372C37004D6573A3
:1077A0006820626564206C6576656C696E67206E22
:1077B0006F74206163746976652E0020453A00205D
:1077C0005A3A0020593A0020453A00205A3A0020FF
:1077D000593A00583A00202D3E200053706F6F6CCC
:1077E0004A6F696E3A20002C2000496E616374690B
:1077F000766974792053687574646F776E004B49AD
:107800004C4C45442E005072696E7465722068615C
:107810006C7465642E206B696C6C28292063616C24
:107820006C656421005A206C6976652061646A7514
:107830007374206F7574206F662072616E67652E99
:107840002053657474696E6720746F20302E204356
:107850006C69636B20746F20636F6E74696E7565FD
:107860002E005A206C6976652061646A75737420F5
:107870006F7574206F662072616E67652E20536588
:107880007474696E6720746F20300020453A302090
:10789000423A00543A00627573793A207061757308
:1078A000656420666F7220696E707574006275730E
:1078B000793A2070617573656420666F7220757304
:1078C000657200627573793A2070726F63657373C5
:1078D000696E670073657269616C2064756D7020F4
:1078E00000496E76616C6964205420636F64652E74
:1078F000004475706C696361746520542D636F6416
:10790000652069676E6F7265642E00416476616EF2
:107910006365204B3D004B206F7574206F662061BE
:107920006C6C6F7765642072616E676521004D4BEA
:10793000322E35004D4B322E354D4D5532001A4FFB
:10794000FA002533642F2533640025336400200AB0
:10795000200A200A200025535374617469737469E6
:1079600063733A0A255320204D37382053256C7510
:107970002054256C750A00255341726320536574A9
:1079800074696E67733A20503A4D6178206C656E69
:10799000677468286D6D2920533A4D696E206C65B7
:1079A0006E67746820286D6D29204E3A436F72729D
:1079B000656374696F6E7320523A4D696E2073650A
:1079C000676D656E747320463A5365676D656E74B6
:1079D000732F7365632E0A255320204D32313420D6
:1079E00050252E32662053252E3266204E256420E7
:1079F000522564204625640A00255346696C616D52
:107A0000656E742073657474696E67733A20446997
:107A10007361626C65640A00255346696C616D652B
:107A20006E742073657474696E67733A0A25532007
:107A300020204D3230302044252E32660A00255356
:107A4000526574726163743A20533D4C656E67747D
:107A50006820286D6D2920463A537065656420289A
:107A60006D6D2F6D29205A3A205A4C696674202872
:107A70006D6D290A25532020204D323037205325A3
:107A80002E32662046252E3266205A252E32660A70
:107A900025535265636F7665723A20533D4578747D
:107AA0007261206C656E67746820286D6D292046B0
:107AB0003A537065656420286D6D2F6D290A255332
:107AC0002020204D3230382053252E326620462586
:107AD0002E32660A25534175746F2D52657472619A
:107AE00063743A20533D3020746F2064697361627F
:107AF0006C652C203120746F20696E746572707211
:107B0000657420657874727564652D6F6E6C79206C
:107B10006D6F766573206173207265747261637432
:107B200073206F72207265636F7665726965730A80
:107B300025532020204D323039205325640A00255A
:107B400053504944206865617462656420736574AC
:107B500074696E67733A0A25532020204D33303400
:107B60002050252E32662049252E32662044252EAF
:107B700032660A0025535049442073657474696E57
:107B800067733A0A25532020204D33303120502589
:107B90002E32662049252E32662044252E32660A72
:107BA00000255353746570732070657220756E697B
:107BB000743A0A255320204D39322058252E32663A
:107BC0002059252E3266205A252E32662045252E34
:107BD00032660A25534D6178696D756D206665655D
:107BE00064726174657320286D6D2F73293A0A25BC
:107BF0005320204D3230332058252E32662059250F
:107C00002E3266205A252E32662045252E32660AEF
:107C100025534D6178696D756D20616363656C6591
:107C2000726174696F6E20286D6D2F7332293A0A64
:107C3000255320204D3230312058256C7520592590
:107C40006C75205A256C752045256C750A255341A5
:107C50006363656C65726174696F6E3A20503D7044
:107C600072696E742C20523D726574726163742C5B
:107C700020543D74726176656C0A255320204D3284
:107C800030342050252E32662052252E3266205464
:107C9000252E32660A2553416476616E6365642041
:107CA0007661726961626C65733A20533D4D696E0D
:107CB00020666565647261746520286D6D2F732977
:107CC0002C20543D4D696E2074726176656C20667F
:107CD0006565647261746520286D6D2F73292C2091
:107CE000423D6D696E696D756D207365676D656E7A
:107CF000742074696D6520287573292C20583D6D9A
:107D00006178696D756D205859206A65726B2028FD
:107D10006D6D2F73292C20205A3D6D6178696D752A
:107D20006D205A206A65726B20286D6D2F73292C87
:107D30002020453D6D6178696D756D2045206A652F
:107D4000726B20286D6D2F73290A255320204D3228
:107D500030352053252E32662054252E326620429F
:107D6000256C752058252E32662059252E32662026
:107D70005A252E32662045252E32660A2553486F35
:107D80006D65206F666673657420286D6D293A0AEB
:107D9000255320204D3230362058252E326620596A
:107DA000252E3266205A252E32660A004361703A2B
:107DB00025533A25630A0050525553415F4D4D55A6
:107DC0003200455854454E4445445F4D32300041E1
:107DD00055544F5245504F52545F504F5349544998
:107DE0004F4E004155544F5245504F52545F4641FB
:107DF0004E53004155544F5245504F52545F5445D5
:107E00004D50000044656C6574696F6E2066616951
:107E10006C65642C2046696C653A200046696C6587
:107E20002064656C657465643A004E6F7420534439
:107E3000207072696E74696E67005072696E74208A
:107E40007361766564005344207072696E742070AB
:107E50006175736564002533642F2533640066768D
:107E6000007468780050524E0022283229006E6F4C
:107E70002076616C696420636F6D6D616E64007A59
:107E800065726F72697A656400666163746F727996
:107E900020726573746F72656400696E6465782C16
:107EA0002074656D702C2075737465702C20756D51
:107EB0000050494E44412063616C207374617475B5
:107EC000733A2000503A005761697420666F72203F
:107ED00050494E4441207461726765742074656D29
:107EE00070657261747572653A002041002050001F
:107EF000204200204C00205200205A00204E4F54B7
:107F000020494E495449414C495A454400536865FB
:107F100065742000205A2056414C5545204F555439
:107F2000204F462052414E474500496E76616C69AC
:107F3000642073686565742049442E20416C6C6F21
:107F40007765643A20302E2E004155544F004C4145
:107F50004E472053454C20464F5243454400206431
:107F60003A0020693A0020703A0020643A00206903
:107F70003A0020703A00256925250A002569252543
:107F80000A0022283129002F2F0000204558545282
:107F9000554445525F434F554E543A3100204D41B0
:107FA0004348494E455F545950453A00312E300000
:107FB000206261736564206F6E204D61726C696E22
:107FC000204649524D574152455F55524C3A6874CC
:107FD0007470733A2F2F6769746875622E636F6DC2
:107FE0002F707275736133642F50727573612D46F3
:107FF00069726D776172652050524F544F434F4CF8
:108000005F56455253494F4E3A003737333130327D
:10801000346564005F0038323739002B004649521E
:108020004D574152455F4E414D453A50727573610F
:108030002D4669726D7761726520004D31313320B4
:1080400053006F6B20006E2F61003F546F7368699F
:10805000626120466C6173684169722047657449AA
:1080600050206661696C65640A00000125301D0CB2
:10807000FF24311C0BFF232F1B0A17FF0406222BA2
:108080001A03363535382569206D696E2C2025692F
:108090002073656300496E76616C6964204D2063CE
:1080A0006F64653A2025730A0050494E44412070A0
:1080B000726F62652063616C6962726174696F6E70
:1080C000207374617274004E6F2050494E444120F9
:1080D000746865726D6973746F7200736574006E95
:1080E0006F7A7A6C65004D424C004652004C7A0023
:1080F0004C616E6700315F37356D6D5F4D4B3235CA
:108100002D52414D426F3130612D453344763666F4
:10811000756C6C0052657600332E31342E312D385B
:108120003237390046697200534E20696E76616CB1
:10813000696400534E005245534554004D4D55520D
:1081400045530075766C6F0046414E0046414E50D7
:10815000494E54535400505255534100252E31304E
:10816000532000253464004D313034533000473102
:108170005831305931383046343030300047315A78
:1081800031304631333030004D31343053300047D8
:1081900031452D302E3037354632313030004D32BA
:1081A000303453313030300047315A354637323071
:1081B00030004731452D312E3546323130300047C1
:1081C000315A302E32004731583230322E35453850
:1081D0004631343030004731592D3246313030305D
:1081E0000047315832343045323546323230300073
:1081F00047315A302E334631303030004731583510
:1082000035453846323030300047315835453239FF
:1082100046313830300047315835354532394631EE
:1082200030373300473932453000473238004D315E
:108230003039004D31393000252D31322E31325355
:10824000252B382E31660045787472756465723A54
:108250000025632531372E32666D6D00583A00597E
:108260003A005A3A002563252D31332E31335325F8
:108270002B352E3366002533750050494E4441207E
:1082800063616C6962726174696F6E206661696CAA
:1082900065642E20436F6E74696E7565207769740E
:1082A00068207072657373696E6720746865206BEF
:1082B0006E6F622E0050494E44412063616C6962CA
:1082C000726174696F6E20646F6E652E20436F6EED
:1082D00074696E7565207769746820707265737350
:1082E000696E6720746865206B6E6F622E005A306D
:1082F000005A3100593000593100583000583100CF
:10830000456E642073746F70732064696167004701
:108310003830004D3435004D3435205A004737365B
:10832000004D3730312050300057697A6172642037
:1083300073746174653A2025640A0045787065722B
:10834000696D656E74616C00302E383000302E36E9
:108350003000302E343000302E32350044697361E5
:10836000626C65206661726D206D6F646500526598
:10837000736574204D4D55004D4D55004D343400FE
:108380004739390044697361626C65206661726DBA
:10839000206D6F64653F00473238205859004D20EA
:1083A000383400852E2E002533642F3000253364A9
:1083B0002F30006C63645F73656C66636865636B24
:1083C0005F617869732025642C2025640A00486F5A
:1083D00074656E6400426564005A00590058002DAF
:1083E0002D2D2D2D2D2D2D2D2D2D2D2D2D2D2D2DBD
:1083F0002D2D2D00537570657250494E44413A0041
:108400004D6751678F8188817D816E81C8686781E2
:108410008A68473159252E346645252E3466004733
:10842000315A252E326600473158353059313535AD
:108430000024824D67B36CB281A8819E8147315878
:10844000252E346645252E346600473146313038B6
:10845000300016820982FC81F0812482E181D6817C
:10846000C681BF815425640047315A302E340047FD
:1084700031592D33463130303000516733822E82EE
:108480002A8224824D3834205859004D3130392009
:10849000533238300047312058313235205A32308B
:1084A0003020463130303000496E76616C6964208E
:1084B0005049442063616C2E20726573756C74732F
:1084C0002E204E6F742073746F72656420746F2059
:1084D000454550524F4D2E004D3330312050252E02
:1084E00032662049252E32662044252E3266004D04
:1084F0003330332045302053253375005243004438
:108500004556004245544100414C5048410000004E
:108510002100240027002A002D0030003300010133
:108520000000040107010A010000220025002800C4
:108530002B002E003100340002010000050108016B
:108540000B01000020002300260029002C002F0032
:1085500032000001000003010601090105050505BF
:10856000070508080808020202020A0A08080404AB
:1085700004040101010101010101030303030303D9
:108580000303040707070C0C0C0C0C0C0C0C020268
:10859000020206060606060606060B0B0B0B0B0B65
:1085A0000B0B07070A0A0A0A0A0A05050504040450
:1085B00008080102102020080810204010204080E8
:1085C0000201020108040201010204081020408097
:1085D0008040201008040201800402018040201025
:1085E000080402010804020101020408102040806E
:1085F0000102040810204080100804088010204068
:10860000044080102040048000000A0B02090C0D79
:108610000E08070304010000000000000000000035
:10862000000000000000000000000000000000004A
:108630000000000012111000000000000000000007
:10864000000000000000000000000000000000002A
:108650000000000000000000000000000000332EB9
:1086600031342E31000A204F726967696E616C20C7
:1086700050727573612069330A202020507275731F
:10868000612052657365617263680A2532302E324B
:1086900030530053706F6F6C4A6F696E206973209E
:1086A000006164635F696E697400200A200A200A11
:1086B0002000416C6C2044617461005365727669DE
:1086C00063652070726570005368697070696E67C9
:1086D0002070726570005374617469737469637398
:1086E000004C616E67756167650045524153494EA4
:1086F0004720616C6C206461746100466163746F33
:1087000072792052455345540050525553413344D9
:1087100046570003000E0001004000030002000065
:108720000004007072757361336400323032352D8D
:1087300030342D32322032323A30333A3533002061
:10874000332E31342E312D383237395F37373331CC
:108750003032346564007374617274004D323900D4
:10876000252D392E39535B00200A200A20000000F5
:108770004842000058419A998D41333353404D4D42
:1087800055323A004D494E54454D50204245442003
:108790006669786564004D494E54454D5020484FF8
:1087A00054454E4420666978656400457872656D6D
:1087B00065207370616E206F6620746865205A2092
:1087C00076616C756573210025642F39004D4D5518
:1087D000323A002533640018010419020A0B55953A
:1087E000541B54AE536553D3525B52F351A451847E
:1087F000513851845121512151215121512151216F
:1088000051215121512151215121512151215121D8
:1088100051215121512151215121512151215121C8
:1088200051EA50A9505F50EC4FB74F6D4F234FC5E1
:108830004E8C4E4A4E2D4E01010101010101027183
:108840000171013232320303030303030303030301
:1088500003030303030303030393932438039303E2
:1088600001025603650066006700680069006A003F
:108870006B006C00730074007D007E00C900D300A3
:10888000DD00CA00D400DE002D01370141012E01B8
:10889000380142012F013901430130013A014401FD
:1088A00031013B014501320191019201F501F601CF
:1088B000F701F801F901FA01FB01FC018403985565
:1088C00001568D5584557D554658934776556C55C0
:1088D000252E3230530A70727573612E696F2F30F6
:1088E00034256875007B5B4552523A00332E313493
:1088F0002E31005D5B4657523A005D5B54494D3A5C
:10890000005D5B464E4D3A005D5B46454D3A005D6D
:108910005B5043443A005B5446553A005B50524E1C
:108920003A005B50464E3A305D005B4449413A00A4
:108930005D5B4154423A005D5B4154303A005D5BFF
:108940005354423A005B5354303A007B5B50524ED2
:108950003A355D007B5B50524E3A305D007B5B5098
:10896000524E3A395D007B5B50524E3A385D007B87
:108970005B5245533A305D5B46494C3A007B5B5253
:1089800045533A315D5B46494C3A000000211042A4
:108990002063308440A550C660E770088129914A61
:1089A000A16BB18CC1ADD1CEE1EFF13112100273E8
:1089B000325222B5529442F772D662399318837BB1
:1089C000B35AA3BDD39CC3FFF3DEE3622443342038
:1089D000040114E664C774A44485546AA54BB52801
:1089E000850995EEE5CFF5ACC58DD55336722611C8
:1089F000163006D776F6669556B4465BB77AA71951
:108A0000973887DFF7FEE79DD7BCC7C448E558868F
:108A100068A7784008611802282338CCC9EDD98EA0
:108A2000E9AFF9488969990AA92BB9F55AD44AB727
:108A30007A966A711A500A333A122AFDDBDCCBBFF0
:108A4000FB9EEB799B588B3BBB1AABA66C877CE4F7
:108A50004CC55C222C033C600C411CAEED8FFDEC40
:108A6000CDCDDD2AAD0BBD688D499D977EB66ED507
:108A70005EF44E133E322E511E700E9FFFBEEFDD90
:108A8000DFFCCF1BBF3AAF599F788F8891A981CA6D
:108A9000B1EBA10CD12DC14EF16FE18010A100C24C
:108AA00030E3200450254046706760B9839893FBFB
:108AB000A3DAB33DC31CD37FE35EF3B1029012F39C
:108AC00022D2323542145277625672EAB5CBA5A84B
:108AD0009589856EF54FE52CD50DC5E234C324A0EC
:108AE0001481046674476424540544DBA7FAB799DB
:108AF00087B8975FE77EF71DC73CD7D326F236913C
:108B000006B01657667676154634564CD96DC90EA2
:108B1000F92FE9C899E9898AB9ABA944586548068B
:108B2000782768C018E1088238A3287DCB5CDB3F3A
:108B3000EB1EFBF98BD89BBBAB9ABB754A545A37DB
:108B40006A167AF10AD01AB32A923A2EFD0FED6C0A
:108B5000DD4DCDAABD8BADE89DC98D267C076C642B
:108B60005C454CA23C832CE01CC10C1FEF3EFF5D1A
:108B7000CF7CDF9BAFBABFD98FF89F176E367E557B
:108B80004E745E932EB23ED10EF01E7C3C3E3F2FC3
:108B90002A225C0024F4D43050C38E20C2A2401795
:108BA000828B7011127A910D816CD90AA861E1084B
:108BB000C7586607615143061E4B5D05C145A704B2
:108BC0001A411104093D9803713931034036DB0223
:108BD00065339102D4305402802E1D02632CEE01C5
:108BE000752AC501B028A001102781018F256401D5
:108BF0002B244B01E0223401AC211F018D200D01FB
:108C0000801FFC00841EED00971DDF00B81CD20001
:108C1000E61BC600201BBC00641AB200B219A800F3
:108C20000A19A0006A189900D117910040178B000B
:108C3000B516840031167E00B31579003A1573001D
:108C4000C7146F0058146A00EE136600881363009F
:108C500025135E00C7125B006C12570015125400FA
:108C6000C111510070114F0021114B00D610490065
:108C70008D1047004610440002104200C00F400013
:108C8000800F3E00420F3C00060F3B00CB0E380029
:108C9000930E37005C0E3500270E3400F30D3200C2
:108CA000C10D3100900D3000600D2E00320D2D00F1
:108CB000050D2C00D90C2B00AE0C2900850C2900C9
:108CC0005C0C2700350C27000E0C2600E80B240056
:108CD000C40B2400A00B23007D0B23005A0B2100A2
:108CE000390B2100180B2000F80A1F00D90A1E00BA
:108CF000BB0A1E009D0A1D00800A1D00630A1C009D
:108D0000470A1B002C0A1B00110A1A00F7091A0057
:108D1000DD091900C4091900AB09190092091700EF
:108D20007B091800630917004C0916003609160064
:108D3000200916000A091500F5081500E0081400BE
:108D4000CC081400B8081400A408140090081300FC
:108D50007D0812006B081300580812004608120024
:108D60003408110023081100120811000108110035
:108D7000F0071000E0071000D0071000C007100037
:108D8000B0070F00A107100091070E0083070F0026
:108D900074070F0065070E0057070E0049070E0005
:108DA0003B070D002E070E0020070D0013070D00D6
:108DB00006070D00F9060C00ED060D00E0060C009C
:108DC000D4060C00C8060C00BC060C00B0060C0053
:108DD000A4060B0099060C008D060B0082060B0002
:108DE00077060B006C060B0061060A0057060B00A5
:108DF0004C060A0042060A0038060A002E060A003F
:108E000024060A001A060A001006090007060A00CE
:108E1000FD050900F4050900EB050900E20509005C
:108E2000D9050900D0050900C7050900BE050900DC
:108E3000B5050800AD050800A50509009C0508005A
:108E4000940508008C050800840508007C050800CE
:108E5000740508006C050700650508005D0507003E
:108E6000560508004E0507004705070040050800A5
:108E700038050700310507002A050700230507000C
:108E80001C050600160507000F050700080506006B
:108E900002050700FB040600F5040700EE040600C7
:108EA000E8040600E2040700DB040600D50406001F
:108EB000CF040600C9040600C3040600BD04060072
:108EC000B7040600B1040500AC040600A6040600C1
:108ED000A00405009B04060095040500900406000C
:108EE0008A04050085040500800406007A04050054
:108EF00075040500700405006B0405006604050098
:108F0000610405005C0405005704050052040500D7
:108F10004D04050048040500430405003E04040018
:108F20003A04050035040500300404002C04050053
:108F300027040400230405001E0404001A0404008E
:108F400016040500110404000D04040009040500C2
:108F50000404040000040400FC030400F8030400FB
:108F6000F4030400F0030400EC030400E80304002D
:108F7000E4030400E0030400DC030400D80304005D
:108F8000D4030400D0030400CC030400C80303008E
:108F9000C503030024F404D9201BC40C5C0E980400
:108FA000C4095F0265077101F405F900FB04B30011
:108FB00048048700C10369005803550003034500B6
:108FC000BE023A008402310053022A002902250021
:108FD00004022000E4011C00C8011900AF011700C1
:108FE0009801140084011300710110006101100048
:108FF00051010E0043010D0036010B002B010B0047
:1090000020010B00150109000C01090003010800F3
:10901000FB000800F3000800EB000700E400060076
:10902000DE000600D8000600D2000600CC000500D5
:10903000C7000500C2000500BD000400B90004001F
:10904000B5000400B1000400AD000400A900040054
:10905000A5000300A20003009F0004009B00030082
:1090600098000300950002009300030090000300A5
:109070008D0002008B0003008800020086000200C1
:1090800084000300810002007F0002007D000200D6
:109090007B000200790002007700010076000200E8
:1090A0007400020072000100710002006F000200F3
:1090B0006D0001006C0002006A00010069000200FE
:1090C0006700010066000100650001006400020005
:1090D0006200010061000100600001005F00020009
:1090E0005D0001005C0001005B0001005A0001000E
:1090F000590001005800010057000100560001000E
:10910000550001005400010053000000530001000D
:109110005200010051000100500001004F00010009
:109120004E0000004E0001004D0001004C00010007
:109130004B0000004B0001004A0001004900010003
:109140004800000048000100470001004600000000
:1091500046000100450000004500010044000100F8
:1091600043000000430001004200000042000100F3
:109170004100000041000100400001003F000000EC
:109180003F0001003E0000003E0001003D000000E5
:109190003D0001003C0000003C0000003C000100DC
:1091A0003B0000003B0001003A0000003A000100D3
:1091B00039000000390001003800000038000000CC
:1091C00038000100370000003700010036000000C1
:1091D00036000000360001003500000035000000B8
:1091E00035000100340000003400000034000100AC
:1091F00033000000330000003300010032000000A3
:109200003200000032000100310000003100000097
:10921000310001003000000030000000300001008B
:109220002F0000002F0000002F0000002F00010081
:109230002E0000002E0000002E0001002D00000076
:109240002D0000002D0000002D0001002C0000006A
:109250002C0000002C0000002C0001002B0000005E
:109260002B0000002B0000002B0001002A00000052
:109270002A0000002A0000002A0001002900000046
:109280002900000029000000290000002900010039
:10929000280000002800000028000000280000002E
:1092A0002800010027000000270000002700000020
:1092B0002700000027000100260000002600000013
:1092C0002600000026000000260001002500000006
:1092D00025000000250000002500000025000000FA
:1092E00025000100240000002400000024000000EC
:1092F00024000000240001002300000023000000DF
:1093000023000000230000002300000023000000D1
:1093100023000100220000002200000022000000C3
:1093200022000000220000002200010021000000B5
:1093300021000000210000002100000021000000A9
:10934000210000002100010020000000200000009A
:10935000200000002000000020000000200000008D
:1093600020000000200001001F0000001F0000007E
:109370001F0000001F0000001F0000001F00000071
:109380001F0001001E0000001E0000001E00000063
:109390001E00000045303A20005A3A2000593A2079
:1093A00000583A20004D53312C4D53322050696EF5
:1093B0007300504944204175746F74756E65206662
:1093C000696E6973686564212050757420746865DE
:1093D000206C617374204B702C204B6920616E648B
:1093E000204B6420636F6E7374616E7473206672B9
:1093F0006F6D2061626F766520696E746F20436FB8
:109400006E66696775726174696F6E2E6800504987
:1094100044204175746F74756E65206661696C6572
:1094200064212074696D656F75740020403A0054A2
:109430003A00423A00504944204175746F74756E89
:1094400065206661696C6564212054656D70657284
:10945000617475726520746F6F2068696768002099
:109460004B643A2000204B693A2000204B703A2090
:109470000020436C617373696320504944200020CD
:1094800054753A2000204B753A2000206D61783ADF
:109490002000206D696E3A200020643A200020628E
:1094A0006961733A2000504944204175746F7475A6
:1094B0006E65207374617274005049442041757464
:1094C0006F74756E65206661696C65642E204261FB
:1094D00064206578747275646572206E756D62655E
:1094E000722E00486F74656E642066616E20737022
:1094F000656564206973206C6F776572207468619C
:109500006E206578706563746564005072696E746E
:109510002066616E207370656564206973206C6FCE
:10952000776572207468616E206578706563746514
:1095300064004D494E54454D5020424544004D492C
:109540004E54454D50004D415854454D50004D41ED
:109550005854454D50204245440070012C01900163
:109560002701B0012201C0011D01F0011801100204
:10957000130130020E016002090190020401C002D1
:10958000FF000003FA004003F5008003F000D00361
:10959000EB002004E6007004E100E004DC0040057C
:1095A000D700C005D2004006CD00D006C800800715
:1095B000C3003008BE00F008B900C009B400B00A0A
:1095C000AF00B00BAA00D00CA500000EA000500FF9
:1095D0009B00C01096005012910000148C00C01522
:1095E0008700B0178200B0197D00D01B7800001EE4
:1095F000730040206E0090226900F0246400402730
:109600005F0090295A00E02B5500102E50002030AA
:109610004B0010324600E033410090353C001037DB
:10962000370070383200A0392D00B03A2800A03B36
:109630002300603C1E00103D1900903D1400103EB8
:109640000F00703E0A00C03E0500003F00002048A9
:109650004F54454E4420544845524D414C2052559C
:109660004E415741590020484541544245442054F9
:109670004845524D414C2052554E41574159005496
:109680004845524D414C2052554E41574159004298
:10969000454420544845524D414C2052554E415767
:1096A00041590020544845524D414C2052554E419D
:1096B00057415920285052454845415420484F545D
:1096C000454E44290020544845524D414C205255A6
:1096D0004E41574159202850524548454154204851
:1096E0004541544245442900505245484541542083
:1096F0004552524F52004245442050524548454140
:1097000054204552524F5200207472696767657247
:1097100065642100486561746572732073776974AC
:1097200063686564206F66662E20003A20004572EB
:10973000723A200000FF0102010002FFFFFE00015B
:10974000FE01FF00506C6561736520726573746182
:109750007274005553415254322072782046756C11
:109760006C212121003A2000252D31322E31325337
:10977000252D642F36002533642F252D33640020DA
:109780003A200025335300252D377300252D313520
:109790002E313553252D35640A252D31352E3135A1
:1097A00053252D35640A0025530A20252D31362EE8
:1097B000313653252D33640A20252D31362E31368E
:1097C00053252D33640025530A20252D31362E31A3
:1097D0003653252D33640A20252D31362E3136534C
:1097E000252D33640A20252D31362E313653252D73
:1097F00033640025530A20252D31362E313653256A
:109800002D33640A25530A20252D31362E31365347
:10981000252D33640A0020257325336481200A0036
:1098200025752E25752E25752E2575002000200006
:10983000466C6173684169722049502041646472CA
:109840003A004D4D5520202020202020204E2F4131
:109850000025642E25642E2564002046573A0032E8
:109860003032352D30342D32320045334476366671
:10987000756C6C0052414D426F31306100315F3781
:10988000356D6D5F4D4B32350020486173683A3756
:10989000373331303234656400205265706F3A706E
:1098A0007275736133640020332E31342E312D38BC
:1098B000323739004669726D776172653A003E0051
:1098C000464C4558202D20203234302F353000466C
:1098D0004C4558202D20203234300050502020207C
:1098E0002D20203235342F313030005050202020B0
:1098F0002D20203235340048495053202D2020326D
:1099000032302F3130300048495053202D20203242
:1099100032300041425320202D20203235352F3166
:1099200030300041425320202D2020323535005068
:10993000412020202D20203237352F393000504152
:109940002020202D20203237350050564220202D57
:1099500020203231352F37350050564220202D201F
:10996000203231350050432020202D202032373541
:109970002F3130350050432020202D202032373524
:109980000041534120202D20203236302F313035F8
:109990000041534120202D202032363000504554C4
:1099A00020202D20203233302F38350050455420D0
:1099B000202D202032333000504C4120202D2020FB
:1099C0003231352F363000504C4120202D202032AE
:1099D0003135006E6F7A7A6C65202D20203235305B
:1099E0002F30006661726D2020202D20203235300E
:1099F0002F3830001000C90210012C014001220153
:109A000070011801B0010E01F00104015002FA00CA
:109A1000B002F0003003E600D003DC009004D20076
:109A20007005C800A006BE000008B400B009AA0076
:109A3000D00BA000600E960060118C000015820013
:109A400020197800C01D6E00A0226400B0275A00C3
:109A5000902C500000314600E0343C0010383200B9
:109A6000903A2800603C1E00A03D1400803E0A0091
:109A7000203F00004D6561737572652063656E74EB
:109A8000657220200078797A63616C5F6D6561731F
:109A90007572655F656E7465720A0078797A6361C4
:109AA0006C5F73706972616C382063783D25642047
:109AB00063793D2564207A303D256420647A3D2514
:109AC00064207261646975733D25642061643D257D
:109AD000640A0078797A63616C5F736561726368A8
:109AE0005A206E6F207369676E616C0A20783D257D
:109AF0006C6420793D256C64207A3D256C640A00F5
:109B0000204F4E2D5349474E414C20617420783DE3
:109B1000256420793D2564207A3D25642061643DDB
:109B200025640A0078797A63616C5F73656172639A
:109B3000685A20783D256C6420793D256C64207A34
:109B40003D256C640A002530327800205B256620B4
:109B500025665D206D6D207061747465726E206382
:109B6000656E7465720A00205B25662025665D5B64
:109B700025665D206D6D20646976657267656E632C
:109B8000650A000000F000F801FC03FE07FE07FE76
:109B900007FE07FC03F801F000000000000000F0E1
:109BA00000F801FC03FC03FC03FC03F801F00000D7
:109BB00000000078797A63616C5F6D65617375721E
:109BC000655F6C656176650A00203C200057415254
:109BD0004E494E473A2046726F6E7420706F696E20
:109BE00074206E6F7420726561636861626C652EAB
:109BF000205920636F6F7264696E6174653A00006A
:109C0000000040410000804000005C4300008040B4
:109C100000005C4300004443000040410000444316
:109C200025642F3400497465726174696F6E3A203F
:109C30000043616C6962726174696F6E206661696C
:109C40006C65642120436865636B207468652061DE
:109C500078657320616E642072756E20616761693A
:109C60006E2E0078797A63616C5F73706972616CD3
:109C7000322063783D25642063793D2564207A3065
:109C80003D256420647A3D256420726164697573A2
:109C90003D25642061643D25640A000A00436F7518
:109CA0006E74646F776E3A202564200025640A0084
:109CB0005363616E20636F756E74646F776E3A20C4
:109CC000005061747465726E2063656E74657220F5
:109CD0005B25662025665D2C206D617463682025F8
:109CE0006625250A00205B25662C2025665D5B2500
:109CF000665D2066696E616C20636972636C650ADB
:109D0000000000A0400000A0400000004000007AD9
:109D100043000056439AD95143FFFFFFE02D903E88
:109D20008988B24111369C3E7777C14129CBB03E3C
:109D3000EFEEDA41BA49CC3EEFEEFC4161C3F33EAF
:109D4000EFEE16429CA2133FCDCC36428AB0113FB3
:109D5000ABAA56428863DD3DABAA5642B8AF433F3B
:109D6000555572421826533F33B38242302A593F29
:109D7000EF6E8642000070C10000C8420000C4C1FE
:109D80000000A0410000E0C000002041000060C0D1
:109D90000000C0400000A0412222F2400000A0C10B
:109DA0009A99A14000000CC255550542436F6F6C53
:109DB000696E672074696D65722073746F70706569
:109DC000640048656174657220636F6F6C646F77BF
:109DD0006E00436F6F6C696E672054696D656F75B7
:109DE00074207374617274656400536176696E6780
:109DF00020616E64207061726B696E6700486561F6
:109E000074657220636F6F6C646F776E2070656E1F
:109E100064696E6700526573756D696E6720585985
:109E20005A0057726974696E6720746F2066696C96
:109E3000653A200046696C6520616C7265616479E1
:109E4000206F70656E656400BA5AA95A955A805A97
:109E50006A5A575A415A2D5A1C5A065A955AA95AA3
:109E6000F259E359CF59BE59A959ED619359815916
:109E70006E595D594859355921590C590359F158B2
:109E8000DC584D363030204155544F0046494E4441
:109E9000412066696C616D656E742072756E6F75B8
:109EA000742100436F6D6D756E69636174696F6EC7
:109EB0002074696D656F75740050726F746F636F95
:109EC0006C204572726F72000300035665727369ED
:109ED0006F6E206D69736D6174636800436F6D6DA3
:109EE000616E64204572726F7200436F6D6D616EBA
:109EF000642072656A6563746564004D4D55204247
:109F00007574746F6E207075736865640052657443
:109F10007279427574746F6E507265737365640004
:109F2000175D025DEB5CD65CC15CAD5C9D5C865CE4
:109F30006F5C585C445C305C1A5C1A5C1A5C055CB3
:109F4000055C055CF25BF25BF25BDF5BDF5BDF5BBA
:109F5000C85BC85BC85BB35BB35BB35B9D5B9D5B7E
:109F60009D5B8D5B785B625B4C5B3D5B305B195B43
:109F7000065BF45AE15ACF5ABF5A427574746F6E39
:109F800000436865636B55736572496E7075742D17
:109F900062746E4C4D522000526573657452657444
:109FA0007279417474656D7074730046493A20206B
:109FB00046533A202020203E20208220202081006D
:109FC000486F74656E642074656D70657261747538
:109FD0007265207265616368656400526573756DB2
:109FE000696E672054656D7000436F6F6C646F77A6
:109FF0006E20666C616720636C6561726564002029
:10A00000573A0020453A00543A004E6F20307846C7
:10A01000462072656365697665640053656E6469A0
:10A020006E6720307846460046696C652073656C23
:10A030006563746564002053697A653A2000466957
:10A040006C65206F70656E65643A20004E6F7720F6
:10A0500066726573682066696C653A20004E6F779A
:10A0600020646F696E672066696C653A2000222063
:10A07000706F73002220706172656E743A22005313
:10A080005542524F5554494E452043414C4C207443
:10A0900061726765743A2200747279696E67207420
:10A0A0006F2063616C6C207375622D67636F6465EC
:10A0B0002066696C6573207769746820746F6F20FF
:10A0C0006D616E79206C6576656C732E00062833A1
:10A0D000D036C23E013F154132423B43F2443B453C
:10A0E000F24622473B48F2493B4AF05898590C5AED
:10A0F000085B0C5C086110679B6E2271077208FF99
:10A10000095A0D000EF019145E0820642B6D322FD1
:10A11000FF2022257322002025236C780044495219
:10A120005F45584954004449525F454E5445523AA0
:10A1300020257320222573220A006175746F25691A
:10A140002E6700041A44656372656D656E7452650E
:10A15000747279417474656D70747300081B1C0B04
:10A1600014525354436F6D6D54696D656F7574006F
:10A170002C206C6173742062797465733A2000221C
:10A18000206661696C65643A204275666665722076
:10A1900066756C6C21002200456E717565696E678D
:10A1A00020746F207468652066726F6E743A202286
:10A1B000004572726F723A004D4D5532746F6F6C7C
:10A1C0003D004D4D55323A004D4D55323A006563D4
:10A1D000686F3A003E53302A63362E004D4D5520AD
:10A1E00069732000F2379F6311241FBECFEFD1E2C5
:10A1F000DEBFCDBF00E00CBF13E0A0E0B2E0E2EDB7
:10A20000F4E503E00BBF02C007900D92A230B10746
:10A21000D9F727E1A2E0B3E001C01D92A731B20750
:10A22000E1F710E5C3EFD0E500E006C02197010992
:10A23000802FFE010F94ADA4C23FD10780E0080734
:10A24000A9F70E9432EB0D9457AA0C94CF842F9259
:10A250003F924F925F926F927F928F929F92AF92B6
:10A26000BF92CF92DF92EF92FF920F931F93CF9303
:10A27000DF93CDB7DEB72F970FB6F894DEBF0FBED2
:10A28000CDBF6C011B015A01FC011782168283812C
:10A290009E012F5F3F4F490181FDD2C08FEF9FEF9D
:10A2A000EEC2F12C512C00E0003238F48B3209F16F
:10A2B00090F48032F9F0833209F107FD34C020EDCB
:10A2C000280F2A3020F506FF1BC0FAE0FF9E200D64
:10A2D0001124F22E05C08D3279F0803371F70160C0
:10A2E000F10193FD859193FF81911F018111DCCFD5
:10A2F0001AC002600460F4CF0860F2CF0061F0CFB2
:10A300003AE0539E200D1124522E0062E9CF8E3286
:10A3100021F406FDB1C20064E3CF8C3611F400686D
:10A32000DFCF8836E9F29BEB980F933008F05FC0DF
:10A330000061805E06FD02C046E0F42E102F1F7300
:10A34000853609F05BC0106417FF61C08F2D9BE359
:10A350009F1508F48BE344244394480E27E035010D
:10A36000F4E06F0E711CF50160817181828193812F
:10A37000042DA4010F9456A05C01F981FC87F0FF25
:10A3800003C00DE2F3FF07C00BE211FD04C0012F73
:10A39000047012FD00E22C852C70E22E09F46BC0D3
:10A3A0000111D8C2F3E0E12CF515A0F483E0E52C0F
:10A3B000E81A13FD08C0B60180E290E00F9405A2F0
:10A3C000EA94E110F8CF002329F0B601802F90E045
:10A3D0000F9405A23C8528E7A22E21E7B22E33FD7B
:10A3E00004C09CE7A92E91E7B92E107122C09BE909
:10A3F000980F933008F047C10F7E9CCF863611F43A
:10A400001068A2CFFF2009F49FCFFA949DCFE7E018
:10A410002F2DEF1518F427E037E0F32E412C9FCFB6
:10A4200011118052B60190E00F9405A28FEFA81A87
:10A43000B80AF50184918111F3CFE11084C2530170
:10A44000F6019381F10193FD859193FF81911F01A5
:10A45000882309F411C2853241F493FD859193FF5D
:10A4600081911F01853209F01CCFB60190E00F9455
:10A4700005A23501E4CF17FF6FC04A0CFC85F4FF3D
:10A4800004C08A81813309F44A9414140CF086C004
:10A4900028E0241510F488E0482E85E090E017FFAE
:10A4A00006C0C501B7FE02C090E080E00196011130
:10A4B0000196FF2031F02F2D30E02F5F3F4F820FAC
:10A4C000931F5816190619F014F0E52CE81A812F7D
:10A4D000897011F4E11067C0002329F0B601802FC4
:10A4E00090E00F9405A213FD02C0E11063C017FFB6
:10A4F0007CC08501B7FE02C010E000E0C5018419F0
:10A5000091092C016F2D70E0EE27FF27E61BF70B5A
:10A51000FF87EE870F3F100729F4B6018EE290E027
:10A520000F9405A2A016B1060CF44BC040165106BC
:10A530000CF047C0F501E01BF10BE80DF91D81811E
:10A54000015011092E853F8502171307E4F1B6016A
:10A5500090E00F9405A2DECF16FD9FCFEF2DF0E027
:10A56000EA15FB0534F03CEFA3163FEFB3060CF001
:10A5700010683296E80DF91D01C0FA94FF2019F019
:10A5800082918033D1F317FF88CF442443944F0C3A
:10A59000FA141B0431F02CF0FA187FCF44244394B2
:10A5A0007CCFF12C7ACFB60180E290E00F9405A227
:10A5B000EA9490CFB60180E390E00F9405A2EA946C
:10A5C00094CF80E3BDCFA016B10641F49A819633B3
:10A5D00050F4953319F43C8534FF05C0B60190E082
:10A5E0000F9405A22ACF81E3F9CF8A81813319F034
:10A5F0009C859F7E9C87B60190E00F9405A2FF206A
:10A60000A9F0B6018EE290E00F9405A2F394F394C2
:10A61000E2E001E00E0FE80DF92DF11D8081B60199
:10A6200090E00F9405A2E02F0F11F3CF85E690E0A4
:10A6300014FF02C085E490E0B6010F9405A2B7FCB8
:10A6400006C0A114B104C1F4EC85E4FF15C0B194B7
:10A65000A194B1088DE2B60190E00F9405A280E3C9
:10A660002AE0A216B10454F4B60190E00F9405A2BA
:10A67000B601C501C096B4CF8BE2EDCF8F5FFAE093
:10A68000AF1AB108EDCF8336C9F0833771F1833546
:10A6900009F05BC03501F2E06F0E711CF501A0807E
:10A6A000B1806F2D70E006FD02C06FEF7FEFC50136
:10A6B0000F9499A19D878C8700680DC0350132E009
:10A6C000630E711CF5018081898321E030E03D87B4
:10A6D0002C8754010F7703FD06C02C853D8552164B
:10A6E000130609F0A8F4E52C2BC0350132E0630E07
:10A6F000711CF501A080B1806F2D70E006FD02C0D5
:10A700006FEF7FEFC5010F94BEA19D878C87E2CFCD
:10A71000B60180E290E00F9405A25A94DECFF501D5
:10A7200007FD859107FF81915F01B60190E00F94CD
:10A7300005A2E110EA948C859D8501979D878C8701
:10A74000EC85FD85EF2B59F778CE843619F08936E4
:10A7500009F074C0350107FF66C0F4E06F0E711C8C
:10A76000F5016081718182819381102F1F7697FF9F
:10A7700008C090958095709561957F4F8F4F9F4F42
:10A7800010682AE030E0A4010F942CA3A82EA8188A
:10A79000BA2C012F16FF0AC00E7FAF1438F414FF35
:10A7A00004C012FD02C0012F0E7EBF2C04FFA3C007
:10A7B000FE01EA0DF11D8081803309F095C0097E0C
:10A7C000F02FF870EF2E03FDA5C000FF9FC0FA2CFC
:10A7D000B51410F4F50CFB1804FFA2C0B60180E319
:10A7E00090E00F9405A202FF09C088E790E001FF06
:10A7F00002C088E590E0B6010F9405A2AF1408F4FA
:10A800009BC0AA940A2D10E00F5F1F4F080D191D61
:10A81000F80182918F01B60190E00F9405A2801695
:10A820009106B1F70ACEF2E06F0E711CF50160815E
:10A830007181072E000C880B990B97CF102F85374D
:10A84000A9F41F7E2AE030E0350117FF44C0F4E090
:10A850006F0E711CF5016081718182819381A40169
:10A860000F942CA3A82EA8181F7792CF197F8F368C
:10A8700079F1F0F4883539F1F601868197812F96C8
:10A880000FB6F894DEBF0FBECDBFDF91CF911F9101
:10A890000F91FF90EF90DF90CF90BF90AF909F907F
:10A8A0008F907F906F905F904F903F902F90089582
:10A8B000803739F0883701F714FD146020E130E06B
:10A8C000C3CF1061F9CF04FD166020E132E0BCCFA8
:10A8D00028E030E0B9CFF2E06F0E711CF501608125
:10A8E000718190E080E0BBCF02FD02C0B39468CFDD
:10A8F000B394B39465CF802F867809F461CFF6CFF7
:10A90000B60180E290E00F9405A2B394B514C0F3B1
:10A91000E12C62CFE52CEB18B51408F45DCFF8CF2D
:10A92000802F867809F46ACF8BE201FF80E207FD71
:10A930008DE2B60190E060CFB60180E390E00F9425
:10A9400005A2FA945BCFB60180E290E00F9405A2D5
:10A95000EA9473CD24E0E12C251508F036CD84E08F
:10A9600026CD20E030E040E85FEB60917E02709100
:10A970007F0280918002909181020F94BAA5882372
:10A9800021F1E0913812F0913912E55BFF4E8081A0
:10A990008B7F8230D1F480E1EEE7F2E0A1E6B2E114
:10A9A00001900D928A95E1F780E090E0A0E8BFEB7E
:10A9B00080937E0290937F02A0938002B0938102E5
:10A9C00080914D1290914E12089581E090E008958B
:10A9D00080E1E9E2F6E0A1E6B2E101900D928A950C
:10A9E000E1F70895E0E5F6E7833021F0E82FF0E0A5
:10A9F000E35BF94884910895809142059091430565
:10AA00002091440530914505821B930B8F77992740
:10AA10000895982F9F7083FF0DC080917B00886000
:10AA200080937B0080917C00887F9770892B809336
:10AA30007C00089580917B00877FF2CF4FEF5FEF1E
:10AA4000BA0185EE9FE00F94D3A34FEF5FEFBA01F9
:10AA500089EE9FE00F94D3A34FEF5FEFBA018DED26
:10AA60009FE00F94D3A34FEF5FEFBA0181EE9FE019
:10AA70000F94D3A34FEF5FEFBA0185ED9FE00F94E2
:10AA8000D3A34FEF5FEFBA0189ED9FE00F94D3A3FB
:10AA90004FEF5FEFBA0185EC9FE00F94D3A34FEF28
:10AAA0005FEFBA0189EC9FE00F94D3A34FEF5FEF04
:10AAB000BA018DEC9FE00F94D3A34FEF5FEFBA0183
:10AAC00081ED9FE00D94D3A380369105F8F4409179
:10AAD0003812509139122091491030914A10421782
:10AAE000530739F460913C1270913D121616170607
:10AAF0006CF0B901680F791FFB01E359FF4F241770
:10AB0000350730F481E04E175F0708F480E00895C0
:10AB1000EE3EF140F8F06C5F7F4F6E3E714018F4EE
:10AB200049365105B8F483599F4F4817590770F3B8
:10AB30004DEE51E0421B530B70E060E0C901855BB4
:10AB40009F4E0F94CFA98FB7F89410924A1010928D
:10AB500049108FBF81E0089580914405909145058B
:10AB600090934305809342058CEE99E69F938F93D3
:10AB700080913E1290913F12A0914012B0914112EB
:10AB80000196A11DB11DBF93AF939F938F938BE44B
:10AB900094E69F938F9382E594E69F938F930F940F
:10ABA0005FA28DB79EB70A960FB6F8949EBF0FBEF0
:10ABB0008DBF08950F931F93CF93DF93EC01C60FC2
:10ABC000D71F8C179D0779F08C010F5F1F4F0F94D3
:10ABD0009DA38F3F31F081E0DF91CF911F910F91C5
:10ABE0000895C801EECF80E0F7CF682F880F770B6C
:10ABF0008091381290913912825B9F4E0F94F4A984
:10AC00009C019093BC048093BB0481E0232B09F446
:10AC100080E008958091BB049091BC044AE050E02C
:10AC200070E060E001960F94289F862F0895809130
:10AC3000BB049091BC044AE050E070E060E00196F3
:10AC40000F94289FCB0108950F931F93CF93DF9309
:10AC50008C01862FEA010E94F555882319F10E9484
:10AC600017569C0197FF03C0319521953109253670
:10AC700031059CF09F938F9381EB91EA9F938F9383
:10AC80008DEC96E79F938F930F945FA20F900F9098
:10AC90000F900F900F900F9080E0DF91CF911F9158
:10ACA0000F910895F80180818823B1F3CE01DF91DF
:10ACB000CF911F910F910D949DA38091BB04909112
:10ACC000BC044AE050E070E060E001960D94289FDB
:10ACD00060E086E69FE00F94C1A360E088E69FE015
:10ACE0000F94C1A360E085E69FE00F94C1A360E0EC
:10ACF00084E69FE00F94C1A360E082ED9EE00F9494
:10AD0000C1A360E08FEC9EE00D94C1A32F923F920F
:10AD10004F925F926F927F928F929F92AF92BF926B
:10AD2000CF92DF92EF92FF920F931F93CF93DF9317
:10AD3000CDB7DEB7CC58D2400FB6F894DEBF0FBE09
:10AD4000CDBFCB58DD4F688379838A839B83C557FA
:10AD5000D240FE01E754FE4F88E2DF011D928A9542
:10AD6000E9F7E85BF1401F0180E991E0DF01FC01B8
:10AD70001D923197E9F7C75ADD4F19821882C955DC
:10AD8000D2409E012F513E4FC159DD4F3983288358
:10AD9000CF56D2408E01075A1D4FCE018F5C9D4F7A
:10ADA000C359DD4F99838883CD56D2403C01490178
:10ADB00040EBA42E4FE0B42E53E2C52ED12CF12C43
:10ADC000E12CB6010D2C000C880B990B0F942B9ED7
:10ADD000D4016D937D938D939D934D01F801619105
:10ADE00071918F01072E000C880B990B0F942B9EED
:10ADF000D3016D937D938D939D933D01BFEFEB1A2E
:10AE0000FB0AE6E0EE16F10409F038C3CB58DD4F3B
:10AE1000288139814A815B81C557D240C159DD4FB4
:10AE2000A881B981CF56D2406D917D918D919C9131
:10AE30000F944EA7412C512C320118160CF402C36A
:10AE4000C359DD4F08811981CD56D2400C5E1F4F8A
:10AE5000C159DD4FE880F980CF56D240B4E1EB0E06
:10AE6000F11C6E01EFEDCE1AEDEFDE0A9E012B55BF
:10AE70003E4FCF58DD4F39832883C157D240D80188
:10AE80004D905D906D907C90F70160817181828121
:10AE90009381D7015E914E913E912E917D010F9449
:10AEA000C4A44B015C01F80152914291329122916C
:10AEB0008F01C301B2010F94C4A4A50194010F94A2
:10AEC000C4A5D6019E938E937E936E936D01CF5849
:10AED000DD4FE881F981C157D240B292A29292929D
:10AEE0008292CF58DD4FF983E883C157D240C359CE
:10AEF000DD4F28813981CD56D2400217130709F062
:10AF0000BECF4E013FE6831A3EEF930A5E0183EF08
:10AF1000A81A8DEFB80A61018101EE24E394F12CA7
:10AF2000D4014D905D906D907D904D012D913D919E
:10AF30004D915C91C301B2010F94C5A49B01AC017A
:10AF40000F94C5A4F80164A775A786A797A7F1E099
:10AF5000EF16F10461F0D80198964D925D926D92D2
:10AF60007C929B97F8014482558266827782FFEF3C
:10AF7000EF1AFF0AF501208131814281538184E07B
:10AF8000A80EB11C64817581868197810F94C4A439
:10AF900020E030E040EC50E40F946A9ED601DC964D
:10AFA0006D937D938D939C93DF97045D1F4FB8E263
:10AFB000CB0ED11CE5E0EE16F10409F0B1CF7E0115
:10AFC000FDE2EF0EF11C28E2A22EB12C00EB1FEFE8
:10AFD00024E0220E311CD7012D913D914D915C91C1
:10AFE000139798966D917D918D919C919B970F945D
:10AFF000C4A52B013C016101C01AD10A88248394A5
:10B00000912CF601E00FF11FEA0DFB1D208131812B
:10B0100042815381C301B2010F946A9E9B01AC012E
:10B02000F60160817181828193810F94C4A4D6015D
:10B030006D937D938D939D936D01BFEF8B1A9B0A4A
:10B04000E6E08E169104E9F63CE2E30EF11C0852AC
:10B05000110988E2A80EB11C08339FEF190709F007
:10B06000BACF1E01F5EB2F0E311C6E0121EBC20E83
:10B07000D11C7E0137E3E31A3EEFF30A04E010E04F
:10B080004801B12CA12C412C512C3201F601EA0DC2
:10B09000FB1DD701AA0DBB1D2D913D914D915C91DA
:10B0A00060817181828193810F946A9E9B01AC01C2
:10B0B000C301B2010F94C5A42B013C018FEF881A84
:10B0C000980A94E0A90EB11CA5E08A169104F1F645
:10B0D000A3019201F10160817181828193810F94BA
:10B0E000C4A4D6012D913D914D915C910F94C4A5BE
:10B0F000F701608371838283938301501109F8E221
:10B100002F1A31082CE2C21AD10834E0E31AF108F0
:10B110000115110509F0B4CFCB50DE4F888199811C
:10B12000AA81BB81C55FD140CF57DD4F888399830A
:10B13000AA83BB83C158D2401E0197E4291A9EEF0F
:10B14000390A10E000E0C159DD4FA881B981CF561E
:10B15000D240CD90DD90ED90FD90C159DD4FB98387
:10B16000A883CF56D240CB58DD4F288139814A8100
:10B170005B81C557D240C701B6010F94BAA5181616
:10B18000B4F0CB58DD4F288139814A815B81C557A6
:10B19000D240C159DD4FE881F981CF56D24060815C
:10B1A0007181828193810F944EA787FF18C004306C
:10B1B000110509F030C1CB58DD4F288139814A8112
:10B1C0005B81C557D240CF57DD4F688179818A8135
:10B1D0009B81C158D2400F94BAA587FF1CC1D101F1
:10B1E00014968D909D90AD90BC9017978D919D91E8
:10B1F0000D90BC91A02DCF58DD4F88839983AA83F1
:10B20000BB83C157D240F801EE0FFF1FEE0FFF1FA7
:10B2100021E931E02C0F3D1FE20FF31F40805180E8
:10B2200062807380C359DD4FA881B981CD56D24069
:10B230008D919D910D90BC91A02DC358DD4F8883B9
:10B240009983AA83BB83CD57D240A7019601CB58DF
:10B25000DD4F688179818A819B81C557D2400F94E7
:10B26000C4A46B017C0120E030E040E450E40F9482
:10B2700035A8CB57DD4F688379838A839B83C55874
:10B28000D240C358DD4F288139814A815B81CD5737
:10B29000D240C359DD4FE881F981CD56D240648157
:10B2A0007581868197810F94C4A4A30192010F94A4
:10B2B000C4A5C758DD4F688379838A839B83C957A8
:10B2C000D240A3019201C301B2010F94C5A4CF588B
:10B2D000DD4F288139814A815B81C157D2400F946B
:10B2E0006A9EC757DD4F688379838A839B83C958D9
:10B2F000D240A3019201C501B4010F946A9E9B0143
:10B30000AC01C757DD4F688179818A819B81C9581B
:10B31000D2400F94C5A420E030E040EC50E40F94FC
:10B32000C4A59B01AC01C758DD4F688179818A8132
:10B330009B81C957D2400F94C4A4A70196010F94D2
:10B340006A9EC758DD4F688379838A839B83C95778
:10B35000D240CF58DD4F288139814A815B81C15766
:10B36000D240C501B4010F94C4A44B015C0120E09C
:10B3700030E040EC50E4C301B2010F946A9E9B019F
:10B38000AC01C501B4010F94C4A5CB57DD4F288192
:10B3900039814A815B81C558D2400F946A9E4B0126
:10B3A0005C0120E030E040E05FE3CF58DD4F688192
:10B3B00079818A819B81C157D2400F946A9E2B016B
:10B3C0003C01A7019601C701B6010F946A9E9B013B
:10B3D000AC01C301B2010F946A9E9B01AC01C5018F
:10B3E000B4010F94C5A49B01AC01C758DD4F68811F
:10B3F00079818A819B81C957D2400F94C5A4C358D3
:10B40000DD4F288139814A815B81CD57D2400F942D
:10B41000C5A42B013C010F5F1F4FF4E02F0E311C20
:10B42000C359DD4F28813981CD56D2402C5F3F4F23
:10B43000C359DD4F39832883CD56D24005301105DD
:10B4400009F081CEC301B201C457DD4F0FB6F894A5
:10B45000DEBF0FBECDBFDF91CF911F910F91FF9047
:10B46000EF90DF90CF90BF90AF909F908F907F90A4
:10B470006F905F904F903F902F900895C5010F946B
:10B48000ABA3D8018D939C93B5E0CB0ED11CE2E029
:10B49000AE0EB11C96CC0F931F93CF932091011346
:10B4A000213079F58C0180E50E94F555882349F11A
:10B4B0000E940A56C82F853020F5013C82E018070B
:10B4C00049F0023C124069F08C2FCF911F910F91EF
:10B4D0000D94469D60E08C2FCF911F910F910D949C
:10B4E000899D8EEC9EE00F949DA3882351F00F94CC
:10B4F0006379882331F08C2FCF911F910F910D9498
:10B50000069ECF911F910F9108958F929F92AF92B7
:10B51000BF92CF92DF92EF92FF920F931F93CF9340
:10B52000DF930091BB041091BC040F5F1F4F6801B3
:10B530008FEFC81AD80AD801DC918D2F90E00F94B4
:10B540002EA17C01892B01F5DD3201F56801B2E005
:10B55000CB0ED11CF801D181C1E086010150110947
:10B5600043E050E064E876E7C8010F9464A1892BBA
:10B57000C1F460E070E080E89FEFC111DBC060E0E3
:10B5800070E080E89FE7D6C08601D1CFDB3239F486
:10B590006801F2E0CF0ED11CD8011196DC91C0E019
:10B5A000DCCF43E050E061E876E7C8010F9464A186
:10B5B000892B09F4CCC0F60110E000E020E030E077
:10B5C000A9016F01D053DA3060F5BC2E6894B1F850
:10B5D0008C2F8870C2FF09C0811102C00F5F1F4FFE
:10B5E0003196D601DC91CB2DECCF882311F00150A0
:10B5F0001109A5E0B0E00F9432A49B01AC01220F29
:10B60000331F441F551F2D0F311D411D511D28395A
:10B61000B9E93B074B07B9E15B0710F3C660BC2EE5
:10B62000DFCFDE3F31F4C3FD33C0BC2E6894B3F8E6
:10B63000D7CFD53369F580818D3231F4C061BF0138
:10B640006E5F7F4F818105C0BF018B32C9F36F5F91
:10B650007F4F80538A30E0F4FB01B0E8EB16BCE08A
:10B66000FB065CF4B701660F771F660F771FE60EC7
:10B67000F71EEE0CFF1CE80EF11C819180538A30FE
:10B6800060F3C4FF03C0F194E194F1080E0D1F1D97
:10B69000CA01B9010F94299EC370C33009F49058B0
:10B6A0004B015C0120E030E0A9010F94BAA588238A
:10B6B00009F43EC0CDE7D6E717FF05C01195019507
:10B6C0001109C5E6D6E76E01E8E1CE1AD10880E29D
:10B6D000E82EF12C0DC0FE01259135914591549134
:10B6E0000E191F09C501B4010F946A9E4B015C013C
:10B6F000D501C4010E151F0574F72497F594E7943E
:10B70000CC16DD06A9F78A2F880F8B2F881F8F3F55
:10B7100049F020E030E0A901C501B4010F94BAA5B9
:10B72000811106C082E290E090930C1780930B1772
:10B73000C501B401DF91CF911F910F91FF90EF9060
:10B74000DF90CF90BF90AF909F908F90089560E072
:10B7500070E080EC9FE7EECF2F923F924F925F9286
:10B760006F927F928F929F92AF92BF92CF92DF9211
:10B77000EF92FF920F931F93CF93DF93CDB7DEB776
:10B78000A1970FB6F894DEBF0FBECDBF84EC92E058
:10B790009D8F8C8F81E6282E82E1382E09E216E0FB
:10B7A00091E09A8F198EEC8DFD8D8191FD8FEC8F3C
:10B7B0000E94F555E82E882309F454C1F0905712E1
:10B7C000FA8DFF220E94855A2B013C01F80140822C
:10B7D000518262827382F98DF33009F045C0DD2415
:10B7E000D394F11001C0D12C8090100290901102DE
:10B7F000A0901202B090130220E030E040E85FE336
:10B80000C501B4010F94BAA5882359F1F11015C0F0
:10B8100020916D1230916E1240916F125091701202
:10B82000C301B2010F94C4A4609335067093360629
:10B830008093370690933806DE2CA5019401609121
:10B8400035067091360680913706909138060F9430
:10B850006A9E609335067093360680933706909300
:10B860003806D11003C05FC0FF2089F0F1012081AC
:10B87000318142815381F80160817181828193819C
:10B880000F94C5A4F8016083718382839383F98D3B
:10B89000F230D9F58091BB03823009F0EEC08CE024
:10B8A000E0EAF2E0DE011D9601900D928A95E1F743
:10B8B0008CE0ECEAF2E0DE01119601900D928A959F
:10B8C000E1F7C0903106D0903206E0903306F09058
:10B8D000340620E030E0A901C701B6010F94BAA5F3
:10B8E00087FF52C0CE0101967C01D12CF7016191F6
:10B8F0007191819191917F010F9436A68D2D0F94B6
:10B900001318D394F3E0DF12F1CFF98DFF5FF98FB5
:10B910008A8D880F8A8F94E0290E311C0C5F1F4F8F
:10B92000F43009F040CF86E40E94F555882399F061
:10B930000E94855A6B017C0120E030E0A9010F9440
:10B940004EA7181644F4C0927A02D0927B02E0927D
:10B950007C02F0927D02A1960FB6F894DEBF0FBE76
:10B96000CDBFDF91CF911F910F91FF90EF90DF90AE
:10B97000CF90BF90AF909F908F907F906F905F908F
:10B980004F903F902F90089520E030E048E453E43A
:10B99000C701B6010F944EA71816A4F4CE010D9658
:10B9A0007C01D12CF70161917191819191917F017D
:10B9B0000F9436A68D2D0F941318D394F3E0DF1255
:10B9C000F1CFA3CFCE01019699A388A3FE013D96A6
:10B9D000FF8FEE8F1B8EE8A1F9A1C190D190E1906D
:10B9E000F190F9A3E8A3EE8DFF8D619171918191A2
:10B9F0009191FF8FEE8FA70196010F94C4A420E0D0
:10BA000030E048E453E40F94C4A54B015C0120915D
:10BA100031063091320640913306509134060F942E
:10BA20006A9E2B013C0120E030E0A901C501B40170
:10BA30000F946A9E9B01AC01C701B6010F94C4A488
:10BA40009B01AC01C301B2010F94C5A40F9436A6AB
:10BA50008B8D0F941318FB8DFF5FFB8FF33009F074
:10BA6000BACF53CFF10180819181A281B381F801D6
:10BA700080839183A283B38348CFEA8DEE0FEA8F50
:10BA8000F4E02F0E311C0C5F1F4F83E0898F8BCEAB
:10BA9000609113177091141790E08A3020F0895A42
:10BAA0009F4F0D9405A2C096FCCF2FB784FF1EC0F8
:10BAB000F894909105019260909305012FBF2FB7E4
:10BAC00085FF19C0F894909105019160909305014C
:10BAD0002FBF86FF15C0459A87FF14C0469A739AF8
:10BAE00085E08A95F1F7000073980895F894909195
:10BAF00005019D7FE1CFF894909105019E7FE6CFEF
:10BB00004598EACF4698EBCF0F931F93CF93DF93DF
:10BB1000C82FD62F8A0160FF15C05F9A8AE18A95E7
:10BB2000F1F700C08C2F0E94555DD1FD04C08C2F11
:10BB300082950E94555DC801DF91CF911F910F91B1
:10BB40000C94CCD05F98EACFCF92DF92EF92FF9225
:10BB5000CF93DF93EC016A017B010F94A5A36F3FA4
:10BB60007F4F8F4F9F4F59F4B701A601CE01DF9150
:10BB7000CF91FF90EF90DF90CF900D94F3A3DF91E2
:10BB8000CF91FF90EF90DF90CF9008957F928F92AA
:10BB90009F92AF92BF92CF92DF92EF92FF920F935C
:10BBA0001F93CF93DF93CDB7DEB760970FB6F894AE
:10BBB000DEBF0FBECDBF5C016B01742E81E08093B0
:10BBC00078021F930F931F922F938DE893E69F9314
:10BBD0008F930F945FA281E40E94F5550F900F9010
:10BBE0000F900F900F900F90882389F08091BB04E5
:10BBF0009091BC04FC012181283709F056C040E136
:10BC000050E070E060E002960F94289F5B0183E4AF
:10BC10000E94F555882309F44DC00E945D564B01E2
:10BC20007501CA14DB0408F47601C4018E0D9F1D52
:10BC3000C816D90618F08E159F0518F446018E18FF
:10BC40009F0888E50E94F555882309F471C020916A
:10BC5000BB043091BC042F5F3F4FCE0101965C01C5
:10BC6000DC01D12CC12CF90180812F5F3F4F88234B
:10BC7000B9F190E1C916D10499F18032A1F38A306B
:10BC800079F190ED980F9A30C8F48295807F9F01EA
:10BC90002E5F3F4F918140ED490F4A30B8F4842B1D
:10BCA0008D93EFEFCE1ADE0ADECF0E94855A0F94F5
:10BCB00036A6ACCF88248A94982CB2CF9FE9980FEF
:10BCC000963058F48295807F8057E1CF4FE9490F35
:10BCD000463018F49755892BE3CFD194C194D108FD
:10BCE000912C812CC814D90491F0F50161915F0168
:10BCF000C4018E0D9F1DF1E07F1631F0FC016083C1
:10BD0000FFEF8F1A9F0AEECF0F94E5A3F9CFFF92B2
:10BD1000EF921F930F939F928F9283E693E69F93E8
:10BD20008F930F945FA20FB6F894DEBF0FBECDBF06
:10BD3000472DB401C70160960FB6F894DEBF0FBE61
:10BD4000CDBFDF91CF911F910F91FF90EF90DF90CA
:10BD5000CF90BF90AF909F908F907F900D948F78F1
:10BD6000682F70E090E080E00F94299E20E030E0A2
:10BD700048E052E40F946A9E20E030E040E85FE340
:10BD80000F94C5A4089582E00F949C1860936912E3
:10BD900070936A1280936B1290936C1289E692E111
:10BDA0000D94953A4F925F926F927F928F929F92ED
:10BDB000AF92BF92CF92DF92EF92FF920F931F93B9
:10BDC000CF93DF9301E612E1CAE9D4E028813981FB
:10BDD0004A815B81F80160817181828193810F9436
:10BDE000C4A44B015C012C813D814E815F81F8012F
:10BDF00064817581868197810F94C4A46B017C0155
:10BE0000CAE8D4E0288139814A815B81C501B40147
:10BE10000F946A9E2B013C012C813D814E815F81F4
:10BE2000C701B6010F946A9E9B01AC01C301B20128
:10BE30000F94C5A4F801608371838283938328855E
:10BE400039854A855B85C501B4010F946A9E4B0113
:10BE50005C012C853D854E855F85C701B6010F9439
:10BE60006A9E9B01AC01C501B4010F94C5A4F80101
:10BE70006483758386839783DF91CF911F910F91A0
:10BE8000FF90EF90DF90CF90BF90AF909F908F90FA
:10BE90007F906F905F904F9008954F925F926F9256
:10BEA0007F928F929F92AF92BF92CF92DF92EF924A
:10BEB000FF920F931F93CF93DF9300D000D01F9278
:10BEC0001F92CDB7DEB7DC01CD90DD90ED90FC90F8
:10BED0001397C0926F03D0927003E0927103F092B7
:10BEE000720314960D911D912D913C911797098322
:10BEF0001A832B833C83009377031093780320935A
:10BF0000790330937A03DB010D911D912D913C91C2
:10BF100013970D831E832F83388700937303109329
:10BF20007403209375033093760314964D905D90BF
:10BF30006D907C90179740927B0350927C036092A7
:10BF40007D0370927E03FA01608171818281938109
:10BF500060939A0470939B0480939C0490939D0437
:10BF600084809580A680B78080929E0490929F04E2
:10BF7000A092A004B092A10420E030E0A9010F94A7
:10BF8000BAA58111AAC020E030E0A901C501B40121
:10BF90000F94BAA58111A1C01092A20420E030E054
:10BFA00040E85FE3C701B6010F94BAA5811121C033
:10BFB00020E030E0A9016D817E818F8198850F940A
:10BFC000BAA5811116C020E030E0A90169817A810B
:10BFD0008B819C810F94BAA581110BC020E030E0C9
:10BFE00040E85FE3C301B2010F94BAA5882309F4C6
:10BFF00078C08091A20482608093A204A301920180
:10C00000C701B6010F946A9E4B015C012D813E81F0
:10C010004F81588569817A818B819C810F946A9EBA
:10C020009B01AC01C501B4010F94C4A44B015C0198
:10C03000AC019B01C301B2010F94C4A560938A04B3
:10C0400070938B0480938C0490938D046D817E811A
:10C050008F8198859058A50194010F94C4A5609391
:10C060008E0470938F04809390049093910469815F
:10C070007A818B819C819058A50194010F94C4A56D
:10C080006093920470939304809394049093950426
:10C09000A5019401C701B6010F94C4A5609396044D
:10C0A00070939704809398049093990428960FB600
:10C0B000F894DEBF0FBECDBFDF91CF911F910F91DE
:10C0C000FF90EF90DF90CF90BF90AF909F908F90B8
:10C0D0007F906F905F904F90089581E08093A204CD
:10C0E0005DCF80E090E0A0E8BFE380938A04909366
:10C0F0008B04A0938C04B0938D0410928E04109244
:10C100008F04109290041092910410929204109255
:10C110009304109294041092950480939604909343
:10C120009704A0939804B0939904C0CF4F925F9264
:10C130006F927F928F929F92AF92BF92CF92DF9237
:10C14000EF92FF921F93CF93DF93CDB7DEB7A897FF
:10C150000FB6F894DEBF0FBECDBF48E050E06DEDE6
:10C160007FE0CE0101960F948DA348E050E065ED8D
:10C170007FE0CE0109960F948DA348E050E065EE74
:10C180007FE0CE0141960F948DA389899A89AB896E
:10C19000BC8989A39AA3ABA3BCA38F3F9F4FAF4F8A
:10C1A000BF4F09F4B1C08D899E89AF89B88D8DA329
:10C1B0009EA3AFA3B8A78F3F9F4FAF4FBF4F09F4C8
:10C1C000A3C089809A80AB80BC808FEF88169806C8
:10C1D000A806B80609F498C08D819E81AF81B88504
:10C1E000898F9A8FAB8FBC8F8F3F9F4FAF4FBF4FC1
:10C1F00009F48AC0C984DA84EB84FC848FEFC81602
:10C20000D806E806F80609F47FC08D859E85AF85BF
:10C21000B8898D8F9E8FAF8FB8A38F3F9F4FAF4F41
:10C22000BF4F09F471C0298D3A8D4B8D5C8DC501CE
:10C23000B4010F9461A72B013C0126E636E646E6E1
:10C240005FE30F94BAA511E087FD0BC02DEC3CEC29
:10C250004CE85FE3C301B2010F944EA718160CF02F
:10C2600010E02D8D3E8D4F8D58A1C701B6010F9462
:10C2700061A72B013C0126E636E646E65FE30F9414
:10C28000BAA587FD7FC02DEC3CEC4CE85FE3C30111
:10C29000B2010F944EA718160CF474C02DA13EA144
:10C2A0004FA158A569A17AA18BA19CA10F9461A768
:10C2B00020E030E040E751E40F944EA718160CF44C
:10C2C00011E0A5019401C701B6010F946A9E6B01AC
:10C2D0007C012D8D3E8D4F8D58A1698D7A8D8B8D72
:10C2E0009C8D0F946A9E9B01AC01C701B6010F940F
:10C2F000C5A49F772DEC3CEC4CEC5DE30F944EA76E
:10C30000181614F01123F1F00E941E5580E090E001
:10C31000A0E8BFE389839A83AB83BC831D821E821E
:10C320001F82188619861A861B861C868D879E8713
:10C33000AF87B88B198A1A8A1B8A1C8A1D8A1E8AA3
:10C340001F8A188EAE014F5E5F4FBE01675F7F4F41
:10C35000CE0101960E944D5FA8960FB6F894DEBFFD
:10C360000FBECDBFDF91CF911F91FF90EF90DF9077
:10C37000CF90BF90AF909F908F907F906F905F9085
:10C380004F90089511E08ACFCF93DF93CDB7DEB7FA
:10C3900068970FB6F894DEBF0FBECDBF80E090E087
:10C3A000A0E8BFE389839A83AB83BC831D821E828E
:10C3B0001F82188619861A861B861C868D879E8783
:10C3C000AF87B88B198A1A8A1B8A1C8A1D8A1E8A13
:10C3D0001F8A188EAE014F5E5F4FBE01675F7F4FB1
:10C3E000CE0101960E944D5F68960FB6F894DEBFAD
:10C3F0000FBECDBFDF91CF9108958091A204882315
:10C40000D1F00E94C4610F94B01880E00F949C1882
:10C41000609361127093621280936312909364121E
:10C4200081E00F949C18609365127093661280935C
:10C43000671290936812089580916304909162044A
:10C4400089130BC090916104992339F020911E0645
:10C4500030911F068217130639F081E09091C403D2
:10C46000911103C080E0089581E008952091630454
:10C4700080911E0690911F062817190611F080E280
:10C4800008958EE3089582E08093590280916304B9
:10C490008F5F8093630484E0809360041092620451
:10C4A00010926104089580916004843038F5809181
:10C4B000630490E020911E0630911F06281739076B
:10C4C00044F0019790931F0680931E0687E00F9417
:10C4D000622380911E062091920330E02D5F3F4F32
:10C4E0008217130659F054F09DEF980F9093920322
:10C4F0008450809362048FEF809360040895E6E98E
:10C50000F3E080E2DF011D928A95E9F70895CF9369
:10C510003FB7F894E0910204F0910304E817F9079B
:10C52000C9F0C42F909303048093020470931F06F4
:10C5300060931E061092920382E0809359023FBFDF
:10C54000222319F080E00F946223CC2321F0CF91B5
:10C550000C947F623FBFCF910895DC01262F90910C
:10C56000DF039730D8F4492F50E0FA01EE0FFF1F98
:10C57000E40FF51FE95AFC4F409102045091030467
:10C580005183408380911E069F5F9093DF038283D7
:10C5900041E070E060E0CD010C9487620895982F2F
:10C5A0008091DF039817A8F4891B8093DF0390E044
:10C5B000FC01EE0FFF1FE80FF91FE95AFC4F6281E3
:10C5C000062E000C770B20E041E0808191810C94D5
:10C5D000876280E0EACF81E00C94CF621F920F92D5
:10C5E0000FB60F9211240BB60F922F933F934F93D8
:10C5F0006F937F938F939F93EF93FF938091C800E6
:10C6000084FF12C08091CE00FF91EF919F918F9196
:10C610007F916F914F913F912F910F900BBE0F9093
:10C620000FBE0F901F9018954091CE0080911C0670
:10C63000813051F72091420530914305C90101969F
:10C640008F77992760914405709145058617970764
:10C65000D9F22E533B4FF9014083909343058093C9
:10C660004205D2CF1F920F920FB60F9211240BB634
:10C670000F922F933F934F936F937F938F939F933B
:10C68000EF93FF938091C00084FF12C08091C60099
:10C69000FF91EF919F918F917F916F914F913F917A
:10C6A0002F910F900BBE0F900FBE0F901F901895FB
:10C6B0004091C60080911C068111EACF209142056D
:10C6C00030914305C90101968F7799276091440500
:10C6D0007091450586179707D9F22E533B4FF90104
:10C6E00040839093430580934205D2CF80E1E1E6F9
:10C6F000F2E1A0E9B2E001900D928A95E1F7809114
:10C700008E0290918F029093601280935F128091BD
:10C710005D1290915E1290935C1280935B128091F7
:10C720005912809358128091571283FB882780F901
:10C730008093561280915512809354120895CF938E
:10C74000DF9387E696E10E947B7985EA94E1892B65
:10C7500051F0C7E7D5E1A397CE010E947B7984E130
:10C76000C53AD807C1F782E894E10E947B798DE54C
:10C7700094E1DF91CF910C947B79CF93DF93C1E665
:10C78000D2E120E030E048EC51E46C857D858E8577
:10C790009F850F94C5A46C877D878E879F8763E3F1
:10C7A00073E383E590E4DF91CF910D940A4A60E052
:10C7B00085EA9FE00F94C1A360E08FE79CE00F94AF
:10C7C000C1A380E090E0A0E8BFEB80937E0290934D
:10C7D0007F02A0938002B093810282E0809379026D
:10C7E00010927312089580915B1290915C122091C7
:10C7F0005D1230915E122817390771F090935E1226
:10C8000080935D1281E08093CB030F94560B0F94BD
:10C81000427482E08093CB03089580917312882341
:10C8200041F080918E0290918F02909360128093DC
:10C830005F120895CF92DF92EF92FF92C090FF0DAA
:10C84000D090000EE090010EF090020E8091FE0D4F
:10C85000882309F44EC020E030E0A901C701B601E9
:10C860000F944EA718160CF044C02BED3FE049E49E
:10C8700050E4C701B6010F946A9EA70196010F9478
:10C880006A9E20E030E040E85EE30F946A9E9B01E0
:10C89000AC0160E070E080E89FE30F94C4A56B01F9
:10C8A0007C01609175027091760264367105A1F089
:10C8B000072E000C880B990B0F942B9E2AE037ED66
:10C8C00043E25CE30F946A9E9B01AC01C701B60191
:10C8D0000F946A9E6B017C01C0921002D0921102EB
:10C8E000E0921202F0921302FF90EF90DF90CF904F
:10C8F0000895C12CD12C80E8E82E8FE3F82ED1CFFB
:10C900008F929F92AF92BF92CF92DF92EF92FF925F
:10C9100081EF9FE00F94A96C6B017C018DEE9FE08D
:10C920000F94A96C4B015C010F9422152CE330E0AD
:10C9300040E050E00F9410A4BA01A901480D591D20
:10C940006A1D7B1D8DEE9FE00F94D3A360911706A7
:10C95000709118068091190690911A0628EE33E01E
:10C9600040E050E00F9410A4BA01A9014C0D5D1DE8
:10C970006E1D7F1D81EF9FE00F94D3A30F94BF1610
:10C9800010921706109218061092190610921A06A5
:10C9900080910113813081F4609105137091061329
:10C9A00090E080E00F94916C1092061310920513A2
:10C9B0001092081310920713FF90EF90DF90CF9022
:10C9C000BF90AF909F908F900895809155121F92C5
:10C9D0008F9380913E031F928F93E7EBF3E04281A8
:10C9E00053812CE3249FC001259F900D11249F9318
:10C9F0008F9340815181249FC001259F900D112468
:10CA00009F938F9384E294E69F938F930F945FA2FA
:10CA10008DB79EB70A960FB6F8949EBF0FBE8DBF16
:10CA2000089588E493E00D947F0D20E030E040E726
:10CA300052E40F94C4A508951092770240913903EF
:10CA400050913A0360913B0370913C0340937A020A
:10CA500050937B0260937C0270937D0290938F02CF
:10CA600080938E0288E493E00D947F0D1F93CF9303
:10CA7000DF93182F80917A0290917B02A0917C0223
:10CA8000B0917D028093390390933A03A0933B03C6
:10CA9000B0933C03C0918E02D0918F0284E690E067
:10CAA00090938F0280938E0288E493E00F947F0D21
:10CAB00010937702CE01DF91CF911F910895CF920D
:10CAC000DF92EF92FF920F931F93CF93DF9390E04B
:10CAD000EC01CC0FDD1FCC0FDD1FFE01E156F94844
:10CAE0002591359145915491FE01E154F24FC0805A
:10CAF000D180E280F3808E010F591D4EC701B6012F
:10CB00000F94C5A4F8016083718382839383FE012F
:10CB1000ED56F94825913591459154918E010C5D62
:10CB20001D4FC701B6010F94C5A4F801608371833E
:10CB300082839383FE01E957F94825913591459108
:10CB40005491C85EDD4FC701B6010F94C5A4688338
:10CB500079838A839B83DF91CF911F910F91FF90FF
:10CB6000EF90DF90CF90089540E050E0BA018DEE55
:10CB70009FE00F94D3A340E050E0BA0181EF9FE023
:10CB80000F94D3A30E94685670E060E085E09FE0B8
:10CB90000F94DFA370E060E083E09FE00F94DFA3D9
:10CBA00070E060E081E09FE00F94DFA370E060E060
:10CBB0008FEF9EE00F94DFA370E060E083ED9EE0D6
:10CBC0000F94DFA370E060E080ED9EE00F94DFA3A0
:10CBD00040E050E0BA0188EA9CE00D94D3A3F894B9
:10CBE00088E19FE00FB6F894A895809360000FBE8F
:10CBF00090936000FFCF85EA9FE00F949DA391E0A2
:10CC0000811101C090E0892F08958091CD03811199
:10CC100006C081E090918B03923009F080E0089586
:10CC20008091D71381110AC080914212811106C0F0
:10CC300081E090918B03913009F080E00895CF93CB
:10CC4000DF93C0917112C1111FC0809172128111C6
:10CC50001CC00E940566811118C0D0915E0DD430B1
:10CC600061F480915D1290915E12892B91F4809114
:10CC7000591290915A12892B61F40E941066C82FA4
:10CC8000811103C0C1E0D111C0E08C2FDF91CF91A1
:10CC90000895C1E0FACF0E941F66882389F020E042
:10CCA00030E040E050E46091691270916A12809126
:10CCB0006B1290916C120F94BAA5881F8827881F59
:10CCC00008950E941066811118C00E9405668111A6
:10CCD00014C080917312811110C080915E0D81117A
:10CCE0000BC080910213811107C0809171128111D4
:10CCF00004C080917212089581E0089580E1E1E618
:10CD0000F2E1A9E2B6E001900D928A95E1F708956B
:10CD10004F925F926F927F928F929F92AF92BF924B
:10CD2000CF92DF92EF92FF920F931F93CF93DF93F7
:10CD300000D000D01F921F92CDB7DEB720917312A2
:10CD4000222309F473C12091CE03223009F46EC16D
:10CD50002091CE03213011F41092CE032B013C011F
:10CD600010925512109158126091BC037091BD033E
:10CD70008091BE039091BF030F943DA6611731F0DF
:10CD8000812F90E090935A12809359120E94F3637E
:10CD9000809154128093551290915712809156129F
:10CDA000819589278870892780935712A301920162
:10CDB00060919C0270919D0280919E0290919F02D1
:10CDC0000F94C4A46D837E838F839887CE010596CC
:10CDD0000F94623A1092400220E030E040E85FEBAE
:10CDE00060919002709191028091920290919302D1
:10CDF0000F94BAA5811120C08091611290916212A6
:10CE0000A0916312B091641280939002909391026A
:10CE1000A0939202B0939302809165129091661252
:10CE2000A0916712B091681280939402909395023A
:10CE3000A0939602B0939702A301920160919C0285
:10CE400070919D0280919E0290919F020F94C4A4C4
:10CE500069837A838B839C83E0906912F0906A12D5
:10CE600000916B1210916C122091940230919502F6
:10CE700040919602509197026091900270919102B8
:10CE800080919202909193021F921F921F921F9283
:10CE9000E2E68E2EE7E29E2EE6E7AE2EE2E4BE2E1E
:10CEA000FE0131966F010F94BC3AA301920160918B
:10CEB0009C0270919D0280919E0290919F020F941E
:10CEC000C4A469837A838B839C83E0909802F0905A
:10CED000990200919A0210919B0220919402309144
:10CEE0009502409196025091970260919002709144
:10CEF000910280919202909193021F921F921F9231
:10CF00001F920F94BC3AE0909802F0909902009121
:10CF10009A0210919B0220919402309195024091C7
:10CF200096025091970260919002709191028091C7
:10CF30009202909193021F921F921F921F92812C36
:10CF4000912CF8EEAF2EF2E4BF2EACE9CA2EA2E08F
:10CF5000DA2E0F94BC3A0F94B01811E010934002EF
:10CF600060914F127091501290E080E00F94299ED2
:10CF700060937A0270937B0280937C0290937D028F
:10CF800080915F129091601290938F0280938E0235
:10CF900080E1E0E9F2E0A1E6B2E101900D928A952C
:10CFA000E1F70E947E66809179020FB6F894DEBFA9
:10CFB0000FBECDBF811151C06091451270914612D4
:10CFC00080914712909148126093EB167093EC1683
:10CFD0008093ED169093EE160F94E86780914512BA
:10CFE00090914612A0914712B09148128093491235
:10CFF00090934A12A0934B12B0934C121093D713F4
:10D0000060E085EA9FE00F94C1A360E08FE79CE0B9
:10D010000F94C1A386EE9BE60E9485DC82E080939C
:10D0200079021092731281E08093420D28960FB618
:10D03000F894DEBF0FBECDBFDF91CF911F910F914E
:10D04000FF90EF90DF90CF90BF90AF909F908F9028
:10D050007F906F905F904F900895813089F6809116
:10D06000451290914612A0914712B09148128093B8
:10D070003E1290933F12A0934012B093411210922F
:10D080004810109247100E94AC55BACF3F924F9271
:10D090005F926F927F928F929F92AF92BF92CF9248
:10D0A000DF92EF92FF920F931F93CF93DF93309015
:10D0B000A204332009F480C08B01EC0131FE54C07E
:10D0C00088809980AA80BB80FB01C080D180E280EB
:10D0D000F380209177033091780340917903509148
:10D0E0007A03C501B4010F946A9E2B013C01209183
:10D0F0007B0330917C0340917D0350917E03C701F7
:10D10000B6010F946A9E9B01AC01C301B2010F945A
:10D11000C5A42B013C0120916F0330917003409115
:10D12000710350917203C501B4010F946A9E4B01C3
:10D130005C01209173033091740340917503509109
:10D140007603C701B6010F946A9E9B01AC01C5012D
:10D15000B4010F94C5A4688379838A839B83F80103
:10D16000408251826282738230FE26C020919A04EE
:10D1700030919B0440919C0450919D046881798179
:10D180008A819B810F94C5A4688379838A839B835A
:10D1900020919E0430919F044091A0045091A104DD
:10D1A000F80160817181828193810F94C5A4F80197
:10D1B0006083718382839383DF91CF911F910F915D
:10D1C000FF90EF90DF90CF90BF90AF909F908F90A7
:10D1D0007F906F905F904F903F9008952F923F9275
:10D1E0004F925F926F927F928F929F92AF92BF9277
:10D1F000CF92DF92EF92FF920F931F93CF93DF9323
:10D2000000D000D01F921F92CDB7DEB78C011B015A
:10D21000FC0180819181A281B38189839A83AB8350
:10D22000BC83FB0180819181A281B3818D839E8328
:10D23000AF83B887BE016B5F7F4FCE0101960E941E
:10D240004668C980DA80EB80FC8020E030E0A901EC
:10D25000C701B6010F94BAA587FF35C019821A829B
:10D260001B821C82FF24F3948D809E80AF80B88443
:10D2700020E030E040E850ECC501B4010F94BAA5BD
:10D2800087FF35C080E090E0A0E8B0EC8D839E83FE
:10D29000AF83B887CD80DE80EF80F88489809A8064
:10D2A000AB80BC807090A20471104CC0F8018082E9
:10D2B0009182A282B382F101C082D182E282F382A2
:10D2C000FF24F39425C020E030E04AE753E4C7018F
:10D2D000B6010F944EA7F12C181634F680E090E0BA
:10D2E000AAE7B3E489839A83AB83BC83BBCF20E0F6
:10D2F00030E042E553E4C501B4010F944EA718167F
:10D300002CF480E090E0A2E5B3E4C0CFF110C2CFEE
:10D310008F2D28960FB6F894DEBF0FBECDBFDF91DC
:10D32000CF911F910F91FF90EF90DF90CF90BF9022
:10D33000AF909F908F907F906F905F904F903F90B5
:10D340002F90089570FE1CC020919A0430919B0488
:10D3500040919C0450919D04C501B4010F94C4A454
:10D360004B015C0120919E0430919F044091A004E8
:10D370005091A104C701B6010F94C4A46B017C01B4
:10D3800071FE9ECF20918A0430918B0440918C04D1
:10D3900050918D04C501B4010F946A9E2B013C018C
:10D3A00020918E0430918F0440919004509191040B
:10D3B000C701B6010F946A9E9B01AC01C301B20183
:10D3C0000F94C5A4F80160837183828393832091B5
:10D3D0009204309193044091940450919504C501B6
:10D3E000B4010F946A9E4B015C0120919604309128
:10D3F00097044091980450919904C701B6010F9485
:10D400006A9E9B01AC01C501B4010F94C5A4F10152
:10D41000608371838283938353CFCF93DF930E9482
:10D420001165C1E6D2E180E090E0A0EAB0E488872F
:10D430009987AA87BB8765E575E585E591E40F9433
:10D44000BC4E8DEC9CECACE4BEE388839983AA834C
:10D45000BB8383E393E3A3E7B0EC8C839D83AE832C
:10D46000BF8365E672E1CE010E94EE6860E070E085
:10D4700086E193E40F94BC4E8AE999E9A9E1BEE301
:10D4800088879987AA87BB8765E575E585E591E477
:10D49000DF91CF910D94BC4ECF92DF92EF92FF922D
:10D4A000CF93DF93EC01BC016C5F7F4F0E94EE686D
:10D4B000C0902C02D0902D02E0902E02F0902F020E
:10D4C000A7019601688579858A859B850F94BAA501
:10D4D00087FF04C0C886D986EA86FB86C0902002F2
:10D4E000D0902102E0902202F0902302A701960141
:10D4F000688579858A859B850F944EA7181624F434
:10D50000C886D986EA86FB86DF91CF91FF90EF909F
:10D51000DF90CF9008952F923F924F925F926F923B
:10D520007F928F929F92AF92BF92CF92DF92EF92B3
:10D53000FF920F931F93CF93DF93CDB7DEB7A297E0
:10D540000FB6F894DEBF0FBECDBF1C0189E296E096
:10D550000E944C6A88E493E00F947F0D4090611222
:10D56000509062126090631270906412C09029060D
:10D57000D0902A06E0902B06F0902C06A701960189
:10D58000C301B2010F94BAA581113FC020912D06AD
:10D5900030912E0640912F06509130066091651211
:10D5A0007091661280916712909168120F94BAA5DB
:10D5B00081112BC020E030E040E752E460917A0214
:10D5C00070917B0280917C0290917D020F94C4A5A2
:10D5D0000F94D7490E94E854A2960FB6F894DEBF84
:10D5E0000FBECDBFDF91CF911F910F91FF90EF90B4
:10D5F000DF90CF90BF90AF909F908F907F906F9073
:10D600005F904F903F902F90089560918E0270919F
:10D610008F02072E000C880B990B0F942B9E2091E4
:10D620007A0230917B0240917C0250917D020F94EE
:10D630006A9E2EE333EC4EE259E30F946A9E6F83A9
:10D64000788789879A8780910913882309F40FC105
:10D65000A3019201C701B6010F94C4A42B013C01A0
:10D6600020916512309166124091671250916812B4
:10D6700060912D0670912E0680912F0690913006B4
:10D680000F94C4A46B877C878D879E87C301B201EA
:10D690009F772B853C854D855E855F770F94C5A46C
:10D6A0006B017C0120E030E0A9010F944EA7181611
:10D6B0000CF0DDC020E030E040EF51E4C701B601DE
:10D6C0000F94C4A50F94A3A50F943DA67E836D83EC
:10D6D0006230710508F4CBC02114310409F4C7C0CD
:10D6E0002091691230916A1240916B1250916C1224
:10D6F0006091310670913206809133069091340624
:10D700000F94C4A46F87788B898B9A8B20916D12AC
:10D7100030916E1240916F125091701260913506E7
:10D720007091360680913706909138060F94C4A404
:10D730006B8B7C8B8D8B9E8BAD81BE81CD01B0E0E0
:10D74000A0E08F8F98A3A9A3BAA32D813E812216B2
:10D75000330608F08CC0B10190E080E00F94299E60
:10D760006B017C016F8D78A189A19AA10F94299EEC
:10D770009B01AC01C701B6010F94C4A56B017C01EC
:10D78000AC019B016B897C898D899E890F946A9E6F
:10D790009B01AC0160916D1270916E1280916F12BD
:10D7A000909170120F94C5A469837A838B839C83B4
:10D7B000A70196016F85788989899A890F946A9E55
:10D7C0002091691230916A1240916B1250916C1243
:10D7D0000F94C5A46F8B788F898F9A8FA7019601BC
:10D7E0006B857C858D859E850F946A9E2091651240
:10D7F0003091661240916712509168120F94C5A43F
:10D800006B8F7C8F8D8F9E8FA7019601C301B20114
:10D810000F946A9E209161123091621240916312BE
:10D82000509164120F94C5A43F922F92A1E6B2E1E9
:10D83000BF93AF938F809884A984BA84DE01119638
:10D840006D01EF88F88C098D1A8D2B8D3C8D4D8DD7
:10D850005E8D0F94BC3A0F900F900F900F908091B7
:10D86000420D8111B7CEBFEF2B1A3B0A6ECFE0906D
:10D870003106F09032060091330610913406209163
:10D880002D0630912E0640912F0650913006609162
:10D89000290670912A0680912B0690912C061F92E2
:10D8A0001F92E1E6F2E1FF93EF938F809884A984C1
:10D8B000BA84E5E3CE2EE6E0DE2E0F94BC3A0F905C
:10D8C0000F900F900F9086CECF92DF92EF92FF9243
:10D8D000CF93C0906912D0906A12E0906B12F090D2
:10D8E0006C12A70196010F94C5A4609369127093FE
:10D8F0006A1280936B1290936C1283B190913B06E5
:10D90000911102C084FF26C081E692E10E944C6A18
:10D910006091830D7091840D8091850D9091860D9D
:10D920000F940A4A0F94B018A701960160916912EA
:10D9300070916A1280916B1290916C120F94C4A432
:10D940006B017C01C701B601CF91FF90EF90DF9092
:10D95000CF90089515980F94B01881E00F943D234F
:10D96000C82F65E575E585E591E40F940A4A0F94A3
:10D97000B01882E00F949C18A70196010F94C4A4DC
:10D980006B017C018C2F0F943D23DCCF8F929F92F3
:10D99000AF92BF92CF92DF92EF92FF924B015C0168
:10D9A000C0906912D0906A12E0906B12F0906C12E5
:10D9B000AC019B01C701B6010F944EA787FF11C0B0
:10D9C000A5019401C701B6010F94C4A49F77FF90ED
:10D9D000EF90DF90CF90BF90AF909F908F900C947E
:10D9E000646CFF90EF90DF90CF90BF90AF909F90CE
:10D9F0008F9008952F923F924F925F926F927F92F5
:10DA00008F929F92AF92BF92CF92DF92EF92FF924E
:10DA10000F931F93CF93DF9300D01F921F92CDB728
:10DA2000DEB7D82E2A013B01322EE982FA820B831F
:10DA30001C830F94B01881E080937112FC2CE32CAE
:10DA4000D31010C0ED2CDC100DC060E070E080EA57
:10DA500090E40E94C66CFF24F394EE24E394222405
:10DA6000239401C02D2C0E94FD61809109138D83A8
:10DA70001092091382E00F949C18609369127093BE
:10DA80006A1280936B1290936C12F1100F94AA5249
:10DA900081E00E9436658C010E947E6610927A02B7
:10DAA00010927B0210927C0210927D02222019F0CB
:10DAB00080E00F946B79EE2019F081E00F946B7980
:10DAC000DD20E9F04114510461047104C1F0C30187
:10DAD000B2010F942B9E9B01AC016091BF0D709120
:10DAE000C00D8091C10D9091C20D0F94C5A460939B
:10DAF00061127093621280936312909364123320C8
:10DB000001F189819A81AB81BC810097A105B105A2
:10DB1000C1F0BC01CD010F942B9E9B01AC01609123
:10DB2000C30D7091C40D8091C50D9091C60D0F94D9
:10DB3000C5A46093651270936612809367129093E8
:10DB40006812FF2009F499C060E070E080EA90E478
:10DB50000E94C66C80913906811102C00F946B79C6
:10DB600080913A06811103C081E00F946B790E9485
:10DB70009660E4E0FCE985919591A591B491E0E08F
:10DB8000FCE9459155916591749140932906509314
:10DB90002A0660932B0670932C0680932D06909393
:10DBA0002E06A0932F06B09330066DE276E089E250
:10DBB00096E00E9446680E94C46120E030E040E8A0
:10DBC00050EC60912D0670912E0680912F06909159
:10DBD00030060F94BAA587FF0CC080E090E0A0E863
:10DBE000B0EC80932D0690932E06A0932F06B09351
:10DBF000300680E090E0A6E1B3E480937A0290934F
:10DC00007B02A0937C02B0937D02109277020F9466
:10DC1000CA4860917A0270917B0280917C02909157
:10DC20007D020F94D7490F94B018809129069091E6
:10DC30002A06A0912B06B0912C0680936112909336
:10DC40006212A0936312B093641280912D0690919A
:10DC50002E06A0912F06B091300680936512909306
:10DC60006612A0936712B093681281E080937702E6
:10DC70000F94592382E00F946B79CC20E9F0811442
:10DC80009104A104B104C1F0C501B4010F942B9E0D
:10DC90009B01AC016091C70D7091C80D8091C90DB9
:10DCA0009091CA0D0F94C5A46093691270936A1283
:10DCB00080936B1290936C120F94CA48C8010E9413
:10DCC0001C650F9459230E9496600E94D25ED11069
:10DCD00007C0311005C08B8D811102C0CC2039F1F5
:10DCE000F11025C09D81992311F181E080930913E2
:10DCF0000F949C186B017C0180E00F949C18A70185
:10DD000096010F9435919B01AC016091691270915D
:10DD10006A1280916B1290916C120F94C4A460935C
:10DD2000691270936A1280936B1290936C1284E163
:10DD30000F9402300F94B018109271120F900F9040
:10DD40000F900F900F90DF91CF911F910F91FF9047
:10DD5000EF90DF90CF90BF90AF909F908F907F908B
:10DD60006F905F904F903F902F900895E1E3F3E024
:10DD70009FE781918F3731F0DF01119787FF07C04F
:10DD80008F778C9383E0E933F80799F708959C9394
:10DD9000F9CF90915902981710F48093590280910D
:10DDA0005A02882339F0E0910404F0910504309779
:10DDB00009F019940895CF93DF93CDB7DEB7AE0184
:10DDC0004A5F5F4FFA0161917191AF0182EF93E079
:10DDD0000F94E4A2DF91CF91089562EF73E00D9468
:10DDE00035A262EF73E0082E000C990B0D9405A28A
:10DDF000CF93C82FC15020F080E20E94F16EFACF7D
:10DE0000CF9108950F931F93CF93DF93EB01142FBE
:10DE1000052F0E94F16ECE010E94ED6E8AE30E94F2
:10DE2000F16ECE010F945BA19EE0981B892F0E949A
:10DE3000F86E0F931F9383E691E89F938F930E9450
:10DE4000DB6E0F900F900F900F90DF91CF911F918D
:10DE50000F910895CF93C82F862F643008F083E088
:10DE6000809330030E94F2548C0F80932F0344E67A
:10DE700050E060E08068CF910C94845D7F928F9237
:10DE80009F92AF92BF92CF92DF92EF92FF920F9349
:10DE90001F93CF93DF93E091630450916204E513E5
:10DEA00073C0FB01483009F06CC0C081D0E049016B
:10DEB000742E6B015C0180915902882359F06091A6
:10DEC000600480E00E942A6F0E943662AE01B501B4
:10DED0000E94026F80916104882309F455C09091DB
:10DEE000630420911E0630911F069217130609F055
:10DEF0004BC08091DF038730D8F4282F30E0F90140
:10DF0000EE0FFF1FE20FF31FE95AFC4F20910204AE
:10DF100030910304318320838F5F8093DF039283EA
:10DF200020E040E070E060E082E593E70E948762D5
:10DF3000B0929703A0929603D0929A03C09299034D
:10DF400070929803D0939C03C0939B0390929E037E
:10DF500080929D031093A00300939F03F092A2036D
:10DF6000E092A103DF91CF911F910F91FF90EF906D
:10DF7000DF90CF90BF90AF909F908F907F900C9448
:10DF80004362C081D18193CF809163048F5F80937E
:10DF90006304DF91CF911F910F91FF90EF90DF907D
:10DFA000CF90BF90AF909F908F907F900895CF9328
:10DFB000DF93EA010E942A6F62EF73E0CE01DF91E6
:10DFC000CF910D9435A2CF93C42F0E942A6F62EF98
:10DFD00073E08C2FCC0F990BCF910D9405A260E0CC
:10DFE00080E00E942A6F10922F03089540E456E0CB
:10DFF00060E081E00E94845D1092300310922F0354
:10E0000048E050E06FE770E081E393E00D94CFA922
:10E0100090915A02981709F180935A028823E9F0E7
:10E0200010921F0610921E061092A40583EE93E034
:10E030000F947F0D0F94560B61507109810991095E
:10E040006093C5037093C6038093C7039093C8037E
:10E050000E94F66F82E00C94C96E0895CF93C82F8A
:10E060001092300310922F0348E050E06FE770E009
:10E0700081E393E00F94CFA944E951E162E080E3AA
:10E080000E94845D46E950E062E080E30E94845D86
:10E0900046E950E062E080E30E94845D46E950E09A
:10E0A00062E080E20E94845D8091000444E650E0DA
:10E0B00060E080620E94845D84E080932E0344E6E9
:10E0C00050E060E08CE00E94845DC1110E94F66F18
:10E0D00044E650E060E086E0CF910C94845D81E0FE
:10E0E0000C942E70CF92DF92FF920F931F93CF93D9
:10E0F000DF9300D000D01F921F92CDB7DEB78A30D9
:10E10000D9F480913003843018F08FEF809330037E
:10E11000609130036F5F80E00E942A6F28960FB6EF
:10E12000F894DEBF0FBECDBFDF91CF911F910F914D
:10E13000FF90DF90CF90089590E8980F44E650E06C
:10E1400061E09A3408F5482F4058550B9A0196E043
:10E15000929FA001939F500D1124FA01EA56FB48AB
:10E16000F490E1E3F3E030E020E09FEF6191782F5D
:10E1700076277F7789F4F901EF5CFC4F8083F22EDC
:10E1800044E650E061E08F2D0E94845D80912F0372
:10E190008F5F80932F03C2CF6F3709F03CC0F90126
:10E1A000EF5CFC4F8083922FF92EFA01EF56FB486B
:10E1B0008E010F5F1F4FD801959188E0182E10FE39
:10E1C00005900294802D9795881F8D931A94B9F726
:10E1D000BF2DE8E0BE02C001112444E650E060E03B
:10E1E00080640E94845D6E01F9E0CF0ED11C44E68C
:10E1F00050E061E0D8018D918D010E94845DC016D0
:10E20000D106A9F780912F0344E650E060E08068D2
:10E210000E94845DB5CF67FF922F2F5F3F4F28305C
:10E22000310509F0A3CF9F3F09F0BECFA9CFCF930F
:10E2300024E1AC01249FC001259F900D1124609121
:10E240006D0370916E030F9466A4C62F653108F0BC
:10E25000C4E180916C038C1748F48FEF0E947270B8
:10E2600080916C038F5F80936C03F3CFCF910895FF
:10E2700081E090E090936E0380936D030E9417718C
:10E280006CE271E080E090E00D94230B8F929F92FE
:10E29000AF92BF92EF92FF920F931F93CF93DF93B2
:10E2A000CDB7DEB7A0970FB6F894DEBF0FBECDBFD7
:10E2B000611571058105910599F480E3A0960FB66B
:10E2C000F894DEBF0FBECDBFDF91CF911F910F91AC
:10E2D000FF90EF90BF90AF909F908F900C947270D2
:10E2E00000E0842E912CB12CA12C9E012F5F3F4F7A
:10E2F0007901A50194010F9410A4F701E00FF11D1D
:10E300006083B901CA010F5F61157105810591052F
:10E3100081F70E0D1F2D111DE016F10659F0F801C1
:10E3200082918F018A3020F4805D0E947270F4CF58
:10E33000895CFBCFA0960FB6F894DEBF0FBECDBFB1
:10E34000DF91CF911F910F91FF90EF90BF90AF9011
:10E350009F908F900895CF92DF92EF92FF926B0182
:10E360007C01F7FE0BC08DE20E947270F094E09485
:10E37000D094C094C11CD11CE11CF11C4AE0C7011F
:10E38000B601FF90EF90DF90CF900C9446710F9301
:10E390001F93CF938C01C62FCC2359F0F801249101
:10E3A000222339F00F5F1F4F84910E947270C15079
:10E3B000F3CF8C2F0E94F86E8C2FCF911F910F916D
:10E3C00008950F931F93CF93DF938C01EB010E946D
:10E3D000F66F10926C0310936E0300936D0361E06F
:10E3E00080E00E942A6F64E1CE010E94C77162E062
:10E3F00080E0DF91CF911F910F910C942A6FEF92E3
:10E40000FF920F931F93CF93DF937091630430912A
:10E41000620473133FC0122FEA01062F7C01809122
:10E4200059028823D1F00E943662482F609160041F
:10E4300080E00E94E36F61E1C7010E94C771402F35
:10E440006091600493E1981B892F0E94E36F40E282
:10E450006091600483E10E94E36F809161048823EE
:10E46000C9F02091630480911E0690911F06281721
:10E47000190681F410925A02812FFE01199581E04C
:10E4800080935A02DF91CF911F910F91FF90EF90EF
:10E490000C944362809163048F5F80936304DF91E7
:10E4A000CF911F910F91FF90EF9008950F931F93BD
:10E4B000CF93C82F8B010E943662482F6091600471
:10E4C00080E00E94E36F62E1C8010E94C7718C2F57
:10E4D000CF911F910F910C94F16ECF93DF933091F8
:10E4E000630420916204321321C0EB01BC018091CE
:10E4F0005902882319F080E20E94567280916104CB
:10E500008823A1F02091630480911E0690911F063C
:10E510002817190659F410925A02FE01199581E044
:10E5200080935A02DF91CF910C94436280916304EF
:10E530008F5F80936304DF91CF91089530916304DE
:10E5400020916204321319C0BC01809159028823C2
:10E5500019F083E80E94567280916104882369F063
:10E560002091630480911E0690911F0628171906BA
:10E5700021F40E94EB620C944362809163048F5FEC
:10E58000809363040895CF93DF93309163042091C7
:10E59000620432131EC0EB01BC0180915902882332
:10E5A00019F08EE70E94567280916104882389F0E9
:10E5B0002091630480911E0690911F06281719066A
:10E5C00041F460E0CE010E94AD62DF91CF910C94E6
:10E5D0004362809163048F5F80936304DF91CF91E6
:10E5E00008953091630420916204321319C0BC0174
:10E5F00080915902882319F080E20E94567280911E
:10E600006104882369F02091630480911E06909133
:10E610001F062817190621F40E94436281E008951D
:10E62000809163048F5F8093630480E008950F936B
:10E630001F93CF938C01C62FCC2349F0F801819111
:10E640008F01882321F00E947270C150F5CF8C2F6A
:10E650000E94F86E8C2FCF911F910F910895CF9348
:10E66000DF93EC018991882319F00E947270FACF30
:10E67000DF91CF9108950E94727090E080E008953C
:10E68000109295031092A7050895CF93809195035A
:10E69000C1E0811104C0C0E08C2FCF9108950E9489
:10E6A0004073FACF80915902882309F452C0209117
:10E6B000A1033091A20380919D0390919E032115A7
:10E6C0003105D9F040911E0650911F0641155105A4
:10E6D000A1F07CF040919B0350919C03481759078F
:10E6E00041F430939C0320939B0310921F061092D9
:10E6F0001E061092A2031092A10320919B03309159
:10E700009C0340911E0650911F06240F351F109246
:10E710001F0610921E062817390744F080919F03A8
:10E720009091A003281739070CF4C90190939C031A
:10E7300080939B0361E080E00E942A6F40919B03DD
:10E7400050919C03609196037091970380E20E9420
:10E75000026F0E944573882341F1E0919903F09183
:10E760009A0380919B0390919C032091980380834E
:10E770002830C9F48091DF038823B9F08150809359
:10E78000DF0390E0FC01EE0FFF1FE80FF91FE95ACD
:10E79000FC4F6281062E000C770B20E040E0808168
:10E7A00091810C9487629183E5CF08950E9445730F
:10E7B00081110C94EB62089580911E0690911F06C2
:10E7C00097FF07C010921F0610921E0687E00F9455
:10E7D000622380911E0690911F06209192032817B4
:10E7E000190619F014F0809392038091920380939C
:10E7F00062040E9445738093610408958EEF9FE048
:10E800000F949DA38E3F39F091E020912D032813A2
:10E8100090E0892F089580E0089510922D036EEF07
:10E820008EEF9FE00D94C1A3853728E6920709F487
:10E8300059C0F8F48E3625E6920709F459C050F411
:10E84000833723E69207B1F185369446B1F182EA27
:10E8500093E60895823726E6920791F1823728E6FB
:10E86000920709F442C08337954689F789EF93E60A
:10E8700008958C3620E7920731F170F48C362EE63D
:10E88000920721F18F362EE6920731F184379946AF
:10E89000F1F687EE93E608958B3623E79207F9F0B9
:10E8A000863723E79207A9F08F36924781F685EAEB
:10E8B00093E6089589E094E6089581E094E608954A
:10E8C00080EF93E6089580EE93E6089585ED93E654
:10E8D00008958DEC93E6089587EC93E608958CEB0C
:10E8E00093E6089585EB93E608958CEA93E6089500
:10E8F00081E194E60895EDE8F4E785919591A5917D
:10E90000B4918F3F9F4FAF4FBF4FB1F020E031E048
:10E9100081E0F9014591559165917491453A5A45C7
:10E92000644B7B4409F00895F90134964591549164
:10E93000240F351F8F5FEDCF81E008950F931F9354
:10E94000811113C010922C0310922B0310922D03EF
:10E9500090912D0398135CC0682F8EEF9FE00F9469
:10E96000C1A381E01F910F910895813089F7E0E004
:10E97000F1E04591559165917491453A5A45644B42
:10E980007B4431F7E4E0F1E0A591B491E8E0F1E0F7
:10E990006591749150E040E030E020E0A417B507A5
:10E9A00029F5261B370B32272327322762177307D7
:10E9B00009F0CECFECE0F1E005911591259134916D
:10E9C000EDE8F4E7459155916591749104171507A9
:10E9D0002607370709F0BCCF20E031E030932C0345
:10E9E00020932B0391E090932D03B2CFFA01E050D6
:10E9F000FF4FE491F0E098E040FD90E002C0EE0FA0
:10EA0000FF1F9A95E2F72E0F3F1F4F5F5F4FC6CF54
:10EA100080E0A8CF20912D03211104C0FC01329683
:10EA2000CF01089540912B0350912C0341155105BE
:10EA3000A9F3FC01259134912F3F320779F3F901B5
:10EA40003896EE0FFF1FE40FF51F25913491FA0160
:10EA5000E20FF31F2491222309F3E2CF8F929F92BA
:10EA6000AF92BF92CF92DF92EF92FF920F931F93DC
:10EA7000CF93DF93E091630430916204E31373C09A
:10EA8000C22F6A017B015C01809159028823A1F1A8
:10EA90000E94366201E08E3309F000E00C2B802FDB
:10EAA0008270882EE114F10409F46FC0E70190E24E
:10EAB000992E882009F441C0CE010F945BA114E087
:10EAC000180F4EE300FF40E26091600480E00E9476
:10EAD000E36F64E1611BC5010E94C7718BE50E9471
:10EAE000F16ECE01882089F10E94ED6E8DE50E94C5
:10EAF000F16E892D0E94F16E80916104882399F155
:10EB00002091630480911E0690911F062817190614
:10EB100051F5EF28E9F460E0C6010E94AD62DF9193
:10EB2000CF911F910F91FF90EF90DF90CF90BF900A
:10EB3000AF909F908F900C944362FE010190002053
:10EB4000E9F7EC1B13E01E0FBCCF0E942F73CECF52
:10EB500010925A02C114D10411F0F601199581E006
:10EB600080935A02DCCF809163048F5F80936304AB
:10EB7000DF91CF911F910F91FF90EF90DF90CF9099
:10EB8000BF90AF909F908F90089580E298E40E948C
:10EB90000A75EC018EE7982E8CCF0F931F93CF93BD
:10EBA000DF938C01EB0185E29EE40E940A759F933E
:10EBB0008F938CE591E89F938F93DF93CF930F947E
:10EBC000B4A2C80FD11D47E050E0B801CE010F94A8
:10EBD0008DA31F820F900F900F900F900F900F90AA
:10EBE000DF91CF911F910F9108950F931F93CF93B2
:10EBF000DF93CDB7DEB763970FB6F894DEBF0FBED5
:10EC0000CDBF3091630420916204321338C08B0170
:10EC1000209159022223A9F0BE016F5F7F4F0E940D
:10EC2000CD750E943662482F6091600480E00E949A
:10EC3000E36F62E1CE0101960E9417738EE70E9496
:10EC4000F16E809161048823D1F02091630480915A
:10EC50001E0690911F062817190689F460E0C80166
:10EC60000E94AD620E94436263960FB6F894DEBFC5
:10EC70000FBECDBFDF91CF911F910F91089580916D
:10EC800063048F5F80936304EFCFCF93DF93EC0136
:10EC900020E030E04CE852E460916D1270916E1209
:10ECA00080916F12909170120F94C5A460936D12B1
:10ECB00070936E1280936F129093701260E070E008
:10ECC00080EA91E40F940A4A0E94BD630E94F66FA5
:10ECD0008DEE91E60E940A75AC0160E080E00E9432
:10ECE000D76F8881882339F061E080E00E942A6F25
:10ECF000CE010E942F7385E699E30E940A75AC014C
:10ED000062E080E00E94D76F83E49BE20F943E09AB
:10ED1000DF91CF910D94B0180F947F658F3F11F163
:10ED200080E00E9408700E94F66F89EA99E50E94CF
:10ED30000A75AC0161E080E00E94D76F80E20E941A
:10ED400072700F947F65682F70E06F5F7F4F072EA2
:10ED5000000C880B990B0E94AB710F942E9D81E0E3
:10ED60000C94087008951F920F920FB60F92112401
:10ED70000BB60F922F938F939F93EF93FF93E09196
:10ED80002603E830E8F4F0E08827E653F9488F4F8F
:10ED90000D94ADA4D276EC76F77605771B772477C1
:10EDA000477759778091280681110AC08091EE0536
:10EDB000880F80932503882319F081E08093260330
:10EDC000FF91EF919F918F912F910F900BBE0F901C
:10EDD0000FBE0F901F901895809124038F5F809332
:10EDE000240390912503981758F382E0E7CF83E03E
:10EDF000809326038FE0809323038FEF86BD81E00D
:10EE000085BD84B58F7E84BDDBCF80912303829541
:10EE1000807F819588BD80912303882321F08150D4
:10EE200080932303CDCF84E0809326038FEF88BDAA
:10EE30008EEF86BDC5CF85E0809326038FEF88BD1A
:10EE400086BD82E085BDBCCF2FEF28BD809128060E
:10EE50008111B6CF809124038F5F8093240390911A
:10EE60002503891708F4ACCF8091EE0590E08F3729
:10EE700091050CF0A5CF86E0809326038FE0809368
:10EE8000230326BD81E085BD84B58061BCCF809120
:10EE900023038295807F819588BD80912303811112
:10EEA000BECF87E08093260380E886BD8FEF88BDC4
:10EEB00087CF1092260380E886BD8FEF88BDC1CF33
:10EEC000CF93C82F682F87E69FE00F94C1A3CC2370
:10EED00019F0CF910D94866D1092F1161092FD16D7
:10EEE000CF9108951092B6030F94560B60930717B5
:10EEF000709308178093091790930A1708958093C9
:10EF0000220380FD1CC010923E0320913E038FEF30
:10EF1000820F8E3FE8F08091A000877F8093A00051
:10EF20001092AD001092AC009FB7222361F0F894CC
:10EF3000809102018062809302019FBF08958FEF4C
:10EF400080933E03E2CFF894809102018F7DF3CF4E
:10EF5000EFB7F8948091A00088608093A00030E023
:10EF6000809172004FEF50E081FF04C04091A800F3
:10EF70005091A900249FC001259F900D349F900DB2
:10EF800011246FEF70E00F9466A47093AD0060934E
:10EF9000AC00EFBF08951F93CF93DF93D09122036E
:10EFA000D1FD1DC01091CC03C1E020E030E048E469
:10EFB00052E460915A0D70915B0D80915C0D9091BF
:10EFC0005D0D0F944EA718160CF0C0E0DE7FCD2B20
:10EFD00081E0111101C080E0C82BC0932203809111
:10EFE0002203DF91CF911F910C947F77EF92FF92D4
:10EFF0000F931F93CF93DF93EC018B017A010E9453
:10F00000DA5581110BC0A801BE01C701DF91CF9174
:10F010001F910F91FF90EF900D94B1A3DF91CF91CD
:10F020001F910F91FF90EF9008950F931F93CF932F
:10F03000DF938C01D62FC72F0F94ABA38F3F980778
:10F0400039F46D2F7C2FC8010F94FBA38D2F9C2FBB
:10F05000DF91CF911F910F9108950F931F93CF933D
:10F060008C01C62F0F949DA38F3F29F46C2FC801EC
:10F070000F94E5A38C2FCF911F910F910895CF93FB
:10F08000DF93EC010F94ABA3BC016F5F7F4FCE0108
:10F09000DF91CF910D94FBA3CF93DF93EC010F94FD
:10F0A0009DA361E0680FCE01DF91CF910D94E5A3A0
:10F0B0002BE0829FC0011124805B924F0F94ABA381
:10F0C00021E0019609F420E0822F0895CF93DF9389
:10F0D000C82FD8E0CF5FC8300CF0C0E08C2F0E9462
:10F0E0005878811103C0D150A9F7CFEF8C2FDF9151
:10F0F000CF91089581EA9DE00F949DA30E946678C8
:10F1000087FD05C0682F81EA9DE00D94C1A3089595
:10F110000F931F93CF93C82F8B0160E474E7823065
:10F1200070F069E374E7843050F061E374E7843091
:10F1300031F069E274E7853011F062E274E7C801EA
:10F140000F9454A18CEF8C0F823028F0C170CF5CEB
:10F15000F801C6831782CF911F910F91089561E046
:10F1600080EC9FE00F94C1A360E08FEB9FE00F94D1
:10F17000C1A360E08EEB9FE00F94C1A360E08DEB34
:10F180009FE00F94C1A360E08CEB9FE00D94C1A3BE
:10F19000CF93C82F82958F700E94485D8C2F8F70FF
:10F1A000CF910C94485D40913C1250913D1290E0FB
:10F1B00080E041155105B1F120913812309139129A
:10F1C00090E080E0F901E55BFF4EA081A23021F4E0
:10F1D00061817281860F971F4150510919F1F90120
:10F1E000E25BFF4EA1919F012B543041A111FACF58
:10F1F000F901E55BFF4E2D3EA1E03A0730F4A19105
:10F20000A111E0CF2F5F3F4FF6CF2D3EE1E03E074B
:10F21000C9F6EBE4F0E19F012B543041A191AA2300
:10F22000D1F3D0CF089580913C1290913D121816E1
:10F2300019060CF043C0019790933D1280933C1245
:10F24000892BA1F48091471090914810892B21F4CB
:10F2500010924A10109249108091491090914A10D2
:10F26000909339128093381281E00895809138127A
:10F27000909139120396FC01E55BFF4E20810196C7
:10F280002111F9CFFC01E55BFF4E8D3E21E0920795
:10F2900040F441919C012F5F3F4F4111E1CFC901E3
:10F2A000F4CFEBE4F0E18D3E21E09207C9F6CF0107
:10F2B0008B54904121912223D1F3D2CF80E0089545
:10F2C000FC0120E03EE2DB014D91BD01403249F0FE
:10F2D000283011F430833196DB0111974C91408333
:10F2E00031962F5F2B3079F71082089540E050E07F
:10F2F000BA010D94942AFC01238121110D94722CE2
:10F30000089590911C06911107C09091C00095FF3F
:10F31000FCCF8093C6000895913031F49091C800DD
:10F3200095FFFCCF8093CE0008958F929F92AF926D
:10F33000BF92EF92FF920F931F93CF93DF93CDB7BE
:10F34000DEB7A0970FB6F894DEBF0FBECDBF611534
:10F3500071058105910599F480E3A0960FB6F894A4
:10F36000DEBF0FBECDBFDF91CF911F910F91FF90F8
:10F37000EF90BF90AF909F908F900C94817900E0B8
:10F38000842E912CB12CA12C9E012F5F3F4F79012F
:10F39000A50194010F9410A4F701E00FF11D608303
:10F3A000B901CA010F5F611571058105910581F7EA
:10F3B0000E0D1F2D111DE016F10659F0F801829176
:10F3C0008F018A3020F4805D0E948179F4CF895CBE
:10F3D000FBCFA0960FB6F894DEBF0FBECDBFDF9176
:10F3E000CF911F910F91FF90EF90BF90AF909F90A2
:10F3F0008F900895CF92DF92EF92FF926B017C0184
:10F40000F7FE0BC08DE20E948179F094E094D094D5
:10F41000C094C11CD11CE11CF11C4AE0C701B6011B
:10F42000FF90EF90DF90CF900C9495798F929F9200
:10F43000AF92BF92CF92DF92EF92FF92CF936B0188
:10F440007C01B42E20E030E0A9010F94BAA587FF1B
:10F4500007C08DE20E948179F7FAF094F7F8F094F2
:10F46000C0E060E070E080E09FE3CB1541F020E079
:10F4700030E040E251E40F94C4A5CF5FF6CF9B018A
:10F48000AC01C701B6010F94C5A46B017C010F94B8
:10F490003DA64B015C014AE00E949579CC2391F195
:10F4A000C501B4010F94299E9B01AC01C701B601AF
:10F4B0000F94C4A46B017C018EE20E948179C1503B
:10F4C00008F120E030E040E251E4C701B6010F94BA
:10F4D0006A9E4B015C010F9436A66B01770FEE0814
:10F4E000FF08C701B6010E94FA79C701B6010F945F
:10F4F0002B9E9B01AC01C501B4010F94C4A46B0108
:10F500007C01DDCFCF91FF90EF90DF90CF90BF9047
:10F51000AF909F908F9008958AE00C9481790E941B
:10F52000817990E080E00895CF93DF93EC01FE01B4
:10F530008491882321F00E9481792196F8CFDF9170
:10F54000CF910895CF92DF92EF92FF92C0905A0D23
:10F55000D0905B0DE0905C0DF0905D0D83E998E735
:10F560000E94947A42E0C701B6010E94167A8BE8A5
:10F5700098E70E94947A6091BC037091BD038091DA
:10F58000BE039091BF0341E00E94167AFF90EF9076
:10F59000DF90CF900C948C7A4F925F926F927F9213
:10F5A0008F929F92AF92BF92CF92DF92EF92FF9293
:10F5B0000F931F93CF93DF93CC24CA94DC2C760156
:10F5C0000EEA1FE093E2892E912CA12CB12C412C44
:10F5D000512C3201D0E0C0E08FEFC81609F45DC0B5
:10F5E000C8010F94ABA3EC01BC01990F880B990BD8
:10F5F0000F942B9E2091730D3091740D4091750DD9
:10F600005091760D0F94C4A52B013C01C701B601A2
:10F610000E94FA7987EE97E70E94947AC501B401B7
:10F620000E94FA7987EE97E70E94947ABE010D2E28
:10F63000000C880B990B0E94FA7987EE97E70E94DD
:10F64000947A20E030E04AE754E4C301B2010F9419
:10F650006A9E0F947A6585E0880E911CA11CB11CEE
:10F660000E5F1F4F8FEFC81AD80AE80AF80A0A3B44
:10F670008FE0180709F0B0CFDF91CF911F910F9164
:10F68000FF90EF90DF90CF90BF90AF909F908F90C2
:10F690007F906F905F904F90089580E298E40E9471
:10F6A000947AB8CF882371F18BED97E70E94947A12
:10F6B0006091901270E090E080E00E94FA79809171
:10F6C00090128430D8F01092901286ED97E70E9445
:10F6D000947A8091901290E00F94976580919012A7
:10F6E00020915B1230915C1230935E1220935D1278
:10F6F0000E94EBFB0E94BD630D94B0188F5F809356
:10F700009012E3CF83EC9CE30E940A7570E060E006
:10F710000E94B9CFE5CFCF93DF9383ED97E70E94A7
:10F72000947AC1E6D2E1688179818A819B8142E045
:10F730000E94167A8FEC97E70E94947A6C817D8103
:10F740008E819F8142E00E94167A8BEC97E70E949F
:10F75000947A688579858A859B8542E00E94167A2D
:10F7600087EC97E70E94947A6C857D858E859F85CE
:10F7700042E00E94167A89E194E60E94947A80E041
:10F780000F948E180F942B9EC7E6DDE02C813D81EF
:10F790004E815F810F94C4A542E00E94167A83ECEB
:10F7A00097E70E94947A81E00F948E180F942B9E15
:10F7B000288539854A855B850F94C4A542E00E945F
:10F7C000167A8FEB97E70E94947A82E00F948E1856
:10F7D0000F942B9E2C853D854E855F850F94C4A587
:10F7E00042E00E94167A8BEB97E70E94947A83E0BE
:10F7F0000F948E180F942B9E288939894A895B892A
:10F800000F94C4A5DF91CF910D947A658AEC96E7A9
:10F810000E94947A60915A0D70915B0D80915C0DFD
:10F8200090915D0D41E00E94167A87EC96E70E9468
:10F83000947A60915D1270915E12072E000C880B15
:10F84000990B0F942B9E41E00E94167A83EC96E769
:10F850000E94947A6091BC037091BD038091BE03B5
:10F860009091BF0341E00E94167A80EC96E70E94D7
:10F87000947A6091591270915A12072E000C880BDD
:10F88000990B0F942B9E41E00E94167A8BEB96E722
:10F890000E94947A60915A0D70915B0D80915C0D7D
:10F8A00090915D0D41E00E94167A88EB96E70E94E8
:10F8B000947A60915D1270915E12072E000C880B95
:10F8C000990B0F942B9E41E00E94167A84EB96E7E9
:10F8D0000E94947A6091F50570E090E080E00E94CB
:10F8E000FA798FEA96E70E94947A6091EE0570E0CB
:10F8F00090E080E00E94FA798BEA96E70E94947A81
:10F9000060918503709186038091870390918803AD
:10F9100041E00E94167A0C948C7A0E94947A0C949E
:10F920008C7A8F929F92AF92BF92CF92DF92EF929A
:10F93000FF920F94560B6B017C012091320222231F
:10F9400009F1409178024130E9F0809114029091E0
:10F950001502A0911602B091170246015701881AAC
:10F96000990AAA0ABB0A30E0A8EEB3E00F943DA4BE
:10F9700086169706A806B9066CF0443031F19CF45F
:10F980004230D4F4C0921402D0921502E0921602D2
:10F99000F0921702FF90EF90DF90CF90BF90AF9062
:10F9A0009F908F900895453069F78EEC91EA0E9400
:10F9B000947A86E998E706C08EEC91EA0E94947AE0
:10F9C00083EC98E70E948D7CDDCF8EEC91EA0E945B
:10F9D000947A8DEA98E7F6CFCF9381EA9DE00F9471
:10F9E0009DA3CBE08C9FC0011124805B924F0F94AC
:10F9F000ABA38156904F803A9F40C8F082E698E7CB
:10FA00000E948D7C81EA9DE00F949DA38C9FC00194
:10FA1000112470E060E0805B924F0F94FBA385E2BD
:10FA200098E70E9485E881E0CF910C940870CF910F
:10FA300008952F923F924F925F926F927F928F9292
:10FA40009F92AF92BF92CF92DF92EF92FF920F936D
:10FA50001F93CF93DF93CDB7DEB7A4970FB6F8947B
:10FA6000DEBF0FBECDBF0F94B0188091420D811143
:10FA700017C081E08093721280913906882349F083
:10FA800080913A06882329F020913B062F8321118B
:10FA900020C081E0809353128DEC98E60F94496763
:10FAA000A4960FB6F894DEBF0FBECDBFDF91CF9105
:10FAB0001F910F91FF90EF90DF90CF90BF90AF908C
:10FAC0009F908F907F906F905F904F903F902F907E
:10FAD00008958BEA9DE00F949DA3182F8EE40E9459
:10FAE000F555082F0E940A568E83002329F087308F
:10FAF00009F4C9C0833029F0133009F0C3C063E0B2
:10FB00006E8380E090E0A0E8BFE38A839B83AC83B0
:10FB1000BD838AEA9DE00F949DA3888F83E40E94B1
:10FB2000F555182F0E940A56112329F0882319F041
:10FB30008B3008F4888F88E50E94F555882309F4F6
:10FB4000ABC00E94855A20E030E048E052E40F94B8
:10FB5000C4A420E030E048EB51E40F94C4A46A87C9
:10FB60007B878C879D8789E50E94F555882309F45A
:10FB70009CC00E94855A20E030E048E052E40F9497
:10FB8000C4A420E030E040EA50E40F94C4A46C8B9D
:10FB90007D8B8E8B9F8B87E50E94F555882309F41A
:10FBA00089C00E94855A2A853B854C855D850F94C6
:10FBB000C5A420E030E048E852E40F94C5A4698F62
:10FBC0007A8F8B8F9C8F88E40E94F555882309F4E7
:10FBD0007AC00E94855A2C893D894E895F890F948D
:10FBE000C5A420E030E048E852E40F94C5A46D8F2E
:10FBF0007E8F8F8F98A30F94A07B80912C02909181
:10FC00002D02A0912E02B0912F0280930A1390939F
:10FC10000B13A0930C13B0930D130F94AA5205EC81
:10FC20001FE0C8010F94ABA3019609F051C00E5F0D
:10FC30001F4F053D8FE01807A1F7212CA9E0B3E184
:10FC4000BAA3A9A3B987A887512C412C312C042D24
:10FC5000842D63E00F944CA4988B6884798410E021
:10FC6000F889F11137C0812F63E00F944CA49111F2
:10FC700031C021103FC17E81733009F470C08F8183
:10FC80008E8737C01E836AE979E989E19FE36A8339
:10FC90007B838C839D833DCF80E090E0A0E8BFEF25
:10FCA0008A879B87AC87BD875ECF60E070E080E885
:10FCB0009FEF6DCF80E090E0A0E8BFE7898F9A8F3B
:10FCC000AB8FBC8F80CF60E070E080E89FE78FCF84
:10FCD0002F80B4CF60E070E080EC9FE7D3011196F5
:10FCE0006D937D938D939C931497BE81B330C1F136
:10FCF0001E86812F0E94B05E4B015C01802F0E9406
:10FD0000B05E6B017C01A50194016A857B858C85C1
:10FD10009D850F944EA718160CF41CC1298D3A8DA1
:10FD20004B8D5C8DC501B4010F944EA718160CF4D1
:10FD300011C1A70196016C897D898E899F890F94D5
:10FD40004EA718160CF406C12D8D3E8D4F8D58A16F
:10FD5000C701B6010F944EA718160CF4FBC03394DC
:10FD60001F5F24E0620E711C173009F079CF6FEF2E
:10FD7000461A560A888599854C969987888797E010
:10FD80004916510409F063CF0F947A92A0915D0651
:10FD9000AF83B091DE03B88781E080935D068AE08F
:10FDA000830D8093DE0381E00E94C96E80E090E0C5
:10FDB000A0EAB0E48093691290936A12A0936B1248
:10FDC000B0936C1265E575E585E591E40F940A4AF8
:10FDD00080E00E9436659CA38BA3312C832D67E0C5
:10FDE0000F944CA4F82E092F682F70E07F876E8740
:10FDF00080FF03C076E0791B072F802F63E00F940C
:10FE00004CA4911105C08F2D0F944CA411E09111B9
:10FE100010E0802F0E94B05E688B798B8A8B9B8B61
:10FE20008F2D0E94B05E4B015C018E81833009F002
:10FE300099C01111C8C027E0AE85BF852A9FF00187
:10FE40002B9FF00D1124E00FF11DEE0FFF1FEE0FA1
:10FE5000FF1FE75FFC4E60E070E080EC9FE761838E
:10FE60007283838394833394E1E33E12B7CF80E0BF
:10FE700090E0A0EAB0E48093691290936A12A09394
:10FE80006B12B0936C1265E575E585E591E40F940E
:10FE90000A4A0F94B018B1E33B1609F43CC28091B2
:10FEA0003D0391E0980F90933D03882309F4D3C15B
:10FEB00060E080E00E94EADC84E396E30E940A7539
:10FEC0000E9485E880E00E94E3E781E08093780269
:10FED00086EE9BE60E9485DC2F8120935D06688577
:10FEE0006093DE0382E00E94C96E0F94B0181092F6
:10FEF0007212D6CD011103C0112309F4BCCE812F9B
:10FF000063E00F9458A4840D952D911D880F991FBF
:10FF10008D53904F0F94ABA3BC01990F880B990B95
:10FF20000F942B9E2AE037ED43E25CE30F946A9E28
:10FF30009B01AC0160910A1370910B1380910C131B
:10FF400090910D130F94C5A4F30161837283838391
:10FF5000948391CEFE85FF2309F402CF222009F479
:10FF6000FECEFECE288939894A895B896A857B85E0
:10FF70008C859D850F944EA7181604F12889398920
:10FF80004A895B89698D7A8D8B8D9C8D0F94BAA57A
:10FF900087FD14C0A50194016C897D898E899F8994
:10FFA0000F944EA7181654F0A50194016D8D7E8D07
:10FFB0008F8D98A10F94BAA587FF05C0112309F46E
:10FFC00052CF211050CF10E0A7E08E859F85A89FCB
:10FFD000F001A99FF00D1124E00FF11FEE0FFF1F9C
:10FFE000EE0FFF1FE75FFC4E4180528063807480FC
:10FFF000C12CD12CE0EAEE2EE0E4FE2E222051F0BE
:020000021000EC
:1000000023E333E343EB5EE3C301B2010F94C5A4E2
:100010006B017C01A70196016091691270916A12CF
:1000200080916B1290916C120F94BAA587FF10C04B
:10003000C0926912D0926A12E0926B12F0926C1226
:1000400065E575E585E591E40F940A4A0F94B018CB
:10005000688979898A899B89609361127093621299
:10006000809363129093641280926512909266124C
:10007000A0926712B092681265E672E181E692E1A1
:100080000E94EE6860E070E086E193E40F940A4A13
:100090000F94B0188091420D882339F07F817093BE
:1000A0005D0688858093DE03FBCC812C912C70E269
:1000B000A72E71ECB72E222051F02A813B814C8172
:1000C0005D81C301B2010F94C4A44B015C01488D52
:1000D000C501B4010F94AA7B81110BC080EA95E59C
:1000E0000E940A759F938F930F945FA20F900F90B9
:1000F000BECE2091691230916A1240916B125091DC
:100100006C12C701B6010F94C4A420E030E0A9012D
:100110000F94BAA587FF36C060E070E080EA90E4F3
:100120006093691270936A1280936B1290936C12B1
:1001300065E575E585E591E40F940A4A0F94B018DA
:10014000488DC501B4010F94AA7B882339F2209110
:10015000691230916A1240916B1250916C1260E0FA
:1001600070E080EA90E40F94C4A42DEC3CEC4CECDD
:100170005DE30F94BAA587FF05C087E397E70F9467
:1001800086A275CEC0906912D0906A12E0906B1270
:10019000F0906C122220A1F0A7019601C301B201D8
:1001A0000F94C4A49B01AC015F776A817B818C8131
:1001B0009D810F94BAA587FF03C08EEF96E7DFCF2E
:1001C0008FEA9FE00F949DA3882309F440C086EA3C
:1001D0009FE00F949DA38823D1F1609185037091D6
:1001E000860380918703909188030E948656209110
:1001F000730D3091740D4091750D5091760D0F94E3
:10020000C4A59B01AC01E7E0AE85BF85EA9FC001B4
:10021000EB9F900D1124080F191F000F111F000FE5
:10022000111F075F1C4EC701B6010F94C4A4D8016B
:1002300011966D937D938D939C9314978091DE031B
:1002400081508093DE0381E00E94C96E0CCE20E0D5
:1002500030E0A901D8CF85E00F946223C12CD12CC6
:1002600090EAE92E90E4F92E80E096E30E940A7568
:100270000E949ADE90E080E00E94B3DD81E00E945F
:10028000C5F980E00F943D23182F60E070E080E80E
:100290009FEB0E94646C81E00F943D23C092691231
:1002A000D0926A12E0926B12F0926C1265E575E5DD
:1002B00085E591E40F940A4A0F94B018812F0F94AA
:1002C0003D2382E00F949C1820E030E040EA50E4A7
:1002D0000F944EA7181644F2EF81E0935D06F8855F
:1002E000F093DE0381E00E940870DD24D394DF9256
:1002F000812C912C5401CC24C394E12CF12C870146
:1003000021E040E050E0BA0181E00E94FA6CD09216
:1003100053120F90C5CB10923D038BA19CA10E945C
:100320001C65109227061092260680E10E944CD58B
:10033000882391F00E94EC7C81EA9DE00F949DA3BC
:100340002BE0829FC0011124805B924F0F94ABA3DE
:1003500090932706809326066091260670912706C3
:10036000072E000C880B990B0F942B9E9058209110
:10037000730D3091740D4091750D5091760D0F9461
:10038000C4A50F94705280EC9FE00F949DA391E060
:10039000813009F090E099834FEB5FE06CE4CE018F
:1003A00001960E942456F82E4EEB5FE062E5CE01E6
:1003B00001960E942456082F4DEB5FE066E4CE01C3
:1003C00001960E942456182F4CEB5FE062E4CE01A8
:1003D00001960E942456212F110F330B082E000C7A
:1003E000990B5C01A21AB30A8F2DFF0C990B280FF1
:1003F000391F46E0429F6001439FD00C1124F12C2D
:10040000E12C002E000C110B081B190BB701665FC5
:100410007C4E3B01460177E07A83D3012D903D90DD
:100420004D905D903D01FD013497FB87EA87B40153
:10043000092C000C880B990B0F942B9E2FE333ECA7
:100440004EE259E30F946A9EA20191010F94C5A454
:10045000AA85BB856D937D938D939C931397BA81E9
:10046000B150BA83800E911EB111D7CFCA0CDB1CDC
:10047000ECE1EE0EF11CF4ECEF16F10439F60F94FA
:100480007A928DE40E94F555882309F484C00E9475
:100490000A562E81273009F094C0882309F491C0B0
:1004A000BB24B394AA24AA94AB0C09A11AA1612C71
:1004B0008EEF882E8B0C6A2D862D0F943B5299243B
:1004C0009394960C81116EC06B2D862D0F943B5228
:1004D000C12CD12C7601712C882381F020E030E0F2
:1004E000A901D8015D966D917D918D919C91909718
:1004F0000F94C5A46B017C0177247394682D862D1D
:100500000F943B52882369F0F8017B972081318159
:1005100042815381C701B6010F94C5A46B017C01D0
:1005200073946A2D892D0F943B52882361F0F80152
:100530002581368147815085C701B6010F94C5A436
:100540006B017C0173946A2D8FEF860D0F943B52E3
:10055000882331F1F8013397208131814281538121
:10056000C701B6010F94C5A46B017C017394672D7C
:1005700070E090E080E00F942B9E9B01AC01C701DE
:10058000B6010F94C4A5D80111966D937D938D93F8
:100590009C93149707C08CEA9DE00F949DA379CF9C
:1005A0007110E5CF692C0C5F1F4FB7E09B1283CF12
:1005B000B394E9A1FAA17C96FAA3E9A3F8E0BF12EB
:1005C00071CF81E0809309138FE40E94F55581116A
:1005D00003C00E940D6A79CC0E940A568111F9CF9E
:1005E0000E94116572CCEC01F8940F943D0E179A9D
:1005F00010923906169A10923A06149A81EB91EAF3
:100600000E94947A86E098E70E948D7C209779F08A
:10061000CE010E948D7CBE0185E99CE00F94FBA376
:1006200062E484E99CE00F94E5A30E94EF65CEEFBD
:10063000D7E7F1CF88E493E00F947F0D80913C12CF
:1006400090913D12892B79F0E0913812F091391296
:10065000E55BFF4E8081813011F0863021F48CEE15
:1006600099E60C948D7C089580913C1290913D12F6
:10067000892B29F00E941A830E941379F5CF1092DA
:1006800039121092381210924A101092491081E0DB
:10069000809353120895EF92FF920F931F93CF937D
:1006A000DF9380910913882389F180E997E70E94FD
:1006B0008D7C8AE797E70E948D7C89E697E70E9408
:1006C0008D7CC7E0DCE1C15058F1CD9F7001112451
:1006D00001E010E086E697E70E94947AF801EE0FB9
:1006E000FF1FEE0FFF1FEE0DFF1DEA5FFC4E608146
:1006F00071818281938145E00E94167A0F5F1F4FBE
:100700000830110539F70E948C7ADDCF8DE997E723
:10071000DF91CF911F910F91FF90EF900C948D7C02
:10072000DF91CF911F910F91FF90EF900895CF929D
:10073000DF92EF92FF926B017C01C0922703D0926F
:100740002803E0922903F0922A0380914303823028
:10075000B1F420E030E040E950E4C7010F94BAA5BD
:1007600087FF14C08091970D9091980DA091990DDD
:10077000B0919A0D803D9740A105B10520F5C701C4
:10078000B601FF90EF90DF90CF9008952AE939E904
:1007900049E95EE3C701B6010F94BAA587FF0AC015
:1007A00020E030E048E351E4C701B6010F946A9EAF
:1007B0006B017C0184E794E70E94947AC701B6013B
:1007C0000F947A65DCCF2AE939E949E95EE3C7018C
:1007D000B6010F94BAA587FDE3CF20E030E040E8F2
:1007E0005EE3C701B6010F946A9E20E030E048E561
:1007F00050E40F94C5A4DCCFCF92DF92EF92FF922A
:10080000CF93909143039817B9F1C82FC090270355
:10081000D0902803E0902903F0902A0320E030E0F4
:10082000A901C701B6010F94BAA5882341F0C0926F
:10083000BB0DD092BC0DE092BD0DF092BE0D87E5D0
:1008400094E70E94947AC13011F1E0F0C23011F1C6
:10085000C09343036091BB0D7091BC0D8091BD0DA1
:100860009091BE0D0E9497836093BB0D7093BC0D59
:100870008093BD0D9093BE0DCF91FF90EF90DF90D0
:10088000CF9008958FE494E70E948D7CE1CF8BE4B4
:1008900094E7FACF87E494E7F7CF0F94B018179A4C
:1008A000E9E3F6E01082169A1182149A80E00E9421
:1008B000FC838FEF9FEF90937302809372022FEF70
:1008C00020936F0290933E0280933D0220933F025B
:1008D000909371028093700290933C0280933B024C
:1008E0000895182FF894CDB7DEB700D0CF90DF90E1
:1008F000EF9088E199E20FB6F894A8958093600094
:100900000FBE909360009FB7F894E2E0F1E0808121
:10091000886080839FBF0F943D0E86E094E70E941D
:100920008D7C8EEF93E70E94947A612F70E090E0C7
:1009300080E04AE00E9495798AEF93E70E94947ADA
:100940008E2DB60190E040E10E94957986EF93E705
:100950000E94947ABE0190E080E040E10E94957987
:100960000E948C7A40E060E072E290E080E00F94B8
:100970008F788CEE99E60E948D7C0E94EF65C82FDF
:10098000729A682F83E09DE00F94C1A380910F06B7
:10099000882319F08C2F0E9471840E94EF651F92AA
:1009A0000F920FB60F92112483E00E94BF841F9212
:1009B0000F920FB60F92112482E00E94BF8441ED86
:1009C00050E065E273E787E69DE00F9437A10F944E
:1009D0002F3A0F9474140E941A648EEC91EA0E94CC
:1009E000947A83E093E70C948D7C44E050E064E1DA
:1009F00070E087E69DE00F948DA343E050E065E250
:100A000073E787E69DE00F947CA1892B09F05DC018
:100A1000E9EEF3E7459155916591749188ED90E089
:100A20000E94A45DEDEEF3E74591559165917491B7
:100A30008CED90E00E94A45DE1EFF3E7649180EE1D
:100A400090E00E942D78E2EFF3E76591749181EEDA
:100A500090E00E941578E4EFF3E76591749183EEDE
:100A600090E00E941578E5EEF3E745915591659188
:100A7000749184ED90E00E94A45D41EC53E760E145
:100A800070E080EB90E00E94F67741ED53E760E183
:100A900070E080EC90E00E94F67741ED50E064E178
:100AA00070E087E69DE00F948DA30E941A640F9476
:100AB0002F3A0F9474148EEC91EA0E94947A89EE86
:100AC00092E70E948D7C81E008950E94DF8464E0BB
:100AD00070E084E190E00E94DA5591E08927089562
:100AE00065E273E787E69DE00F9454A141ED50E085
:100AF00064E170E087E69DE00F94B1A38EEC91EA8B
:100B00000E94947A89ED92E70C948D7CCF93DF93C9
:100B1000EC018991882319F00E948179FACFDF9145
:100B2000CF9108950E9486850C948C7A2F923F92E3
:100B30004F925F926F927F928F929F92AF92BF92ED
:100B4000CF92DF92EF92FF920F931F93CF93DF9399
:100B5000CDB7DEB7A0970FB6F894DEBF0FBECDBFFE
:100B60008FE590E00E946455882309F4A1C00E949B
:100B7000FC548F37910561F48091440590914505AF
:100B800090934305809342058AEC92E70E948D7C06
:100B90006E014FE1C40ED11C992493940E94FC5421
:100BA000181619060CF078C080917312882329F06A
:100BB0000E940566882309F46FC080919303811118
:100BC0006BC020914405309145058091420590917C
:100BD00043058217930711F3F901EE53FB4F808110
:100BE0002F5F3F4F2F7733273093450520934405E0
:100BF0008F3F09F079C080911903882309F471C0EF
:100C000090921803109219031F8E18A280901C0353
:100C1000882021F280911A038F8FF1E0F81518F4E3
:100C200080911B0388A310921C031601822D8C193E
:100C3000881508F0B3CFF10111911F018FE193E006
:100C40000F94B40B17FDF2CF80914710909148108C
:100C50001A3009F44BC11D3009F448C18F35910594
:100C60000CF049C11B3311F490921E0320911E0316
:100C70002111DCCF9C012F5F3F4F30934810209310
:100C800047102091491030914A10255B3F4E820F4A
:100C9000931FFC011383CACF809147109091481095
:100CA000181619060CF451C28091D713811167C22E
:100CB000A0960FB6F894DEBF0FBECDBFDF91CF91E7
:100CC0001F910F91FF90EF90DF90CF90BF90AF906A
:100CD0009F908F907F906F905F904F903F902F905C
:100CE00008959092190390CF90911803992309F4D5
:100CF00058C0893FE9F170F5863F09F44AC0873F43
:100D000009F443C085E992E70E94947A80E992E76A
:100D10000E94947A109117038CE892E710FD02C0AC
:100D200087E892E70E94947A012F027082E892E7A6
:100D300011FD02C08DE792E70E94947A8CE792E75A
:100D40000E948D7C002349F185E480930B02109270
:100D500018035ACF8A3F41F08B3FA1F680911703C9
:100D6000816080931703CECF809117038E7FF9CFD8
:100D700010921C031092180310921703109216037E
:100D80001092190310921503BDCF80911703826052
:100D9000E8CF809117038D7FE4CF90E290930B0210
:100DA000D6CF9091190330911703992331F1E09137
:100DB0001C0330FF49C020911503222309F440C0D1
:100DC00091E09E0F90931C03AE2FB0E0A65EBC4F47
:100DD000FFEFFC9340911603442351F0EE5FE09344
:100DE0001C03E92FF0E0E65EFC4F408310921603EF
:100DF00021502093150310921903E0911C0330FF3A
:100E00006CC090911503992349F121E02E0F209396
:100E10001C03AE2FB0E0A65EBC4F8C9380911603EE
:100E2000882351F0EE5FE0931C03E22FF0E0E65ED2
:100E3000FC4F808310921603915090931503E4CEDB
:100E400042E040931503D7CF91E09E0F90931C038F
:100E5000F0E0E65EFC4F9FEF9083CDCFA82FAF7000
:100E600030E021E0AF3029F0B0E0A050BE4F3C911F
:100E700020E0482F407F403F59F4226020FF13C0FC
:100E80009092150321FF0CC0E2E0E0931503BCCE65
:100E900082958F70A82FB0E0A050BE4F9C91EECFEE
:100EA00090931603B1CE81E08E0F80931C03AE2F7A
:100EB000B0E0A65EBC4F3C933A3009F4A5CE21FFCA
:100EC00003C090921503A0CEEE5FE0931C03E82FC1
:100ED000F0E0E65EFC4F908397CE91E09E0F9093FA
:100EE0001C03F0E0E65EFC4F80838ECE009719F481
:100EF00010921E03DDCE0091491010914A10025B42
:100F00001F4E800F911FFC0110821A83098380916C
:100F10001E038111FDC0F80180818E3409F084C068
:100F20004AE050E0BE016F5F7F4FC80101960F9409
:100F3000289F2B013C01E980FA80F70180818032F3
:100F400031F4FFEFEF1AFF0AFA82E982F4CF8091C1
:100F50003E1290913F12A0914012B0914112019621
:100F6000A11DB11D84159505A605B70549F044E0FE
:100F700050E065EC72E7C7010F947CA1892BA1F4C6
:100F80006AE270E0C7010F94F4A99093BC048093C7
:100F9000BB04009709F441C0F801F12C8E179F079C
:100FA000F1F02191F226FACF81EB91EA0E94947A36
:100FB00080E393E60E94947A60913E1270913F1212
:100FC00080914012909141120E94FA790E948C7A8D
:100FD0000E94AC55109248101092471069CE0E94A2
:100FE0001756F816190639F081EB91EA0E94947AA7
:100FF00081E193E6DFCFE091BB04F091BC04108265
:10100000E980FA8060EC72E7C7010F944BA1892B4D
:1010100039F587E795E60E94F38281EB91EA0E9419
:10102000947A87EE92E6C6CF89819A81FC0120816D
:10103000203221F401969A838983F6CF6AE270E028
:101040000F94F4A9892B39F081EB91EA0E94947AEC
:101050008DEB92E6AFCF44244A94542C3201D0CF8A
:1010600044E050E06BEB72E7C7010F947CA15C0198
:10107000F7018081873481F48091610D853061F0C2
:1010800082E492E10F94B40BF6E0F093610D60E01E
:1010900085EA9FE00F94C1A3AB2821F080913B1219
:1010A000811198CF26E077FC21E080914910909142
:1010B0004A10FC01E55BFF4E208349815A81F8010B
:1010C000DA0140175107A1F501900020E9F79F01CF
:1010D000201B310B0396280F391F2D3EF1E03F07EF
:1010E00079F130934A102093491080913C129091ED
:1010F0003D12019690933D1280933C1277FC08C0FC
:1011000040923E1250923F126092401270924112F1
:1011100010924810109247100E94FC54892B09F439
:10112000C7CD8FE590E00E94645581117FCDC0CD81
:101130006D9161939D01241B350B6111F9CFCACFCD
:1011400010924A1010924910D0CF8091600D60E249
:1011500073E0811102C060ED77E08FE193E00F94BE
:10116000850B882309F4A0CD10921E03109248101D
:101170001092471080EB92E70E948D7C99CD809170
:101180006A16882309F494CD8091471090914810F5
:10119000892B09F08DCD80913C1290913D12892BC5
:1011A00011F410921D0312E001E04091EB165091F2
:1011B000EC166091ED167091EE168091E416909108
:1011C000E516A091E616B091E716481759076A0789
:1011D0007B0708F0C1C080911D038111BDC00F9431
:1011E000C06C40916F16509170166091711670919D
:1011F00072164093EB165093EC166093ED167093B5
:10120000EE1620914710309148108A3061F08D30F1
:1012100051F0833209F487C02F35310524F48F3F14
:10122000980709F087C02115310509F441CD809157
:101230006A16811103C040E050E0BA018091491262
:1012400090914A12481B590BA0914910B0914A1035
:10125000FD01E55BFF4E1083418352831396255BAE
:101260003F4EF901EA0FFB1F1082A55BBF4EFD0147
:1012700001900020E9F73197EA1BFB0BF89480916D
:101280003C1290913D12019690933D1280933C1236
:10129000EC5F8091491090914A10E80FF92FF11DF1
:1012A000F0934A10E093491080916A16882309F45C
:1012B0003DC08091EB169091EC16A091ED16B09187
:1012C000EE168093491290934A12A0934B12B0935A
:1012D0004C12ED3EF14021F410924A101092491048
:1012E000789410921E03109248101092471040916B
:1012F000EB165091EC166091ED167091EE16809100
:10130000E4169091E516A091E616B091E7164817FD
:1013100059076A077B0700F58FE590E00E94645546
:10132000811143CFC5CC00931D037DCF80E090E0B9
:10133000DC01C7CFA9014F5F5F4F50934810409326
:1013400047104091491050914A10455B5F4E240F61
:10135000351FF901838329CF4091EB165091EC168C
:101360006091ED167091EE168091E4169091E5165D
:10137000A091E616B091E716481759076A077B0750
:1013800008F496CC0E94D378892B09F091CC0F9465
:10139000D1658AEA92E60E948D7C0F9422156B013A
:1013A0007C010E9480648CE3882E912CA12CB12CAE
:1013B000C701B601A50194010F9410A4CA01B90197
:1013C000A50194010F9410A47F936F93C701B601F8
:1013D00020E13EE040E050E00F9410A43F932F93B3
:1013E0008CE992E79F938F938E010F5F1F4F1F939E
:1013F0000F930F94B4A28EEC91EA0E94947AC801E4
:101400000E949285C8010E94D9DC0F94E872109264
:1014100056020FB6F894DEBF0FBECDBF8091D81331
:10142000882359F00F9403688091600D882309F494
:101430003FCC86E00F9402303BCC81E00F942773C1
:101440008091D8138111EECFEFCF0F931F93CF93DD
:10145000DF93C82F8091F116813009F449C08230A2
:1014600009F45FC00E9461668111FFC080915D1226
:1014700090915E12009739F42091591230915A12CE
:10148000232B09F4F2C04091330250913402609151
:10149000350270913602411551056105710509F457
:1014A000E4C0892B31F48091591290915A12892B02
:1014B00029F08091AD05882309F43FC18091600D2A
:1014C000882321F040EE52E369E270E08DEA95E076
:1014D0000F94C00B882309F4CAC00F943D0E80E618
:1014E00096E30E940A750E9485E80F946D05BFC0BF
:1014F0000F94476E882309F4B5CF81E09091FE16D2
:10150000911101C080E08093F4168091380E909183
:10151000390E909301178093001782E08093F116A3
:10152000A1CF0F94476E1092F5168091F11682307C
:1015300009F098CF8091F616811140C0D091FE1627
:1015400081E0D11101C080E09091F416891709F46F
:1015500089CF8093F41686EF96E10F94B40BDD23C8
:10156000B1F18091F216882311F1809194038111D9
:101570001EC0809101138130D1F080913E0D909179
:101580003F0D891B8F7099F40E94106681110FC066
:1015900080915E0D843059F08FE59FE00F949DA3FC
:1015A000811105C061E084E697E30E94AD6281E0AD
:1015B0008093F51681E08093590254CF64E670E081
:1015C00086EF96E10F94850B8111B8CF4BCF8091B8
:1015D000F316882379F3809194038111EBCF8091E6
:1015E0003E0D90913F0D891B8F7021F40E94106673
:1015F000882301F3809173128111DCCF8091011354
:101600008130C1F280915E0D8430A1F28FE59FE0C0
:101610000F949DA38111CECF88E794E69F938F937B
:101620008EE594E69F938F930F945FA21092F3162A
:101630001092F21660E070E0CB010F94DE6560E07E
:1016400070E0CB010E94886685E69FE00E944C789E
:1016500081E09FE00E943F788EE59CE60F94496709
:101660000F900F900F900F90A5CF1092AD05809125
:101670003C1290913D12039714F40E94968590912C
:101680003E0D80913F0D981781F08091610D86305D
:1016900061F468E873E182E492E10F94850B88239A
:1016A00021F082E492E10F94B40B409144035091F5
:1016B000450360914603709147034115510561054B
:1016C000710509F03FC04091370250913802609196
:1016D000390270913A024115510561057105A9F071
:1016E00088E493E00F94C00B882379F090913E0D2D
:1016F00080913F0D981309C0C11107C0179A10922D
:101700003906169A10923A06149AC0915512909181
:101710003F0D80913E0D981701F180913F0D9EE69F
:10172000899FF0011124EC55F94FC08190913E0D35
:10173000981799F08F5F8F70F9CF8DEA95E00F942D
:101740007F0D95CF88E493E00F94C00B882309F4B4
:10175000BACF8AEE97E70E94F382CC2309F4BEC089
:1017600080913F0390914003A0914103B0914203C7
:10177000892B8A2B8B2B81F40F94560B605E7C4F48
:101780008F4F9F4F60933F037093400380934103BB
:1017900090934203CFEF0FC00F94560B00913F037D
:1017A000109140032091410330914203601771076B
:1017B0008207930778F38091B603882309F497C0D2
:1017C000C093650280915F04811107C081E080931E
:1017D0005F040F94F59610925F048091A60588230C
:1017E000C9F11092A6054FB7F8948091A405282F4F
:1017F000082E000C330B37FF03C0319521953109BA
:10180000243031050CF476C0982F87FF02C093E096
:10181000980F9595959520911E0630911F06290FDA
:10182000311D97FD3A9530931F0620931E0683784D
:1018300087FF03C081508C6F8F5F8093A4054FBFDB
:1018400086E00F94622380915902811103C081E0E8
:10185000809359028091A705882361F00E9440730C
:10186000E0910604F0910704309721F080915A022C
:10187000811119952091CF1330E0A8EEB3E00F94B9
:101880003DA4AB01BC0180ED93E10F94C00B882314
:1018900099F08091CE1380FD0E94067C8091CE133A
:1018A00082FD0E948B7B8091CE1381FD0E94E564B6
:1018B00080ED93E10F947F0D8091600D811102C046
:1018C0000E94917C40E355E760E070E08CE893E093
:1018D000DF91CF911F910F910D94C00B10923F0398
:1018E00010924003109241031092420364CFC093C0
:1018F0001D0668CF1092A4054FBF80E0A2CFCF9302
:10190000DF93EC010F94A53781E00E94258A80E0E7
:101910000E94C96E209799F0C233D10540F062E36E
:1019200070E080E090E00F94230BE297EBCFBE01D4
:1019300090E080E00F94230BD0E0C0E0E3CFDF9194
:10194000CF910895CF93DF93C82FDFEF0F94A53782
:1019500081E00E94258A8091FF128F3FD9F4809107
:101960009412843021F4809197128111EFCF8091ED
:10197000D2129091D312019749F78091F912909168
:10198000FA128932904811F360E089E290E80F94EE
:101990005475DCCFD093FF12853039F4CF3FF9F284
:1019A00061E08C2F0F94899DD1CF8430C1F6DF91F7
:1019B000CF910895FF920F931F93CF93DF93EC0184
:1019C000F62E662309F44BC00F945BA18C01C8016D
:1019D0000E946455882309F453C080914910909166
:1019E0004A10FC01E55BFF4E23E02083825B9F4EA3
:1019F000BE01FF20E9F10F9454A18EEC91EA0E9400
:101A0000947A8FE992E60E94947A8091491090919D
:101A10004A10825B9F4E0E9486858AE792E70E9469
:101A20008D7C8091491090914A100496080F191FDF
:101A30000D3E81E01807F9F010934A100093491009
:101A400080913C1290913D12019690933D128093AB
:101A50003C12DF91CF911F910F91FF900895FC01EF
:101A600001900020E9F731978F01081B190BAFCFC8
:101A70000F9408AAC2CF10924A1010924910E0CFDA
:101A800081EB91EA0E94947A8FE992E60E94947A1F
:101A9000CE01FF2059F00E94947A8FE791EADF91FE
:101AA000CF911F910F91FF900C948D7C0E948685A1
:101AB000F4CFCF93DF93309163042091620432130B
:101AC00020C0EB01BC0180915902882319F080E20B
:101AD0000E94567280916104882399F020916304DA
:101AE00080911E0690911F062817190651F4209721
:101AF00021F061E0CE010E94DA8CDF91CF910C944D
:101B00004362809163048F5F80936304DF91CF9180
:101B100008950F931F93CF93DF93D62F8C01C0E0CE
:101B2000F8018591949128E6883C920721F4209150
:101B30000113213019F461E00E94DA8CCF5F0E5F4F
:101B40001F4FDC13EDCFDF91CF911F910F910895BF
:101B5000CF93DF93CDB7DEB76E970FB6F894DEBFA5
:101B60000FBECDBF9E012C5D3F4FF90141915191B8
:101B70009F016EE170E0CE0101960F94F3A260E048
:101B8000CE0101960E94DA8C6E960FB6F894DEBFF5
:101B90000FBECDBFDF91CF9108952F923F924F920C
:101BA0005F926F927F928F929F92AF92BF92CF92ED
:101BB000DF92EF92FF920F931F93CF93DF93CDB7F6
:101BC000DEB7C356D1090FB6F894DEBF0FBECDBF46
:101BD00082E0809378020091381210913912025BF2
:101BE0001F4E45E050E066E571E8C8010F947CA106
:101BF000892B09F09BC18091600D882309F44DC0A9
:101C000085E69EE70F94EB39882379F08091BD0437
:101C10001F928F9382E095E69F938F930F945FA21C
:101C20000F900F900F900F9008C081E69EE70F94E1
:101C3000EB39882341F01092080481E08093780208
:101C40000E941A833AC28EE59EE70F94EB398823EF
:101C500021F18091BB049091BC0461E003960F9444
:101C6000B0710F94C06C8C0180916F1690917016BA
:101C7000A0917116B09172168093EB169093EC16AA
:101C8000A093ED16B093EE16802F0E9481790A3052
:101C9000110539F70F94D165D0CF8CE491E80F94FA
:101CA000EB398111CACF88E491E80F94EB3988238E
:101CB00021F14091B9035091BA032CE3249FC00154
:101CC000259F900D11249F938F934091B7035091BE
:101CD000B803249FC001259F900D11249F938F93DB
:101CE00086E397E69F938F930F945FA20F900F90D8
:101CF0000F900F900F900F90A0CF83E491E80F9476
:101D0000EB39882311F18CE89FE00F949DA381119A
:101D100010C061E083E69CE60E94DA8C60E085EA10
:101D20009FE00F94C1A360E08FE79CE00F94C1A3F4
:101D300084CF813009F081CF0F94DA1682E492E1EA
:101D40000F94B40B0F94620B78CF8CE391E80F944F
:101D5000EB39882321F080E00F9400956ECF86E365
:101D600091E80F94EB3981110E94EF6583E391E8CC
:101D70000F94EB398823A9F044E150E065E17DE060
:101D8000CE0101960F948DA38C89882329F088E2D7
:101D900091E80F9486A251CFCE0101960F942CAA00
:101DA0004CCF84E291E80F94EB39882329F088E145
:101DB00091E80E948D7C41CF84E191E80F94EB394A
:101DC000882319F085EF90E8F4CF80EF90E80F9426
:101DD000EB39882319F00E940D742FCF8DEE90E817
:101DE0000F94EB39882379F081EA9DE00F949DA34D
:101DF0002BE0829FC001112470E060E0805B924F75
:101E00000F94DFA31ACF8AEE90E80F94EB39882362
:101E100051F00E94F66F40E070E060E084E690E0F0
:101E20000F945525D8CF86EE90E80F94EB39882390
:101E3000E1F086E50E94F555882309F4FECE0E9464
:101E4000175611E0892B09F410E00F94B018809117
:101E5000091390E01817190609F4EFCE109309132F
:101E600089E692E10F94953AE8CE8FED90E80F94D1
:101E7000EB39882309F4E1CE84E40E94F5558823E8
:101E8000A1F00E94855A20E030E04AE754E40F9424
:101E90006A9E20E030E040E05FE30F94C5A40F9419
:101EA0003DA6CB010E940FE9C8CE8BED90E80F94C0
:101EB000EB39882349F18091600D882329F18091C5
:101EC000BB049091BC0402969093BC048093BB0425
:101ED0000E94855A6B017C016FEF87EA9DE00F94A9
:101EE000C1A320E030E04AE754E4C701B6010F94F3
:101EF0006A9E20E030E040E05FE30F94C5A40F94B9
:101F00003DA685EA9DE07CCF85EA9DE00F94ABA3DA
:101F1000BC0190E080E00F94299E20E030E04AE789
:101F200054E40F94C4A50F947A6587CED8018C91A0
:101F3000873411F00C94C19A1093BC040093BB0435
:101F40000E94175690935603809355038B34910546
:101F500009F445C60CF04BC18430910509F4AAC5BB
:101F60000CF0C5C097FDCFC002970CF0A2C10E9433
:101F7000B1548C010E94AC5B6091170670911806F9
:101F80008091190690911A060F94299E6B017C018D
:101F900040906D1250906E1260906F12709070129F
:101FA0008090350690903606A0903706B09038069F
:101FB000A5019401C301B2010F94C4A420E030E054
:101FC00048EC52E40F946A9E9B01AC01C701B60134
:101FD0000F944EA71816D4F4A3019201C501B401C1
:101FE0000F94C4A420E030E048EC52E40F946A9EC1
:101FF000A70196010F94C5A40F943DA66093170600
:10200000709318068093190690931A068091E90D33
:10201000882309F446C188E50E94F555811141C124
:1020200089E50E94F55581113CC18AE50E94F5556C
:10203000811137C185E40E94F555882309F431C127
:1020400020916D1230916E1240916F12509170126A
:10205000609135067091360680913706909138066A
:102060000F94C4A46B017C012DEC3CEC4CEC5DEBBB
:102070000F94BAA587FF07C180911B0681110C94AC
:10208000FEB90F94B0188091350690913606A09154
:102090003706B091380680936D1290936E12A0931C
:1020A0006F12B09370128DE692E10F94623A9091A4
:1020B0001B0681E089270F94E98FCD59DF4F0FB6BA
:1020C000F894DEBF0FBECDBFDF91CF911F910F916E
:1020D000FF90EF90DF90CF90BF90AF909F908F9048
:1020E0007F906F905F904F903F902F900895853133
:1020F000910509F4D9C0FCF48A30910509F423C58F
:102100000B9709F424C58091381290913912825BA3
:102110009F4E9F938F931F9287E48F9388E596E657
:102120009F938F930F945FA20F900F900F900F903B
:102130000F900F90B9C08C31910509F40AC54E97E4
:1021400011F70F94B01881E0809371120E943665E8
:102150008C0180E090E0A8E4B4E480937A0290934C
:102160007B02A0937C02B0937D0243E060E070E0CC
:1021700080E291EC0F94AA7B7090691260906A12D1
:1021800050906B1240906C12B0906512A090661245
:102190009090671280906812F0906112E090621245
:1021A000D0906312C09064128EE694E40E940A7587
:1021B0004F925F926F927F928F929F92AF92BF9257
:1021C000CF92DF92EF92FF929F938F9381E197E6F8
:1021D0009F938F930F945FA2C8010E941C65109279
:1021E00071120FB6F894DEBF0FBECDBF5DC088354B
:1021F000910509F459C0F4F48135910511F40C945A
:10220000079A5CF48C34910509F40CC5803591056E
:1022100009F079CF0E94197D47C08635910511F4E8
:102220000C940B9A8735910509F06DCF80E10E94DF
:102230003FD53AC08C35910511F40C94179A74F47B
:102240008A35910511F40C94109A8B35910509F09B
:102250005ACF8091571287600C94139A8236910559
:1022600011F40C94AE9A8336910509F04CCF10927C
:10227000600D60E084EC9FE00F94C1A382E00E94B7
:10228000C96E0C94BD9A2DEC3CEC4CEC5DE3C7019F
:10229000B6010F944EA7181624F480911B068111E5
:1022A000F0CEC8010E948B6A10925603109255031B
:1022B000C4CC0E94B1542E969FAF8EAF2E970E9431
:1022C000AC5B89E40E94F555882309F4A0C30E9401
:1022D000855A60934D0370934E0380934F03909300
:1022E00050038AE40E94F555C12CD12C7601882335
:1022F00021F00E94855A6B017C01C0925103D0925B
:102300005203E0925303F0925403E0915503F0918D
:102310005603A496FFAFEEAFA49780904D03909024
:102320004E03A0904F03B0905003A7019601C50142
:10233000B4010F9461A724966CAF7DAF8EAF9FAFB1
:10234000249760918E0270918F02072E000C880BEB
:10235000990B0F942B9E20917A0230917B02409131
:102360007C0250917D020F946A9E2EE333EC4EE284
:1023700059E30F946A9E68AF79AF8AAF9BAF80E153
:10238000E1E6F2E1DE01119601900D928A95E1F706
:10239000A5019401505828A739A74AA75BA7D701E0
:1023A000C601B0588CA79DA7AEA7BFA729813A81C7
:1023B0004B815C8128962CAF3DAF4EAF5FAF289725
:1023C000C501B4010F94C5A462966CAF7DAF8EAF0A
:1023D0009FAF62978D819E81AF81B8852C968CAF1F
:1023E0009DAFAEAFBFAF2C979C01AD01C701B60149
:1023F0000F94C5A466966CAF7DAF8EAF9FAF669706
:1024000029853A854B855C8560913106709132064D
:1024100080913306909134060F94C4A46A966CAFF1
:102420007DAF8EAF9FAF6A972091290630912A0623
:1024300040912B0650912C066E962CAF3DAF4EAFBF
:102440005FAF6E9762962CAD3DAD4EAD5FAD6297BE
:102450006E966CAD7DAD8EAD9FAD6E970F94C4A49E
:102460006B017C0180912D0690912E06A0912F0684
:10247000B0913006A2968CAF9DAFAEAFBFAFA29722
:1024800066962CAD3DAD4EAD5FAD6697BC01CD01FE
:102490000F94C4A44B015C0130902B0E20902C0EA5
:1024A00090912D0E9CABA0912E0EACAFB091330E3F
:1024B000B8ABA701960168A579A58AA59BA50F943D
:1024C0006A9E2B013C01A50194016CA57DA58EA5FA
:1024D0009FA50F946A9E9B01AC01C301B2010F94AA
:1024E000C5A42B013C01A501940168A579A58AA585
:1024F0009BA50F946A9E4B015C01A70196016CA5F8
:102500007DA58EA59FA50F946A9E9B01AC01C50178
:10251000B4010F94C4A4A30192010F9444A56B01CC
:102520007C0120E030E0A9010F94BAA587FF0AC022
:102530002BED3FE049EC50E4C701B6010F94C5A470
:102540006B017C016091340E7091350E611571053F
:1025500009F461C290E080E00F94299E9B01AC01D8
:102560006BED7FE089EC90E40F94C4A524962CAD2C
:102570003DAD4EAD5FAD24970F946A9E5B018C011B
:102580006091360E7091370E61157105E1F090E0A3
:1025900080E00F94299E20E030E040E752E40F9461
:1025A0006A9E9B01AC0168AD79AD8AAD9BAD0F947D
:1025B000C4A53B014C019501A8010F94BAA587FF62
:1025C00002C05301840140902F0E5090300E609055
:1025D000310E7090320E9501A801B201C3010F9423
:1025E0004EA7181684F09501A801632D722D8CA9B1
:1025F0009CAD0F94BAA52501380187FF04C0432C78
:10260000522C6CA87CACA496EEADFFADA49732978B
:1026100051F42BED3FE049EC50E4C701B6010F94B3
:10262000C4A46B017C016E962CAD3DAD4EAD5FAD8B
:102630006E9728966CAD7DAD8EAD9FAD28970F94AB
:10264000BAA5811123C0A2962CAD3DAD4EAD5FADB4
:10265000A2972C966CAD7DAD8EAD9FAD2C970F944F
:10266000BAA5811113C020E030E0A901C701B6016D
:102670000F94BAA581110AC02BED3FE049EC50E45C
:10268000C701B6010F94C5A46B017C01A701960197
:1026900024966CAD7DAD8EAD9FAD24970F946A9E50
:1026A0006A962CAD3DAD4EAD5FAD6A970F9461A7B4
:1026B0004B015C012FE632E143E85AE30F94BAA5DF
:1026C00087FD9EC19201A301C501B4010F94C4A569
:1026D0000F94A3A50F943DA67DAB6CAB6230710542
:1026E00008F45EC12E964EAD5FAD2E97452B09F4D2
:1026F00057C190E080E00F94299E4B015C01AC0132
:102700009B01C701B6010F94C4A52B013C01A50193
:1027100094016A966CAD7DAD8EAD9FAD6A970F94B6
:10272000C4A528966CAF7DAF8EAF9FAF28972D853F
:102730003E854F85588960913506709136068091A7
:102740003706909138060F94C4A4A50194010F9404
:10275000C4A52C966CAF7DAF8EAF9FAF2C97A30115
:102760009201C301B2010F946A9E6B017C01AC011E
:102770009B01C301B2010F946A9E20E030E040EC5F
:1027800050E40F94C4A59B01AC01C301B2010F94A6
:10279000C4A46CAF7DAF8EAF9FAF20E030E040E0CF
:1027A0005FE3C701B6010F946A9E9B01AC0160E034
:1027B00070E080E89FE30F94C4A424966CAF7DAFD3
:1027C0008EAF9FAF249722242394312CD8A8DA947B
:1027D00058A9511125C1B10190E080E00F94299EC4
:1027E000A30192010F946A9E6B017C010F94BFA517
:1027F0006CA77DA78EA79FA7C701B6010F9485A8D8
:102800004B015C01C0904D03D0904E03E0904F030C
:10281000F0905003F7FAF094F7F8F0948091510398
:1028200090915203A0915303B091540388AB99AB9C
:10283000AAABBBABA70196016CA57DA58EA59FA5F4
:102840000F946A9E68A779A78AA79BA728A939A988
:102850004AA95BA9C501B4010F946A9E9B01AC0112
:1028600068A579A58AA59BA50F94C5A468A779A793
:102870008AA79BA7A7019601C501B4010F946A9E80
:102880006B017C0128A939A94AA95BA96CA57DA582
:102890008EA59FA50F946A9E9B01AC01C701B6014E
:1028A0000F94C4A46CA77DA78EA79FA79091330E09
:1028B00098AB28A539A54AA55BA562966CAD7DAD00
:1028C0008EAD9FAD62970F94C5A469837A838B8385
:1028D0009C832CA53DA54EA55FA566966CAD7DADF0
:1028E0008EAD9FAD66970F94C5A46D837E838F8355
:1028F000988728962CAD3DAD4EAD5FAD2897698584
:102900007A858B859C850F94C5A469877A878B8788
:102910009C872C962CAD3DAD4EAD5FAD2C976D8553
:102920007E858F8598890F94C5A46D877E878F8754
:10293000988BCE0101960E944C6A2E96AEADBFAD2B
:102940002E972A163B06F8F0E984FA840B851C853D
:102950002D813E814F81588569817A818B819C814F
:102960003F922F92E1E6F2E1FF93EF9388AC99ACAE
:10297000AAACBBACFE013D966F010F94BC3A0F9020
:102980000F900F900F908091420D811139C0FFEF91
:102990002F1A3F0A2CA93DA92215330509F016CF9D
:1029A00089E296E00E944C6AE0903106F09032068F
:1029B000009133061091340620912D0630912E0699
:1029C00040912F06509130066091290670912A0699
:1029D00080912B0690912C061F921F92E1E6F2E166
:1029E000FF93EF9388AC99ACAAACBBACA5E3CA2E1D
:1029F000A6E0DA2E0F94BC3A0F900F900F900F9034
:102A00000E94E85488E493E00F947F0D4DCC60E081
:102A100070E0CB015ECCA32CB22C0CA91CADB0CDC8
:102A200028A539A54AA55BA56CAD7DAD8EAD9FAD42
:102A30000F946A9E4B015C012CA53DA54EA55FA598
:102A400024966CAD7DAD8EAD9FAD24970F946A9E9C
:102A50009B01AC01C501B4010F94C5A47B018C019D
:102A600028A539A54AA55BA524966CAD7DAD8EAD94
:102A70009FAD24970F946A9E4B015C012CA53DA548
:102A80004EA55FA56CAD7DAD8EAD9FAD0F946A9EDA
:102A90009B01AC01C501B4010F94C4A468A779A738
:102AA0008AA79BA7D8AAC701D8018CA79DA7AEA7C4
:102AB000BFA7FFCE80E50E94F555C12CD12C760131
:102AC000882331F00E94855A0F943DA66B017C014A
:102AD00083E50E94F555882361F00E94855A20E025
:102AE00030E04AE754E40F946A9E0F943DA66B01D0
:102AF0007C01C114D104E104F10441F080915D0630
:102B0000873021F08DE297E60E9485DC0F94B018A3
:102B10000F94560BC60ED71EE81EF91E88E493E0EC
:102B20000F947F0D0F94560B6C157D058E059F0538
:102B300008F0BACB0F94A53780E00E94258A80E088
:102B40000E94C96EEFCF81E00F94E98FADCB80E09A
:102B5000FBCF88E50E94F555382E412C512C3201CF
:102B6000882321F00E945D562B013C0189E50E94DB
:102B7000F555282E882371F10E945D566CA77DA71C
:102B80008EA79FA78AE50E94F555D82E812C912CFF
:102B90005401882321F00E945D564B015C0187E5BA
:102BA0000E94F55588A78F93CD2CECA4FDA40EA50B
:102BB0001FA5222DB301A201832D0E94FA6C0F9054
:102BC000311072CB211070CB38A531116DCBD110E3
:102BD0006BCB20CB1CA61DA61EA61FA6D3CF08E23A
:102BE00010E0F8E0EF2EF7E6FF2E602F70E090E0A7
:102BF00080E00F94299E0E9486569F938F937F9327
:102C00006F931F930F93FF92EF920F945FA20F5F4A
:102C10001F4F0FB6F894DEBF0FBECDBF0F361105A4
:102C200021F742CB0F949010811105C087EC90E8FA
:102C30000E948D7C39CB82E00E944CD5811107C067
:102C40008AED99E30E940A750E9485E82DCB809158
:102C50003906882341F080913A06882321F0D090EC
:102C60003B06D11008C081E0809353128DEC98E6AA
:102C70000F94496719CB81E999E30E940A750E9474
:102C800085E88AEC9FE30E940A7541E060E00E94BB
:102C9000A3E681116EC080E090E0A0EAB0E48093EA
:102CA000691290936A12A0936B12B0936C1260E059
:102CB00070E088E492E40F940A4A80E090E0A8E48F
:102CC000B2E48093691290936A12A0936B12B0934E
:102CD0006C1280E090E0A4E3B3E4809365129093DB
:102CE0006612A0936712B093681260E070E088E407
:102CF00092E40F940A4A0F94B01880EA9FE30E946E
:102D00000A750E9485E8E4E0FCE985919591A5911A
:102D1000B4918093651290936612A0936712B0935A
:102D20006812E0E0FCE985919591A591B4918093BA
:102D3000611290936212A0936312B093641260E0E8
:102D400070E088E492E40F940A4A0F94B01881E08E
:102D50008F93812C912C5401CC24C394E12CF12C21
:102D6000870120E040E050E0BA0180E00E94FA6C68
:102D70000F9020E030E04CE052E4609185037091C8
:102D8000860380918703909188030F944EA71816AD
:102D90000CF076C08091600D811172C080E090E0EF
:102DA000A8ECB2E48093691290936A12A0936B121C
:102DB000B0936C1260E070E088E492E40F940A4AE9
:102DC0000F943D0E19821A821B821C821D82CE0135
:102DD00001960F947F0DE3E2FE2E06E51EE720E04C
:102DE00030E04CE052E4609185037091860380915D
:102DF0008703909188030F944EA71816C4F583E4B7
:102E000099E30E940A750E949ADE42E864E080E03D
:102E10000E94E36F1F92FF92609185037091860379
:102E200080918703909188030F9436A67F936F93C8
:102E30001F930F930E94DB6E81E80E94F16E88EE73
:102E400093E00E947F8C0E94A27A40E053E567E005
:102E500070E0CE0101960F94C00B0F900F900F9071
:102E60000F900F900F90882309F4B9CFD12C81E0F7
:102E70000E940870D11004C080E00E9492F914CA28
:102E80000F94B01881E0809371120E94087089EA53
:102E900090E80E948D7C8090850390908603A0909E
:102EA0008703B090880320E030E040EA50E4C50199
:102EB000B4010F94C4A50F9436A625E0269FA00167
:102EC000279F500D1124BA01550F880B990B0F94B1
:102ED0002B9E1B017C0120E030E04CE052E40F947B
:102EE000BAA587FF06C0212C312C6CE0E62E72E4D7
:102EF000F72E222D332D4E2D5F2DC501B4010F94D9
:102F00004EA7181664F420E030E040EA50E4622D49
:102F1000732D8E2D9F2D0F94C5A41B017C01FF9254
:102F2000EF923F922F928FEE96E69F938F930F949E
:102F30005FA220E030E040EF51E4622D732D8E2D32
:102F40009F2D0F94C4A420E030E04CE852E40F948D
:102F5000C5A40F9436A670935A126093591284E058
:102F600080935D0681E08093DE0389E795E40E940B
:102F70000A750E9485DC80E090E0A0EAB0E48093CE
:102F8000691290936A12A0936B12B0936C1260E076
:102F900070E088E492E40F940A4A80E090E0A0EAAE
:102FA000B1E48093611290936212A0936312B09384
:102FB000641280E090E0A0E7B2E480936512909301
:102FC0006612A0936712B093681260E070E088E424
:102FD00092E40F940A4A8AE999E9A9E1BEE3809351
:102FE000691290936A12A0936B12B0936C1260E016
:102FF00070E088E492E40F940A4A0F94B0180F909E
:103000000F900F900F900F900F90209185033091AB
:1030100086034091870350918803622D732D8E2D76
:103020009F2D0F944EA718163CF488EE93E00E9453
:103030007F8C0E94A27AE9CF60E086EA9FE00F943D
:10304000C1A380E090E0A0EAB0E48093691290937D
:103050006A12A0936B12B0936C1260E070E088E487
:1030600092E40F940A4AE0E0FCE985919591A591DC
:10307000B4918093611290936212A0936312B09303
:103080006412E4E0FCE985919591A591B491809357
:10309000651290936612A0936712B093681260E075
:1030A00070E088E492E40F940A4A0F94B01843E069
:1030B00060E070E080E89FEB0F94AA7B811105C06F
:1030C0000E9492F910927112EFC89091691298A71C
:1030D000A0916A12ACA7B0916B12B8ABE0916C12E0
:1030E000E8AFEF93BF93AF939F9382EE96E69F93E3
:1030F0008F930F945FA20F900F900F900F900F90EF
:103100000F904EEA842E4FE0942E53E2C52ED12C20
:103110000FEF1FEFB6010D2C000C880B990B0F94CD
:103120002B9E2B013C01DF92CF92C80102969F9308
:103130008F9326EA36E63F932F930F945FA25801B0
:103140005FEFA51AB50A0F900F900F900F900F9098
:103150000F9011F40C940CBA70E060E0C4010F946D
:10316000DFA3A3019201622D732D8E2D9F2D0F944D
:10317000BAA5181644F485E0A816B10411F00C9411
:1031800018BA05E010E0580197E2A91A98EFB90AB9
:10319000AA0CBB1C85E0809F1001819F300C11247C
:1031A0000D5F1F4F2AE9422E29E9522E29E1622E96
:1031B0002EE3722E3DE6832E36E6932EC80102974B
:1031C00005970CF0D4C0B101635D7F4F072E000C52
:1031D000880B990B0F942B9E6B017C011F930F930F
:1031E000A9E9B6E6BF93AF930F945FA20093DE0305
:1031F00020E030E040EF51E4C701B6010F94C4A4D1
:1032000020E030E040E251E40F946A9E20E030E09C
:1032100040EA50E40F94C4A520E030E048E452E4D2
:103220000F94C5A40F9436A670935A126093591246
:1032300080E090E0A0EAB0E48093691290936A1273
:10324000A0936B12B0936C1260E070E088E492E49B
:103250000F940A4A20E030E040EA51E420936112E2
:1032600030936212409363125093641280E090E0B6
:10327000A0E7B2E48093651290936612A093671260
:10328000B093681260E070E088E492E40F940A4A18
:103290004092691250926A1260926B1270926C1294
:1032A00060E070E088E492E40F940A4A0F94B0184A
:1032B0000F900F900F900F9020918503309186030F
:1032C0004091870350918803C701B6010F944EA720
:1032D00018163CF488EE93E00E947F8C0E94A27A3C
:1032E000EBCF80E090E0A0EAB0E480936912909385
:1032F0006A12A0936B12B0936C1260E070E088E4E5
:1033000092E40F940A4AE0E0FCE985919591A59139
:10331000B4918093611290936212A0936312B09360
:103320006412E4E0FCE985919591A591B4918093B4
:10333000651290936612A0936712B093681260E0D2
:1033400070E088E492E40F940A4A0F94B01843E0C6
:1033500060E070E080E89FEB0F94AA7B95E0290E77
:10336000311C0F5F1F4F811104C00E9492F981E050
:10337000A7CE78A56CA598A988AD272F362F492F01
:10338000582F6091691270916A1280916B1290911E
:103390006C120F94C4A4F62EE72ED82EC92E2091BD
:1033A000730D3091740D4091750D5091760DD701CC
:1033B000F6016B2F7A2F8F2F9E2F0F946A9E0F94FA
:1033C00036A66CAB7DAB8EAB9FABCF92DF92EF920C
:1033D000FF92809188038F93809187038F938091D0
:1033E00086038F93809185038F939F928F920F9482
:1033F0005FA26CA97DA9C5010F94DFA3A2E0AA0E6C
:10340000B11C0FB6F894DEBF0FBECDBFD7CE0E9461
:103410004B830C94549180E10E94EAD40C94549113
:1034200080915712887F809357120C945491B4EC7A
:10343000CB2EB2E0DB2E8E010C5D1F4F5801EE2427
:10344000E394F12CD6018D916D010E94F555F501A3
:1034500081935F01882391F00E94855AF701EE0F56
:10346000FF1FEE0FFF1F349721E030E02C0F3D1FB0
:10347000E20FF31F60837183828393833FEFE31A2C
:10348000F30A45E0E416F104E9F69FA0FCA09920B8
:1034900001F120E030E0A9016D857E858F85988956
:1034A0000F94BAA5811115C0F11013C08DA181111F
:1034B00010C08EA181110DC010926D1210926E126B
:1034C00010926F121092701281E0809321040C947C
:1034D00054910F94B018CE0101965C015FEBC52E9C
:1034E0005DE0D52E61E6E62E62E1F62E380193E02E
:1034F000690E711CD8018D918D01882389F0F60128
:103500002081318142815381D5016D917D918D91D1
:103510009C910F94C5A4F701608371838283938388
:10352000F4E0AF0EB11C24E0C20ED11C34E0E30E77
:10353000F11C60167106F1F6992061F08D859E856B
:10354000AF85B88980936D1290936E12A0936F121D
:10355000B09370120F94CA480C94549181E08093F8
:10356000600D61E084EC9FE00F94C1A31092BB0357
:1035700060E08FEF9FE00F94C1A30E944FD70C949F
:1035800054918D3411F00C940EB91093BC04009337
:10359000BB04F801319681918032E9F38930D9F387
:1035A00080538A3030F01F930F9385E990E80C9494
:1035B0000C8E0E9417569093410D8093400D8E3BC8
:1035C000910511F40C94FFA50CF031C38C349105D6
:1035D00011F40C94E8A40CF0DFC18C31910511F4C6
:1035E0000C941FA30CF0F4C08531910509F440C779
:1035F0000CF05AC08131910509F42FC7DCF4029711
:1036000008F493C68091381290913912825B9F4ED4
:103610009F938F931F928DE48F9388E596E69F93F7
:103620008F930F945FA20F900F900F900F900F90B9
:103630000F90DEC68231910511F40C94AAA644972E
:1036400009F781E08093780288E496E60E948D7CF9
:1036500084E50E94F555182F8CE40E94F55500E092
:1036600080FB00F910FB01F98DE594E10E94767969
:1036700083E2EDE5F4E1DE01119601900D928A9569
:10368000E1F720E050E040E0BE016F5F7F4F8FED3B
:1036900092E00F945B69CE0101960E947B798AE3E8
:1036A00096E60E948D7CA4C68831910509F4F1C686
:1036B00084F48631910509F4DFC6479709F0A2CF5B
:1036C0008091BB049091BC0461E004960F94B071AA
:1036D0008FC68A31910509F422C70CF042C704EC69
:1036E00012E0F2E4AF2EF2E0BF2EA4E2CA2EA2E076
:1036F000DA2EB8E1EB2EB2E0FB2E87EC882E82E0CA
:10370000982EF80181918F010E94F555882321F1AF
:103710000E94855AD6014D905D906D907C90A301DA
:1037200092010F94BAA587FD11C00E94855AF70136
:103730004080518062807380A30192010F944EA754
:10374000181624F00E94855A2B013C01D5014D9298
:103750005D926D927C921397B4E0AB0EB11CE4E0E5
:10376000CE0ED11CF4E0EF0EF11C8016910649F646
:1037700083E50E94F555882311F40C94E9B20E9468
:103780000A56811135C680E090E0A8E4B2E4809347
:10379000420290934302A0934402B093450280E01A
:1037A00090E0AEE3B3E48093460290934702A09387
:1037B0004802B093490280E090E0A0EAB1E480932F
:1037C0004A0290934B02A0934C02B0934D0210C654
:1037D0008C32910511F40C94F0A30CF08FC08F3152
:1037E000910509F4D3C70CF052C08D31910509F44D
:1037F000FFC54E9709F006CF8091D813882309F4AE
:10380000F7C50F94D1650091BB041091BC040C5F07
:103810001F4F8091D813882309F4EAC587E696E103
:103820000F94722C1092D7131DA30CA3CE01849673
:103830000F942B71882309F4DBC54CA15DA1609125
:1038400080147091811419821C8222E0CE010196AD
:103850000F949D548111FBC610E0CE0101960E9489
:103860007B79112309F40AC78CE19EE70E94947AC0
:103870008CA19DA10E9492851092EB161092EC16DD
:103880001092ED161092EE160F94EF6EB1C58032C5
:10389000910509F401C78A9709F0B4CE83E50E9427
:1038A000F555882309F4A4C50E940A56082F80E51F
:1038B0000E94F5551DE0882319F00E940A56182F22
:1038C000EAE6F0E88491811709F492C5319630E870
:1038D000E638F307B9F7163009F07FC700935512A1
:1038E00061E0812F0E942ED1602F812F0E9400D194
:1038F000602F70E0812F0E945FD17AC58F329105D1
:1039000009F497C75CF58D32910509F482C78E974B
:1039100009F078CE80914816882309F485C7CE0136
:1039200001960F943478882309F479C789810E941D
:1039300081798EE20E9481798A810E9481798EE26A
:103940000E9481798B810E9481798EE20E94817927
:103950008C810E9481790E948C7A4AC589349105B4
:1039600009F490C78B34910511F40C94E2A48834C7
:10397000910509F047CE83E50E94F555882309F4A7
:1039800072C70E940A56882309F46AC7813009F079
:103990002FC58093610D2CC58B36910511F40C94C5
:1039A000A1A60CF0ABC08435910511F40C94AAA625
:1039B0000CF05DC08F34910511F40C9430A50CF01F
:1039C00047C08D34910511F40C94FBA48E349105FD
:1039D00009F018CE0E941066882311F40C9400A5FB
:1039E00060911706709118068091190690911A0639
:1039F00028EE33E040E050E00F9410A4122F032F84
:103A0000F42EE52E0F9422152CE330E040E050E038
:103A10000F9410A4B901CA0141ED58E521EC38E535
:103A20009F938F937F936F935F934F93EF92FF9248
:103A30000F931F933F932F9381EB95E69F938F9363
:103A40000F945FA20FB6F894DEBF0FBECDBFD0C4F7
:103A50008235910511F40C94A4A68335910509F0E3
:103A6000D1CD80915712886080935712C1C48C3594
:103A7000910511F40C9413A734F58535910511F4D3
:103A80000C94FAA68635910509F0BCCD83E50E9419
:103A9000F555882309F4ACC40E94855A20E030E033
:103AA0004AE754E40F946A9E0F943DA66093330254
:103AB0007093340280933502909336028DEA95E03C
:103AC0000F947F0D95C48936910511F40C9483A54C
:103AD00014F00C9493A68836910509F093CD83E5F4
:103AE0000E94F555882309F483C40E94855A0F94D7
:103AF00036A670935E1260935D127AC48537910585
:103B000011F40C9493A8BCF58037910509F4E8C72B
:103B1000D4F48D36910511F40C94AFA58E36910531
:103B200009F070CD8EE40E94F555882309F460C435
:103B30000E945D5660933E1270933F128093401234
:103B40009093411255C48237910511F40C9490A8BA
:103B500014F40C949DA78337910509F053CD86E5A5
:103B60000E94F555882311F40C94BCA78CEE98E8BC
:103B70000E948D7C3DC48B37910511F40C94EBA809
:103B80000CF048C08637910511F40C94A3A8873730
:103B9000910509F037CD8EE595E60E94947A0E9452
:103BA0008C7A86E595E60E94947A1E9B02C00C945E
:103BB000DBA881E595E60E94947A0E948C7A8FE3D7
:103BC00095E60E94947A1D9B02C00C94DFA881E5C3
:103BD00095E60E94947A0E948C7A87E395E60E948B
:103BE000947A1C9B02C00C94E3A881E595E60E94A0
:103BF000947A0E948C7A8FE295E60E94947A0199D9
:103C000002C00C94E7A881E595E60E94947A0E9490
:103C10008C7AEEC38C38910509F466C78B3991050F
:103C200009F47DC78D37910509F0ECCC58CD843A65
:103C300041E0940711F40C940EAC0CF044C2823EA7
:103C4000910511F40C9498AA0CF06BC18E3C91056F
:103C500011F40C94A7A90CF0B1C08B3C910511F4A0
:103C60000C9431A95CF5883C910511F40C94EEA8F4
:103C7000893C910509F0C6CC04EC12E0B7E6EB2EC6
:103C8000BDE0FB2E88ECC82E82E0D82ED8018D91A5
:103C90008D010E94F555882349F00E94855A0F94A2
:103CA0003DA6F70164A375A386A397A3F4E0EF0EE6
:103CB000F11CC016D10651F70C9492A78C3C9105CB
:103CC00011F40C9450A98D3C910509F09BCC83E52F
:103CD0000E94F555882351F00E94855A6093A30DE8
:103CE0007093A40D8093A50D9093A60D84E50E947A
:103CF000F555882351F00E94855A6093A70D709363
:103D0000A80D8093A90D9093AA0D82E40E94F55509
:103D1000882361F00E94855A0F943DA66093AB0DF5
:103D20007093AC0D8093AD0D9093AE0D88E50E941D
:103D3000F555882391F00E94855A6093B30D7093D6
:103D4000B40D8093B50D9093B60D6093AF0D709345
:103D5000B00D8093B10D9093B20D89E50E94F55599
:103D6000882351F00E94855A6093B30D7093B40D6F
:103D70008093B50D9093B60D8AE50E94F555882382
:103D800051F00E94855A6093B70D7093B80D8093DF
:103D9000B90D9093BA0D85E40E94F555882309F476
:103DA00027C30E94855A0E9497836093BB0D70932E
:103DB000BC0D8093BD0D9093BE0D1AC3813D91053E
:103DC00011F40C94F5A95CF58F3C910511F40C9459
:103DD000C3A9803D910509F015CC83E50E94F555F6
:103DE000882351F00E94855A6093F60D7093F70D69
:103DF0008093F80D9093F90D86E40E94F555882381
:103E000009F4F6C20E94855A0E9415656093FA0D66
:103E10007093FB0D8093FC0D9093FD0DE9C28C3DDA
:103E2000910511F40C9438AA8D3D910511F40C9470
:103E300077AA863D910509F0E5CB80E50E94F5550E
:103E4000882311F40C9424AA0E94855A2B013C016A
:103E500083E50E94F555882311F40C942EAA0E9444
:103E6000855A4B015C018EE40E94F555D090330ECB
:103E7000882329F00E94855A0F943DA6D62E82E50C
:103E80000E94F555E090340EF090350E882329F00D
:103E90000E94855A0F943DA67B0186E40E94F55549
:103EA0000091360E1091370E882329F00E94855A12
:103EB0000F943DA68B0120E030E0A901C301B201BF
:103EC0000F94BAA518160CF093C220E030E0A901B7
:103ED000C501B4010F94BAA587FD8AC2A50194015A
:103EE000C301B2010F94BAA587FD82C240922B0E86
:103EF00050922C0E60922D0E70922E0E80922F0EEC
:103F00009092300EA092310EB092320ED092330EBB
:103F1000F092350EE092340E1093370E0093360E69
:103F200067C28033A1E09A0711F40C9473AB0CF0D4
:103F300078C08D32E1E09E0711F40C94FAAAB4F532
:103F4000803F910509F454C28C32914009F05ACB5C
:103F500080E50E94F55508EE13E0882389F00E9461
:103F6000855A20E030EC4AE555E40F94BAA50CEAF6
:103F70001DE087FF05C00E94855A0F943DA68B0166
:103F800083E50E94F555882311F40C94F2AA0E944F
:103F9000855A0F943DA66115710511F00C94F4AA91
:103FA000B80190E080E00F94230B22C28E3231E002
:103FB000930711F40C94ECAB8F32914009F022CBB3
:103FC00085E40E94F55510E000E0882359F00E9436
:103FD00017568C01C12CD12C6CE8E62E62E4F62E2B
:103FE00097FD06C0C12CD12C76E1E72E73E4F72EA5
:103FF00083E50E94F555882321F00E94855A6B01C4
:104000007C0183E40E94F555882311F40C94FCABE9
:104010000E9417569C01A801C701B6010F940234F3
:10402000E7C1803951E0950711F40C9400AC04F518
:104030008E35B1E09B0711F40C943FB78F3591405A
:1040400009F0E0CA83E50E94F555882371F00E94CB
:10405000855A0F9436A66130710511F40C9475B72A
:104060006230710511F40C9497B70F942217C0C1F8
:104070008539F1E09F0711F40C9404AC863921E0F6
:10408000920711F40C9409AC8339914009F0BACA33
:1040900080910113813009F0ABC185E40E94F55590
:1040A00081110E940A5686E40E94F55581110E94F2
:1040B0000A560F946379882309F49AC160E080E07E
:1040C0000F94679C95C1803C42E0940711F40C94D6
:1040D00081B80CF057C08832A2E09A0711F40C9412
:1040E000CDAE4CF5863FE1E09E0711F40C9416AC82
:1040F0006CF4843F21E0920711F40C9412AC853FDC
:10410000914009F07FCA0E94F58472C1873F41E067
:10411000940711F40C941AAC8D3F914009F072CAC7
:104120000E940D748EEC91EA0E94947A8EE49FE7CF
:104130000E94947A5DC18A35A2E09A0711F40C942A
:10414000F8B25CF48835E2E09E0711F40C9402AFFB
:104150008935924009F4C3CA55CA8D3B22E09207C3
:1041600011F40C94B0B78E3B32E0930711F40C9429
:104170004DB88B35924009F045CA60E080E00E945E
:10418000EADC36C18C3553E0950711F40C941AB46F
:104190000CF042C0833CB2E09B0711F40C948DB844
:1041A0007CF4813CF2E09F0711F40C9487B8823CC8
:1041B000924009F027CA82EC92E00E944B5A18C143
:1041C000853C32E0930711F40C94D6B814F40C94A7
:1041D000AAB88235934009F015CA188683E50E9473
:1041E000F555882311F40C9400B30E940A56182F39
:1041F000883010F40C9405B38AE29FE70E94947A09
:104200004AE067E070E080E090E00E9495798FEDF1
:1042100092E00E949285ECC08438A3E09A0711F4E2
:104220000C9490B60CF04DC08D35E3E09E0711F470
:104230000C94A4B48E35934009F0E4C90E94855AC9
:1042400020E030E040E251E40F946A9E0F943DA6D6
:104250006C5A633011F40C94AAB510F00C943CB570
:10426000613011F40C9465B5623009F0C1C08091E1
:104270000113EEE3F9E7813011F0E0E4F9E705918D
:10428000149180E50E94F555882311F40C9499B59A
:104290000E945D56F090EA03FF2009F4A9C0601760
:1042A000710709F4A5C089E897E30E940A758C019B
:1042B0008BE597E30E940A754F2DB8010E94D0E864
:1042C00097C08C3823E0920709F492C0803A33E01B
:1042D000930709F450C28B38934009F093C988E5DD
:1042E0000E94F555882339F00E94855A0F9436A60E
:1042F00080E00F9413188AE50E94F555882339F061
:104300000E94855A0F9436A681E00F94131885E415
:104310000E94F555882309F46BC00E94855A0F94BA
:1043200036A6CB010F94131763C00091BB04109104
:10433000BC040E5F1F4F80E50E94F555C12CD12CA7
:104340007601882321F00E945D566B017C0183E594
:104350000E94F555882351F00E945D569B01AC01E7
:10436000A8EEB3E00F9432A46B017C01C8010F5F8B
:104370001F4FDC014C914032C9F326E020935D06CB
:10438000C114D104E104F104C9F52C912223B1F147
:104390000E94D9DC0F94B01880913A128460809307
:1043A0003A1288E493E00F947F0DC114D104E10424
:1043B000F104D9F10F94560BC60ED71EE81EF91E54
:1043C00084E0809378020F94560B6C157D058E0562
:1043D0009F0510F182E08093780280913A128B7FE2
:1043E00080933A128091D713882391F110925D0641
:1043F0001092410D1092400D0C941D8E8091600D15
:10440000811107C08EE799E30E940A750E9485DC3E
:10441000C1CF10925D06BECF0E9445738111DACFE5
:1044200090E080E00E947F8CCECF1091780284E0F3
:10443000809378020E9440730E944573811105C0E9
:1044400090E080E00E947F8CF7CF10937802C5CF78
:1044500086EE9BE60E9485DCCBCF83E799E30E9442
:104460000A750E9485DC1798169815981498C0CF85
:1044700081E00F942773BCCF1092D7131092D813FA
:104480008EEC91EA0E94947A84EA98E60E948D7CF0
:10449000AFCF0E940566882319F00E94AADCA8CF3E
:1044A0000E94E1E8882309F4A3CF80916A1688234B
:1044B00061F08091EB169091EC16A091ED16B09101
:1044C000EE16892B8A2B8B2B69F40E94685610926A
:1044D000491210924A1210924B1210924C1280E024
:1044E0000E94FC838091D813882331F081E080936F
:1044F000D71385E08093610D0F94DA168091011334
:10450000813009F075CF8091D712882309F470CFDC
:104510008091FE1681116CCF0F942E9D69CF8091F2
:10452000D813882309F464CF83E50E94F5558823C6
:1045300009F45ECF0E945D566B017C01C092EB16C0
:10454000D092EC16E092ED16F092EE160F94E8671A
:10455000C0924912D0924A12E0924B12F0924C1241
:1045600047CF80E50E94F555182F0E9405668823E5
:1045700091F080917312882349F080917902811122
:1045800005C086E49EE70E948D7C32CF8AE39EE7D9
:104590000E948D7C2DCF8091D713882309F44AC0C7
:1045A0001123E1F10F946D6C0E948C7A80EF94E6F8
:1045B0000E94947A6091EB167091EC168091ED1642
:1045C0009091EE164AE00E9495798FE20E948179DF
:1045D0006091E4167091E5168091E6169091E716C9
:1045E0004AE00E9495790E948C7A0F9422152CE360
:1045F00030E040E050E00F9410A4C9016CE370E09B
:104600000F9466A48C0190E080E00E94FA798AE31E
:104610000E948179C8010F949765EACE8091EE13CC
:10462000882329F08EEE93E10E949285BFCF89ED19
:1046300093E1FACF8AE29EE70E948D7CD9CE8091E9
:10464000BB049091BC0404960F94CC77D1CECE01DC
:1046500001960F94C968882309F4FEC861E0CE0171
:1046600001960F94232C009709F4F6C825EEFC015F
:1046700020831C820F941727182FEFC884E09EE731
:104680000E94947A8CA19DA10E9486858EE20E9450
:1046900081790E948C7AACCE8091D71381110F94CE
:1046A000B0180091BB041091BC040C5F1F4F61E275
:1046B00070E0C8010F94F4A9009719F08C010F5F06
:1046C0001F4F80E50E94F555F82E8091BB04909114
:1046D000BC040817190708F4F12C8091D81388231B
:1046E00009F486CE61E06F25C8010F94B07183E5AF
:1046F0000E94F555882399F08091BB049091BC04E9
:104700008017910760F40E945D566093EB167093DA
:10471000EC168093ED169093EE160F94E867809157
:10472000D813882331F081E08093D71385E08093FC
:10473000610DF1105DCE80916A16882361F0809141
:10474000EB169091EC16A091ED16B091EE16892B18
:104750008A2B8B2B69F40E94685610924912109292
:104760004A1210924B1210924C1280E00E94FC836D
:104770000F94DA163DCE8091BB049091BC0421E0E9
:104780002093D61305960F94CC7732CE0F94221532
:104790002CE330E040E050E00F9410A47F936F933F
:1047A0003F932F9386E890E89F938F938E010F5F3E
:1047B0001F4F1F930F930F94B4A28EEC91EA0E94A7
:1047C000947AC8010E949285C8010E94D9DC0FB674
:1047D000F894DEBF0FBECDBF0BCE17FD09CE80C84B
:1047E00080E10E94EAD481EA9DE00F949DA34BE012
:1047F000849FC001112470E060E0805B924F0F94B1
:10480000DFA382E00E94EAD40E941E550E94FD614F
:10481000EFCD8AE50E94F5550F94DB7CE9CD8AE463
:1048200090E80E94947AE4CD86E490E80E948D7C22
:10483000DFCD84E0809378020E94F66F0E9440737F
:104840000F94A53781E00E94258A0E9437DD0E94DF
:1048500045738823A9F30E94F66F0F946D05C8CDA8
:104860001092610DC5CD8091610D1F928F9388E2EA
:1048700096E69F938F930F945FA20F900F900F90E7
:104880000F90B6CD80E50E94F555882321F00E9457
:104890000A5680936F0282E50E94F555882341F005
:1048A0000E94855A0F943DA6709373026093720222
:1048B00081E50E94F555882321F00E940A568093D5
:1048C0003F0283E50E94F555882341F00E94855AF6
:1048D0000F943DA670933E0260933D0283E40E94D4
:1048E000F5558823A9F00E94855A6B017C0120E0D0
:1048F00030E0A9010F94BAA56FEF7FEF181624F4EA
:10490000C701B6010F943DA67093710260937002C7
:1049100084E40E94F5558823A9F00E94855A6B0112
:104920007C0120E030E0A9010F94BAA56FEF7FEF82
:10493000181624F4C701B6010F943DA670933C02EB
:1049400060933B02809171028F93809170028F93EC
:10495000809173028F93809172028F9380916F0286
:10496000282F082E000C330B3F938F938EEC95E687
:104970009F938F9305ED15E61F930F930F945FA2FE
:1049800080913C028F9380913B028F9380913E02F5
:104990008F9380913D028F9380913F02282F082EA4
:1049A000000C330B3F938F9387EC95E69F938F9387
:1049B0001F930F930F945FA20FB6F894DEBF0FBE44
:1049C000CDBF16CD0E94E1E8882309F411CDD0CEE9
:1049D00080918B03813009F00BCD82E080938B03B3
:1049E0000F94560B60930B0670930C0680930D0684
:1049F00090930E06FDCC0F94FE160E948064F8CCB6
:104A000083E50E94F555882351F00E94855A0F9442
:104A10003DA6AB01BC0181EF9FE00F94D3A384E5D9
:104A20000E94F555882351F00E94855A0F943DA6A7
:104A3000AB01BC018DEE9FE00F94D3A381EF9FE00B
:104A40000F94A5A3162F072FF82EE92E8DEE9FE0C9
:104A50000F94A5A34EEA58E52DE938E50C94109D76
:104A60008CE893E00F947F0D83E50E94F555882331
:104A700009F162E270E08091BB049091BC040F9454
:104A8000F4A98C01892BB1F00F5F1F4F62E270E037
:104A9000C8010F94F4A9892B69F0E5E0F6E083E002
:104AA000DF011D928A95E9F742E050E0B801CF019D
:104AB0000F941DAA8CE89FE00F949DA3813009F00C
:104AC00097CC0E94FB65882309F492CC0E9405666E
:104AD000882309F48DCC84E995E60E948D7C88CCEE
:104AE00087E795E60E94F38283E50E94F5558823C7
:104AF00009F47ECC0E94855A0F9436A670935A1200
:104B00006093591275CC82E490E80E94947A0E94D6
:104B1000067C0E94137981E08093531269CC83E56F
:104B20000E94F555882351F00E940A568093CF13B6
:104B3000882371F080ED93E10F947F0D83E40E9450
:104B4000F555882341F00E940A568093CE1350CC2D
:104B50001092D013F3CF81E08093CE1349CC85E738
:104B600096E50E940A750E9485DC81E08093CB0364
:104B70000F94023083E50E94F555882349F00E9486
:104B8000855A0F9436A670935E1260935D1205C02D
:104B900082E50E94F5558111F2CF0F94560B6B01FF
:104BA0007C0160915D1270915E12072E000C880BE3
:104BB000990B0F942B9E11E020915A0D30915B0DB3
:104BC00040915C0D50915D0D0F944EA718160CF09E
:104BD00010E01093590DC701B6010F94427485E699
:104BE00096E50E940A750E9485DC82E08093CB03E3
:104BF0000F94023088E493E00F947F0DF9CB87E5A2
:104C000096E50E940A750E9485DC83E08093CB03C1
:104C100081E00F94023083E50E94F555182F882318
:104C200049F00E94855A0F9436A670935A126093E9
:104C3000591205C082E50E94F5558111F2CF0F94FB
:104C4000560B6B017C0110925F0D609159127091AF
:104C50005A12072E000C880B990B0F942B9E01E023
:104C60002091BC033091BD034091BE035091BF031E
:104C70000F944EA718160CF000E00093590D809188
:104C80005F0D81111AC06091591270915A12072E4E
:104C9000000C880B990B0F942B9E2091BC03309134
:104CA000BD034091BE035091BF03E091590DEE2327
:104CB00091F00F944EA71816A4F08CE496E50E948C
:104CC0000A750E9485DC84E08093CB0388E493E03E
:104CD0000F947F0D8DCB0F94BAA587FFEECF1111E6
:104CE000ECCF80915E0D823041F30F94560B6C191E
:104CF0007D098E099F09693E73408105910550F039
:104D00008091600D811102C00E94A27A0F94560B0F
:104D10006B017C010F94A53780E00E94258A80E01A
:104D20000E94C96EACCF83E50E94F555882329F017
:104D30000E940A56809355125BCB8FEF80935512D9
:104D400057CB1092551254CB80915712877F809386
:104D500057124ECB83E50E94F555882399F00E94A7
:104D6000855A20E030E04AE754E40F946A9E0F949D
:104D70003DA6609337027093380280933902909376
:104D80003A0236CB88E50E94F5558823D1F00F947E
:104D9000B01888E50E94F555811128C089E50E9468
:104DA000F555882319F0169A10923A068AE50E9462
:104DB000F55585E40E94F555882309F419CB149A1A
:104DC00017CB89E50E94F5558111E1CF8AE50E9454
:104DD000F5558111DCCF85E40E94F5558111D7CFBF
:104DE0000F94B018149A0E944D8402CB179A109217
:104DF0003906D4CF83E50E94F555882309F4F8CA13
:104E00000E94855A20E030E04AE754E40F946A9EFD
:104E10000F943DA66093440370934503809346032B
:104E200090934703E5CA34EC832E32E0932E47E695
:104E3000A42E4DE0B42E10E0F40181914F010E94A8
:104E4000F555882309F467C00E94855A6B017C01DF
:104E5000133009F06AC020E030E040EA51E40F94DA
:104E6000BAA587FF4EC0A70196016091770D70919A
:104E7000780D8091790D90917A0D0F94C4A52B0136
:104E80003C01AC019B016091BB0D7091BC0D809108
:104E9000BD0D9091BE0D0F946A9E6093BB0D7093F3
:104EA000BC0D8093BD0D9093BE0DA3019201609146
:104EB000870D7091880D8091890D90918A0D0F94C6
:104EC0006A9E6093870D7093880D8093890D9093EF
:104ED0008A0D6091B7047091B8048091B9049091E3
:104EE000BA040F94299EA30192010F946A9E0F9415
:104EF0003DA66093B7047093B8048093B90490936F
:104F0000BA04C092770DD092780DE092790DF092AC
:104F10007A0D0F94866DB4E0AB0EB11C1F5F143098
:104F200009F08ACF0F942F3A63CAD5011496CD9217
:104F3000DD92ED92FC921797EECF83E50E94F55536
:104F4000882329F00E940A568093320251CA8EECBF
:104F500091EA0E94947AC0903202D12CF12CE12C7B
:104F60008BE390E80E94947A4AE0C701B6010E9460
:104F700095790E948C7A3CCA85E50E94F555882374
:104F800009F45AC00091BB041091BC040F5F1F4F7D
:104F90001093BC040093BB048091E903882309F4B7
:104FA00027CABE016F5F7F4FC8010E948CD788233C
:104FB00009F41ECA83E197E8DE011196BE01675F1E
:104FC0007F4FFC01459154912D913D91421753071C
:104FD00010F40C9421BA2417350708F409CA029674
:104FE000A617B70771F704CA8FE099E30E940A7504
:104FF000AC0163E080E00E94D76F40E068EE73E0B0
:1050000082E390E00F94552584EF91E00E947F8C1D
:1050100040E068EE73E082E390E00F9455258EE166
:1050200090E00E94B3DD81E00E9408700E94F66F5C
:1050300080E00E94C96EDCC941E150E060E87CE09C
:10504000CE0101960F948DA38DE190E80E94947A91
:105050008CEE98E80E94947A8BE190E80E94947A12
:1050600086E190E80E94947A84E190E80E94947A24
:105070008AE090E80E94947A80EB9FE70E94947AFD
:105080008CEA9FE70E94947A8DE99FE70E94947AC8
:10509000CE0101960E9486858BE89FE70E94947A54
:1050A0008AE89FE70E948D7C1F9221E3F22EFF92F7
:1050B00083EF9DE79F938F930CEA1DE71F930F9358
